:020000040800F2
:100000000020001031E30208FDA2010851A70008FA
:10001000F9A20108F5A20108F1A201080000000000
:10002000000000000000000000000000EDA2010838
:10003000E9A2010800000000E5A2010881BD000856
:1000400099E3020899E3020899E3020899E3020898
:1000500099E3020899E30208959C0108C19D0108F3
:10006000859D0108499D01080D9D0108093300087F
:10007000F9320008E9320008D9320008C932000814
:10008000B5320008A132000899E3020899E302089A
:1000900035A7010899E3020899E30208D19C0108F9
:1000A000D9B4000829B5000899E3020839B5000859
:1000B00019B5000809B5000899E3020899E3020898
:1000C00099E3020899E3020899E3020899E3020818
:1000D00099E302088D930108119301080DBE0008F1
:1000E000599C010899E30208D5A2010899E3020886
:1000F000E9B4000899E30208F9B4000899E302089A
:1001000000000000000000000000000099E3020869
:1001100099E3020899E302084152020825520208B5
:100120008D3200087932000865320008513200082B
:100130003D32000899E302080000000000000000C2
:1001400099E3020899E3020899E30208000000001D
:10015000000000000000000000000000000000009F
:10016000000000000000000099E3020899E3020883
:1001700099E30208000000000000000000000000F9
:080180000000000099E30208F1
:10018800002870B51EDB0928044620DD012303EB97
:1001980083035B00B0FBF3F2092AF8D87BB10E4E5B
:1001A800B4FBF3F00928CCBF57223022A6FB03E5A5
:1001B800024403FB1044EB0801F8012BF0D10023A3
:1001C8000B7070BD2D230B7040420131DBE73030DE
:1001D80001F8010BF3E700BFCDCCCCCC884230B49A
:1001E8004FF001042ED301FB04F4B0FBF4F58D426B
:1001F800F9D284B1AAB901E0B0FBF4F5092DCCBF5E
:10020800572230222A4404FB150003F8012BB4FBC3
:10021800F1F4002CF0D100221A7030BC7047B0FB0A
:10022800F4F5092DCCBF372230222A4404FB1500EF
:1002380003F8012BB4FBF1F4002CF0D100221A7062
:1002480030BC70470546002AEBD1D7E703685A1C33
:1002580002601970704700BF2DE9F047089C2578A7
:10026800002B804689460CBF4FF0200A4FF0300A19
:10027800661C35B3002A29DD334601E0024698B1F1
:1002880013F8011B501E0029F8D1971E60B13D4696
:10029800013D51464046C8476B1C002BF8DC2578C9
:1002A80027EAE770013055B1041B29464046C84784
:1002B800301916F8015B002DF7D1BDE8F087BDE8CD
:1002C800F087002A04DC2846BDE8F0870020EBE729
:1002D800571EDCE783684268D0ED037A00EB8301A0
:1002E8000133934281ED040A836004BF00238360D5
:1002F80000EB830393ED047A036870EE277A9A4241
:10030800C0ED037A77EEC77AC0ED037A0CDA0133D1
:1003180007EE103AF8EEC76AB7EE007A87EEA60A3B
:10032800036030EE070A704707EE102AB8EEC77A66
:1003380087EE870A704700BF90ED057A90ED004A76
:10034800D0ED066AD0ED014AD0ED047A90ED035A5B
:10035800D0ED025AA4EE007AB0EE406AB0EE470A39
:10036800B0EE667AA6EE247A67EEC07AA0EE457AF9
:10037800E6EE257A80ED057AC0ED067A704700BF73
:10038800D0ED057A90ED013AD0ED003AD0ED064A6D
:1003980090ED024A90ED077A90ED035A90ED086AC5
:1003A800D0ED045AC0ED067AF0EE406A27EE830AD3
:1003B800C0ED056AA3EEA60A80ED087AA4EE240A29
:1003C800A5EE470AA5EEC60A80ED070A704700BFEA
:1003D800D0ED007A90ED017A30EE670AE7EE007A08
:1003E800B0EE670AC0ED007A704700BF704700BFE3
:1003F8000A44914214D030B40139551E41F2210209
:1004080011F8014F082380EA042004044CBF82EA53
:1004180040004000013B80B2F7D18D42F0D130BCA2
:10042800704700BF4FF40063838270474FF4006346
:1004380083827047012380F84530704770B40468A0
:10044800037B2268022101FA03F31A4213D042699E
:100458000A495C2000FB02124FF6FE76506852896A
:10046800C5680068296831402960C168D24392B2E2
:100478000A40C260636070BC704700BF0C40002037
:1004880030B40A4B1D7875B1094B002003EBC50544
:100498001A6899885062D4682143D160083323F8D8
:1004A800040CAB42F4D130BC704700BFEC420020D2
:1004B800F042002010B40268047B11680223A340B4
:1004C800194209D00649406800240C7001684FF6AB
:1004D800FE742140016053605DF8044B704700BF13
:1004E800974E0020014B186818F0FABF242000200E
:1004F800F0B5836983B0054613B11A689B881385E4
:100508006869264F8389C3244FF47A734FF0060E27
:100518006E464FF6FF71013703E0013B9BB28B42F9
:100528001DD002899207F8D504734FF47A7302E05C
:10053800A3B28B4213D00289D20703F1FF34F7D557
:10054800027BD2B20EB132700136BEF1000F08D074
:100558000EF1FF3EFF24002FE3D03C78DBE719F0D3
:1005680083FCAB6913B11A689B8893619DF80500F9
:100578009DF801609DF802109DF803409DF8042045
:100588009DF8063041EA062143EA002342EA0422A4
:10059800012029876A87AB8703B0F0BDE8F7020816
:1005A800037C022B01D000207047F0B5836983B02B
:1005B80013B11A689B881385044640F2E9334069F1
:1005C80001E0002B59D00289013B12F0020F9BB2C7
:1005D800F7D0C323037340F2E93301E0002B4CD07A
:1005E8000289013B12F0010F9BB2F7D0037B6069CF
:1005F8004FF0060E83896E464FF47A734FF6FF71FB
:10060800FF2703E0013B9BB28B4233D00289950759
:10061800F8D507734FF47A7302E0ABB28B4229D056
:100628000289D20703F1FF35F7D5027BD2B20EB1AA
:1006380032700136BEF1010EE8D1A36913B11A6810
:100648009B8893619DF804009DF800609DF8011057
:100658009DF802509DF803209DF8053041EA0621D7
:1006680043EA002342EA0522012021876287A38703
:1006780003B0F0BD19F0F8FBDFE719F0F5FBB6E7BA
:10068800037A022B01D000207047F0B5036983B0CC
:1006980013B11A689B881385044640F2E933C06891
:1006A80001E0002B59D00289013B12F0020F9BB2E6
:1006B800F7D0BB23037340F2E93301E0002B4CD0A1
:1006C8000289013B12F0010F9BB2F7D0037BE0686F
:1006D8004FF0060E83896E464FF47A734FF6FF711A
:1006E800FF2703E0013B9BB28B4233D00289950779
:1006F800F8D507734FF47A7302E0ABB28B4229D076
:100708000289D20703F1FF35F7D5027BD2B20EB1C9
:1007180032700136BEF1010EE8D1236913B11A68AF
:100728009B8893619DF804009DF800609DF8011076
:100738009DF802509DF803209DF8053041EA0621F6
:1007480043EA002342EA05220120E18222836383EF
:1007580003B0F0BD19F088FBDFE719F085FBB6E7B9
:100768002DE9F04F87B0019090F85500002840F02F
:100778007185019B1B7C022B00F0E085BB4CBC4DB6
:10078800DFF8F492BB48DFF8F4E24FF0640A4FF068
:10079800100C4FF47A76D9F80430C3F30803002B11
:1007A80040F05684EFF31183002B40F05184216808
:1007B800826800BF23689942F9D12F6806FB07F3C6
:1007C8009B1AB3FBF7F306FB013101270091D9F817
:1007D8000430C3F30803002B40F00084EFF31183C7
:1007E800002B40F0FB832368816800BF2268934296
:1007F800F9D1D5F800B006FB0BF2521AB2FBFBF2A6
:1008080006FB0323009A9B1AB3F57A7FDFD3BAF16C
:10081800010AC0D1019B1B7C022B01F03380DFF859
:1008280058929448DFF854E24FF0640A4FF0100CE5
:100838004FF47A76D9F80430C3F30803002B40F05C
:10084800EB83EFF31183002B40F0E6832168826885
:1008580000BF23689942F9D12F6806FB07F39B1A5A
:10086800B3FBF7F306FB013101270091D9F80430F7
:10087800C3F30803002B40F09483EFF31183002B9C
:1008880040F08F832368816800BF22689342F9D1C2
:10089800D5F800B006FB0BF2521AB2FBFBF206FBCE
:1008A8000323009A9B1AB3F57A7FDFD3BAF1010AC2
:1008B800C0D1019B1B7C022B00F09D87DFF8B8910B
:1008C8006C48DFF8B8E14FF0640A4FF0100C4FF4B1
:1008D8007A76D9F80430C3F30803002B40F0648417
:1008E800EFF31183002B40F05F842168826800BF1A
:1008F80023689942F9D12F6806FB07F39B1AB3FBCB
:10090800F7F306FB013101270091D9F80430C3F34E
:100918000803002B40F02883EFF31183002B40F0ED
:1009280023832368816800BF22689342F9D1D5F8F0
:1009380000B006FB0BF2521AB2FBFBF206FB0323D4
:10094800009A9B1AB3F57A7FDFD3BAF1010AC0D1B6
:10095800019B1B7C022B00F00487DFF81C914548A3
:10096800DFF818E14FF00F0A4FF0100C4FF47A76C9
:10097800D9F80430C3F30803002B40F0F883EFF3F1
:100988001183002B40F0F3832168826800BF23683D
:100998009942F9D12F6806FB07F39B1AB3FBF7F3CB
:1009A80006FB013101270091D9F80430C3F308038D
:1009B800002B40F0BC82EFF31183002B40F0B7828C
:1009C8002368816800BF22689342F9D1D5F800B046
:1009D80006FB0BF2521AB2FBFBF206FB0323009A4A
:1009E8009B1AB3F57A7FDFD3BAF1010AC0D1019916
:1009F80091F84F200B7C042A34BF18261A26022BA4
:100A080000F06786DFF870901A48DFF870E04FF062
:100A18000F0A4FF0100C4FF47A76D9F80430C3F36C
:100A28000803002B40F0F983EFF31183002B40F00B
:100A3800F4832168826800BF23689942F9D12F683E
:100A480006FB07F39B1AB3FBF7F306FB01310127FB
:100A58000091D9F80430C3F30803002B40F04A8210
:100A6800EFF31183002B40F0458209E0946F0020DA
:100A7800986F002010E000E000ED00E0906F00208B
:100A88002368816800BF22689342F9D1D5F800B085
:100A980006FB0BF2521AB2FBFBF206FB0323009A89
:100AA8009B1AB3F57A7FD4D3BAF1010AB5D1019B69
:100AB8001B7C022B00F0C385DFF8DC92B448DFF81A
:100AC800D4E24FF00F0A4FF0100C4FF47A76D9F8B1
:100AD8000430C3F30803002B40F08383EFF3118342
:100AE800002B40F07E832168826800BF236899420A
:100AF800F9D12F6806FB07F39B1AB3FBF7F306FB44
:100B0800013101270091D9F80430C3F30803002B01
:100B180040F0D381EFF31183002B40F0CE8123689E
:100B2800816800BF22689342F9D1D5F800B006FB6E
:100B38000BF2521AB2FBFBF206FB0323009A9B1A34
:100B4800B3F57A7FDFD3BAF1010AC0D1019B1B7CD0
:100B5800022B00F02985DFF840928D48DFF834E257
:100B68004FF00F0A4FF0100C4FF47A76D9F8043092
:100B7800C3F30803002B40F0A482EFF31183002B8A
:100B880040F09F822168826800BF23689942F9D1AA
:100B98002F6806FB07F39B1AB3FBF7F306FB01313B
:100BA80001270091D9F80430C3F30803002B40F063
:100BB8006781EFF31183002B40F06281236881681D
:100BC80000BF22689342F9D1D5F800B006FB0BF2BA
:100BD800521AB2FBFBF206FB0323009A9B1AB3F5E9
:100BE8007A7FDFD3BAF1010AC0D1019B1B7C022BAB
:100BF80000F08184DFF8A0916548DFF898E14FF0B4
:100C0800640A4FF0100C4FF47A76D9F80430C3F325
:100C18000803002B40F03982EFF31183002B40F0DA
:100C280034822168826800BF23689942F9D12F680D
:100C380006FB07F39B1AB3FBF7F306FB0131012709
:100C48000091D9F80430C3F30803002B40F0FB806F
:100C5800EFF31183002B40F0F6802368816800BF12
:100C680022689342F9D1D5F800B006FB0BF2521A6C
:100C7800B2FBFBF206FB0323009A9B1AB3F57A7FBB
:100C8800DFD3BAF1010AC0D1019B1B7C022B00F013
:100C9800E883DFF804913E48DFF8F8E04FF00F0AE8
:100CA8004FF0100C4FF47A76D9F80430C3F30803E8
:100CB800002B40F04082EFF31183002B40F03B8281
:100CC8002168826800BF23689942F9D12F6806FB22
:100CD80007F39B1AB3FBF7F306FB013101270091D9
:100CE800D9F80430C3F30803002B40F08F80EFF3EA
:100CF8001183002B40F08A802368816800BF226836
:100D08009342F9D1D5F800B006FB0BF2521AB2FBA8
:100D1800FBF206FB0323009A9B1AB3F57A7FDFD315
:100D2800BAF1010AC0D1019B1B7C022B00F0508351
:100D3800DFF864801649174F4FF00F094FF0100E77
:100D48004FF47A70D8F80430C3F30803002B40F04E
:100D5800D481EFF31183002B40F0CF8122688E6895
:100D680000BF23689A42F9D1D5F800C000FB0CF304
:100D78009B1BB3FBFCF300FB023300930126D8F85E
:100D88000430C3F308032BBBEFF3118313BB05E057
:100D980010E000E0906F002000ED00E02368D1F83B
:100DA80008A000BF22689342F8D1D5F800B000FB34
:100DB8000BFCACEB0A0CBCFBFBFC00FB03C3009A6E
:100DC8009B1AB3F57A7FDAD3B9F10109BAD107B022
:100DD800BDE8F08FEFF3118A8EF312888A680B68EA
:100DE800DB0344BF3E608A682368D7F800C05FFA17
:100DF8008AFA8AF31188D5F800A09C4400FB0AF30C
:100E08009B1AB3FBFAF300FB0C33D8E7EFF3118816
:100E18008CF3128881680368DB0344BFCEF8007046
:100E280081682368DEF800205FFA88F888F3118863
:100E3800D5F800801A4406FB08F35B1AB3FBF8F3F5
:100E480006FB023367E7EFF311888CF31288816899
:100E58000368DB0344BFCEF8007081682368DEF8BE
:100E680000205FFA88F888F31188D5F800801A44C2
:100E780006FB08F35B1AB3FBF8F306FB0233FBE649
:100E8800EFF311888CF3128881680368DB0344BF91
:100E9800CEF8007081682368DEF800205FFA88F8D1
:100EA80088F31188D5F800801A4406FB08F35B1A0A
:100EB800B3FBF8F306FB02338FE6EFF311888CF3EC
:100EC800128881680368DB0344BFCEF8007081682C
:100ED8002368DEF800205FFA88F888F31188D5F8CF
:100EE80000801A4406FB08F35B1AB3FBF8F306FB11
:100EF800023323E6EFF311888CF3128881680368C4
:100F0800DB0344BFCEF8007081682368DEF8002058
:100F18005FFA88F888F31188D5F800801A4406FB30
:100F280008F35B1AB3FBF8F306FB0233B7E5EFF3FC
:100F380011888CF3128881680368DB0344BFCEF8FC
:100F4800007081682368DEF800205FFA88F888F36B
:100F58001188D5F800801A4406FB08F35B1AB3FB26
:100F6800F8F306FB02333AE5EFF311888CF31288A5
:100F780081680368DB0344BFCEF80070816823688A
:100F8800DEF800205FFA88F888F31188D5F8008029
:100F98001A4406FB08F35B1AB3FBF8F306FB0233AB
:100FA800CEE4EFF311888CF3128881680368DB03C1
:100FB80044BFCEF8007081682368DEF800205FFA2D
:100FC80088F888F31188D5F800801A4406FB08F3DE
:100FD8005B1AB3FBF8F306FB023362E4EFF3118804
:100FE8008CF3128881680368DB0344BFCEF8007075
:100FF80081682368DEF800205FFA88F888F3118892
:10100800D5F800801A4406FB08F35B1AB3FBF8F323
:1010180006FB0233FFF7F6BBEFF311828CF312885D
:1010280087680368D90303D50123CEF800308768A1
:101038002368DEF80010D2B282F311882A681944B6
:1010480006FB02F3DB1BB3FBF2F306FB01310BE4F7
:10105800EFF311828CF3128887680368D90303D5EC
:101068000123CEF8003087682368DEF80010D2B27A
:1010780082F311882A68194406FB02F3DB1BB3FBD1
:10108800F2F306FB0131FFF7A0BBEFF311828CF3FB
:10109800128887680368D90303D50123CEF8003086
:1010A80087682368DEF80010D2B282F311882A68B4
:1010B800194406FB02F3DB1BB3FBF2F306FB013119
:1010C800BDE5EFF311828CF3128887680368D903B2
:1010D80003D50123CEF8003087682368DEF80010B6
:1010E800D2B282F311882A68194406FB02F3DB1B8B
:1010F800B3FBF2F306FB013152E5EFF311868EF3F1
:101108001288D1F808C00B68DA0303D501233B60C5
:10111800D1F808C023683A68F6B286F311882E68B9
:101128001A4400FB06F3A3EB0C03B3FBF6F300FB36
:101138000233009322E6EFF311828CF3128887685A
:101148000368D90303D50123CEF8003087682368E4
:10115800DEF80010D2B282F311882A68194406FB1F
:1011680002F3DB1BB3FBF2F306FB0131B6E5EFF349
:1011780011828CF3128887680368D90303D5012389
:10118800CEF8003087682368DEF80010D2B282F308
:1011980011882A68194406FB02F3DB1BB3FBF2F340
:1011A80006FB0131FFF7FEBBEFF311828CF31288C7
:1011B80087680368D90303D50123CEF80030876810
:1011C8002368DEF80010D2B282F311882A68194425
:1011D80006FB02F3DB1BB3FBF2F306FB0131FFF75F
:1011E80092BBEFF311828CF3128887680368D903E6
:1011F80003D50123CEF8003087682368DEF8001095
:10120800D2B282F311882A68194406FB02F3DB1B69
:10121800B3FBF2F306FB013173E4EFF311828CF3B5
:10122800128887680368D90303D50123CEF80030F4
:1012380087682368DEF80010D2B282F311882A6822
:10124800194406FB02F3DB1BB3FBF2F306FB013187
:10125800FFF7FDBB18F064FB0446002800F09283FA
:10126800036885881A8A15407FF483AA03F13843F6
:101278009B0AA749C5712022C85CA27126F0CCFF41
:10128800A38805952068049304A924F045FAA38847
:101298000199A04ACA60B3FA83F2C2F11F02561C30
:1012A80039D0D1B201F0FC0303F1804303F5803358
:1012B80001F003019E68DFF870E288000F2787407D
:1012C80026EA0706019F21680C374EF822709E60B7
:1012D800D3F808E0904E914FC1F38721814041EA4D
:1012E8000E014FF00108996008FA02FEB118C7F81C
:1012F80000E0082304A804920F7A8DF815308DF8C1
:1013080016808DF8145027F0C1FA854AD35DF02B6A
:1013180000F33D83A388B3FA83F3C3F11F03581C7A
:101328003FF427AA012202FA03F37E490A6813430D
:101338000B60019B1B7C022B7FF420AA019B9B69FD
:1013480013B11A689B881385019B586940F2E933E9
:1013580002E0002B00F0DD820289013B12F0020F4F
:101368009BB2F6D06B23037340F2E93302E0002B03
:1013780000F0CF820289013B12F0010F9BB2F6D038
:10138800037B019B586940F2E93302E0002B00F02F
:10139800BD820289013B12F0020F9BB2F6D0802376
:1013A800037340F2E93302E0002B00F0AF820289B8
:1013B800013B12F0010F9BB2F6D0037B019B9B69A6
:1013C800002B3FF4DBA91A689B889361FFF7D6B915
:1013D800019B9B6913B11A689B881385019B586907
:1013E80040F2E93302E0002B00F0C9820289013B98
:1013F80012F0020F9BB2F6D03823037340F2E933A0
:1014080002E0002B00F0BB820289013B12F0010FC1
:101418009BB2F6D0037B019B586940F2E93302E0A6
:10142800002B00F0A9820289013B12F0020F9BB247
:10143800F6D00123037340F2E93302E0002B00F0F9
:101448009B820289013B12F0010F9BB2F6D0037B0D
:10145800019B9B69002B3FF46BAC1A689B889361D6
:1014680066E4019B9B6913B11A689B881385019BED
:10147800586940F2E93302E0002B00F07A820289D1
:10148800013B12F0020F9BB2F6D03723037340F2F0
:10149800E93302E0002B00F06C820289013B12F074
:1014A800010F9BB2F6D0037B019B586940F2E933E8
:1014B80002E0002B00F05A820289013B12F0020F71
:1014C8009BB2F6D01023037340F2E93302E0002BFD
:1014D80000F04C820289013B12F0010F9BB2F6D05A
:1014E800037B019B9B69002B3FF4D3AB1A689B8855
:1014F8009361FFF7CEBB019A936992F8506013B1DC
:101508001A689B881385019B586940F2E93310E0FB
:10151800001303083D040008E8F70208140401401A
:10152800A03A002000040140603A0020002B00F09F
:101538001A820289013B12F0020F9BB2F6D01923DE
:10154800037340F2E93302E0002B00F00C820289B9
:10155800013B12F0010F9BB2F6D0037B019B586947
:1015680040F2E93302E0002B00F0FA810289013BE6
:1015780012F0020F9BB2F6D0067340F2E93302E094
:10158800002B00F0ED810289013B12F0010F9BB2A4
:10159800F6D0037B019B9B69002B3FF42BAB1A68A9
:1015A8009B889361FFF726BB019A936992F84E6076
:1015B80013B11A689B881385019B586940F2E93377
:1015C80002E0002B00F0C9810289013B12F0020FF2
:1015D8009BB2F6D01A23037340F2E93302E0002BE2
:1015E80000F0BB810289013B12F0010F9BB2F6D0DB
:1015F800037B019B586940F2E93302E0002B00F0BD
:10160800A9810289013B12F0020F9BB2F6D0067342
:1016180040F2E93302E0002B00F09C810289013B93
:1016280012F0010F9BB2F6D0037B019B9B69002B44
:101638003FF491AA1A689B889361FFF78CBA019BC3
:101648009B6913B11A689B881385019B586940F2FE
:10165800E93302E0002B00F07A810289013B12F0A5
:10166800020F9BB2F6D01C23037340F2E93302E069
:10167800002B00F06C810289013B12F0010F9BB234
:10168800F6D0037B019B586940F2E93302E0002B56
:1016980000F05A810289013B12F0020F9BB2F6D08A
:1016A8001823037340F2E93302E0002B00F04C8169
:1016B8000289013B12F0010F9BB2F6D0037B019B1C
:1016C8009B69002B3FF4F8A91A689B889361FFF780
:1016D800F3B98B6913B11A689B881385019B586904
:1016E80040F2E93302E0002B00F02B810289013B34
:1016F80012F0020F9BB2F6D01B23037340F2E933BA
:1017080002E0002B00F01D810289013B12F0010F5D
:101718009BB2F6D0037B019B586940F2E93302E0A3
:10172800002B00F00B810289013B12F0020F9BB2E3
:10173800F6D0067340F2E93302E0002B00F0FE8099
:101748000289013B12F0010F9BB2F6D0037B019B8B
:101758009B69002B3FF456A91A689B889361FFF791
:1017680051B9019B9B6913B11A689B881385019B2A
:10177800586940F2E93302E0002B00F0DC8002896E
:10178800013B12F0020F9BB2F6D06B23037340F2B9
:10179800E93302E0002B00F0CE800289013B12F011
:1017A800010F9BB2F6D0037B019B586940F2E933E5
:1017B80002E0002B00F0BC800289013B12F0020F0E
:1017C8009BB2F6D00123037340F2E93302E0002B09
:1017D80000F0AE800289013B12F0010F9BB2F6D0F7
:1017E800037B019B9B69002B3FF4B7A81A689B8871
:1017F8009361FFF7B2B8019B9B6913B11A689B8884
:101808001385019B586940F2E93302E0002B00F090
:101818008C800289013B12F0020F9BB2F6D06B2339
:10182800037340F2E93301E0002B7ED00289013BCB
:1018380012F0010F9BB2F7D0037B019B586940F26D
:10184800E93301E0002B6DD00289013B12F0020F51
:101858009BB2F7D00023037340F2E93301E0002B79
:1018680060D00289013B12F0010F9BB2F7D0037BD5
:10187800019B9B69002B3FF421A81A689B88936100
:10188800FFF71CB8019B9B6913B11A689B881385E5
:10189800019B586940F2E93301E0002B3FD00289EF
:1018A800013B12F0020F9BB2F7D06823037340F29A
:1018B800E93301E0002B32D00289013B12F0010F1D
:1018C8009BB2F7D0037B019B586940F2E93300E0F3
:1018D80013B30289013B12F0020F9BB2F8D0072321
:1018E800037340F2E93300E0B3B10289013B12F01F
:1018F800010F9BB2F8D0037B019B9B69002B3EF440
:101908008EAF1A689B889361FEF789BF18F0ACFA0E
:1019180054E518F0A9FA34E518F0A6FAECE718F03F
:10192800A3FAD0E718F0A0FAA2E718F09DFA84E726
:1019380018F09AFA55E718F097FA35E718F094FA7C
:1019480005E718F091FAE6E618F08EFAB7E618F00F
:101958008BFA97E618F088FA67E618F085FA48E6F1
:1019680018F082FA16E618F07FFAF7E518F07CFA14
:10197800B7E518F079FA97E518F076FA68E518F0FF
:1019880073FA48E5019A0A4BD3600123CDE4F319B1
:10199800F0211B7E8DF80C3003A803238DF80E5020
:1019A8008DF80F80D1558DF80D3023F07FFEB1E40E
:1019B8003D0400082DE9F04F4269B24C1388DFF866
:1019C800D082B14E23F040031B041B0C13801388F4
:1019D8009BB223F0380343F03003138013889BB283
:1019E80083B043F04003138001900AF081F8DFF8D8
:1019F800A4E2A649844610274FF47A750120DEF840
:101A08000430C3F30803002B40F01D81EFF311836A
:101A1800002B40F018812368D1F8089000BF226895
:101A28009342F8D1D8F800A005FB0AF2A2EB09020C
:101A3800B2FBFAF205FB03239C45E0D0019D284642
:101A4800FEF78EFEAB6913B11A689B881385019B5C
:101A5800586940F2E93302E0002B00F0388102892E
:101A6800013B12F0020F9BB2F6D06A23037340F2D7
:101A7800E93302E0002B00F02A810289013B12F0D1
:101A8800010F9BB2F6D0037B019B586940F2E93302
:101A980002E0002B00F01E810289013B12F0020FC8
:101AA8009BB2F6D01023037340F2E93302E0002B17
:101AB80000F010810289013B12F0010F9BB2F6D0B1
:101AC800037B019B9B6913B11A689B889361DFF8BC
:101AD800C4916E486C4F4FF0640A4FF0100E4FF4EB
:101AE8007A75D9F80430C3F30803002B40F0D4808A
:101AF800EFF31183002B40F0CF802168826800BF8C
:101B080023689942F9D1D8F8006005FB06F39B1ABF
:101B1800B3FBF6F305FB013101260091D9F8043037
:101B2800C3F30803002B56D1EFF31183002B52D1D6
:101B38002368816800BF22689342F9D1D8F800B0C1
:101B480005FB0BF2521AB2FBFBF205FB0323009ACA
:101B58009B1AB3F57A7FE1D3BAF1010AC1D1019B8F
:101B68004A4D5A69484F138823F040031B041B0C45
:101B78001380138823F038031B041B0C138013886D
:101B88009BB243F04003138009F0B2FFDFF804C1B1
:101B980081464FF0100E4FF47A760120DCF80430BD
:101BA800C3F30803002B31D1EFF3118373BB236810
:101BB800A96800BF22689342F9D1D8F800A006FBB3
:101BC8000AF2521AB2FBFAF206FB03239945E5D052
:101BD80003B0BDE8F08FEFF3118C8EF312888168A3
:101BE8000368DA0344BF3E60816823683A685FFA95
:101BF8008CFC8CF31188D8F800C01A4405FB0CF350
:101C08005B1AB3FBFCF305FB0233A0E7EFF311818A
:101C18008EF31288D5F808A02B68DB0344BF386020
:101C2800D5F808A023683A68C9B281F31188D8F8B2
:101C380000101A4406FB01F3A3EB0A03B3FBF1F30C
:101C480006FB0233C2E7EFF3118987F31288D1F854
:101C580008A00B68DB0344BF3060D1F808A02368F4
:101C680032685FFA89F989F31188D8F800901A4424
:101C780005FB09F3A3EB0A03B3FBF9F305FB0233F6
:101C8800DAE600BF946F0020906F002010E000E0BB
:101C9800986F002000ED00E0EFF311828EF31288B8
:101CA80086680368D90302D501233B6086682368E8
:101CB8003968D2B282F31188D8F80020194405FB9C
:101CC80002F39B1BB3FBF2F305FB013124E718F089
:101CD800CBF8D9E618F0C8F8F3E600BF10B490E8DE
:101CE8000600047B40690223A3404B6013685DF83B
:101CF800044B4FF6FE710B40136017F081BBF8B52B
:101D0800174D2B78A52B28D16B78BE2B25D1022215
:101D180029464FF6FF70FEF76BFB124FAC1C22886A
:101D28004AB1A618BE4218D2052A16D92146FEF78E
:101D38005FFB3446F3E721460222FEF759FB0222F5
:101D4800A118FEF755FB0634074B641B1C8041F6AF
:101D58000F53C31A58425841F8BD0020F8BD00BFC0
:101D680000F0030800000408203700202DE9F04F98
:101D7800DFF864914F4F8BB00326A7EB09071822B1
:101D8800002104A82DF0BDFC4B4BCDF81090059711
:101D98001A69120604D5494A5A6002F188325A6013
:101DA80001228DF824203422DA60454B454C1B88EB
:101DB800ADF800300222694604A818F017F902228B
:101DC80069464FF6FF70FEF713FBDFF810A1804657
:101DD8004FF0000B544536D30AAC002524F8245D97
:101DE8000222214604A818F001F9022221464046A1
:101DF800FEF7FEFA40BAC043ADF80800022202A975
:101E080004A818F0F3F8079860B106ABC0F1040213
:101E1800294618442DF075FC069904A818F08CF88A
:101E2800079508909DF82430089A23B122490B6938
:101E380043F080030B61013E2DD0002A9FD1FFF7AC
:101E48005EFF50B332E065888DF80DB0C5F30B0521
:101E5800AB1DADF808302388C3F30B02ADF80A2098
:101E68001B0B062202A904A88DF80C3018F0BEF846
:101E7800062202A94046FEF7BBFA616880462A4658
:101E880004A818F0B3F8616840462A46FEF7B0FA8D
:101E9800143480469EE7002AD1D005201FF0E8FCC4
:101EA800094B0A4A1A600A4B0A4ADA600BB0BDE8C5
:101EB800F08F00BF0000040800200240230167459E
:101EC80007F80208F84B0308FC9F0020EFBEADDEC0
:101ED80000ED00E00400FA0500F0030830500308A4
:101EE8000378202B024600F10100F9D0092BF7D026
:101EF8002D2B2CD02B2B03BF5378B7EE000A0246AC
:101F0800B7EE000AA3F13001C8B209289FED467A5E
:101F180010D8F2EE046A07EE901AF8EEE77A12F893
:101F2800013FE7EE267AA3F13001C8B20928B0EEE6
:101F3800677AF0D92E2B4CD003F0DF03452B0BD05A
:101F4800F7EE007A67EE276A20EE260A7047537884
:101F5800BFEE000A0246D5E710B451782D2959D0B2
:101F68002B290ABF9178501C901C0024A1F1300342
:101F7800092B53D8002303EB830301EB430310F829
:101F8800011FA1F13002092AA3F13003F3D9B3F5F7
:101F98009A7F28BF4FF49A73072B42D9DFED236A43
:101FA8001A46F7EE007A083A072A67EEA67AFAD8B0
:101FB80003F007032BB1F2EE046A013B67EEA67A41
:101FC800FBD124B3C7EE276A5DF8044B20EE260A3E
:101FD80070475378A3F13001C8B2092802F1010211
:101FE800AAD8F2EE046AF0EE665A07EE901AF8EEF6
:101FF800E77A12F8013F87EEA66AA3F13001C8B26A
:10200800092866EEA56A37EE067AEED994E767EEF8
:10201800276AD9E7901C91780124A7E7F7EE007AA0
:10202800CFE7F7EE007AC5E70000000020BCBE4C01
:10203800B5EEC00ADFED317AF1EE10FACCBF30EE22
:10204800270A30EE670ADFED2E7A20EE270A30B530
:10205800FDEEC07A87B017EE904A054684EAE47030
:10206800002303A9A0EBE4700193009302931CF0F2
:10207800AFFE002CACBF20232D2303A88DF8003021
:102088002BF0D4FA012803A924D002282DD0032844
:1020980005BF3023684668468DF801302DF039FBBE
:1020A80068462BF0C3FA0338C4B22246694628466C
:1020B8002DF066FB00232B5528462BF0B7FA2E226D
:1020C800431C2A540DEB0401E8182DF03FFB284669
:1020D80007B030BD302368468DF801308DF80230E6
:1020E8008DF803302DF015FBDAE7302368468DF8BC
:1020F80001308DF802302DF00CFBD1E76F12033A56
:1021080000007A442DE9F041064615460846B6FB1C
:10211800F2F43CB905FB1464124B1B5D00F8013B5B
:10212800BDE8F081B4FBF2F767B90E4B05FB174722
:1021380005FB1464DA5D00F8012B1B5D00F8013B18
:10214800BDE8F081B7FBF2F8B8F1000F02D04046C5
:10215800FFF7D8FF05FB1878024B13F8082000F8A2
:10216800012BE3E7DC1D03082DE9F04714461D4663
:10217800064600234FF47A72204629462BF000FFCA
:10218800DFF848814B4A4C4F88FB00310144C317A4
:1021980082FB002EC3EB611188FB012887FB002717
:1021A8008644464AC3EBEE2EC1EB011C82FB0E2986
:1021B800A0EB8C0C0744424A86F806C0C3EB2747BD
:1021C8004FEAEE7C08EB010ACCEBA90C82FB0782F4
:1021D8004FEAE1780CEB4C0CC8EB6A18AEEBCC0E6E
:1021E800C8EB0818DFF8E8C086F804E0A1EB88011E
:1021F80071718CFB0010F917C1EBE21240F2B55176
:1022080001FB1272C3EBE050B2F5896F4FEA800709
:102218003FDA40F2DA239A4243DCB2F5B77FB4BF23
:102228004FF0000C4FF0010C4FEA4C08254B08EB1F
:102238000C0103EBC1031FFA8CFE588F224908EBEF
:102248000C0301EBC30116310B2301E031F8020D39
:1022580082421BDA013BF9D11A4BC44403EBCC0C84
:102268000123BCF82400B37007F2B2770132121AC6
:10227800BE44F270A6F800E0204629464FF47A7270
:1022880000232BF07DFE3281BDE8F0870133DBB2FD
:10229800E9E74FF0030EF44640F296504FF0060877
:1022A800CCE74FF0020EF44640F229404FF0040804
:1022B800C4E700BFC5B3A29107452EC2ABAAAA2A9C
:1022C80073B06D16E8F702080CF802088988888848
:1022D800792D0311104B2DE93048D3E9004554EA14
:1022E80005020BD10346012200201871587198711C
:1022F8009A70DA7018801881BDE83088074B1A6820
:1023080014EB020B45F1000C5A466346FFF72CFF0D
:102318000120BDE8308800BFD81F0020946F00203E
:10232800F0B402888578164FC37804794179A2F20F
:10233800B27202F0030606EB4606013D05EB860580
:1023480007EB4505013BAE8C8579008940F2B5570E
:10235800920807FB0232931903EB430304EBC30310
:10236800C3EB031301EB8303C3EB031305EB8303F5
:1023780000214FF47A72C2FB0301F0BC704700BF22
:10238800E8F70208FAB170B48E18044603E0101A90
:1023980014D1B14214D014F8012BA2F14103192B26
:1023A80011F8013BA3F1410598BF2032192D03F123
:1023B8002000ECD9D01A01D1002BEAD170BC7047AB
:1023C800002070BC70471046704700BF4FF0FF32C6
:1023D800FFF7D8BFA0F16103192B98BF20387047C9
:1023E800A0F14103192B98BF20307047202805D051
:1023F800093804288CBF002001207047012070474D
:10240800613819288CBF00200120704741381928ED
:102418008CBF002001207047303809288CBF00206D
:1024280001207047A0F13003092B07D920F02000C4
:10243800413819288CBF00200120704701207047BF
:1024480030B402681146531C036011F8024B016056
:10245800D31C517803609378151D05601B0443EA6B
:102468000123D078234343EA006030BC704700BFA3
:102478000368591C1A46016012F8021B026058785A
:1024880041EA0020704700BF03685A1C02601878B0
:10249800704700BF38B50446006815462CF034F87C
:1024A80022682A44226038BD036810B40A0A5C1CFA
:1024B80004601A7003685A1C026019705DF8044BB6
:1024C800704700BF03685A1C026010B41970036893
:1024D8000A0A5C1C04601A7003680A0C5C1C04601D
:1024E8001A700368090E5A1C026019705DF8044BD3
:1024F800704700BF03685A1C026019700368090A14
:102508005A1C0260197070472DE9F047002488B002
:1025180080460F461E46A14605AD531C039311780D
:1025280039B3252933D1931CCDF8109003935078F3
:1025380030284ED04FF0000AA0F13003DBB2092B4F
:1025480042D96C2819D0642800F0938024D8252813
:102558001CD063D9582876D063281BD131784046DF
:10256800B847039A531C03931178043601340029A1
:10257800D7D1204608B0BDE8F087039B5A1C0392C8
:102588001B78642B7CD02AD8252B54D12521404692
:102598000134B847039AC0E7732833D044D9752863
:1025A8004FD106F1040E30682B4600220A217646E8
:1025B800FDF714FE049A0095534639464046FDF748
:1025C8004BFE039A0444A8E704AA03A91CF046FB9F
:1025D800B7E7D31C039390784FF0010AACE7732B4D
:1025E80010D05BD9752B3AD0782B96D1A3F158022D
:1025F800B2FA82F2306852092B4610210436FDF7F0
:10260800EDFDD7E73368049A009339460023404626
:10261800FDF722FE04360444039A7EE70028B9D168
:10262800204608B0BDE8F0876E28B3D1039A336816
:1026380004361C6071E72AD9582BD7D0632B8DD06C
:102648006BE77828A6D1A0F15802B2FA82F2306876
:1026580052092B461021FDF7C1FD0436AAE706F101
:10266800040E30682B4600220A217646FDF7B6FD97
:10267800A0E7331D306829461E46FDF781FD99E71E
:10268800331D306829461E46FDF77AFD92E7002B78
:102698007FF443AF204608B0BDE8F0876E2BC6D064
:1026A8003BE700BF0EB400B584B005AB019053F80A
:1026B800042B0649039301A8FFF726FF019B00227C
:1026C8001A7004B05DF804EB03B0704755020008B7
:1026D8000FB430B583B006AB0A490B4853F8042B46
:1026E800096800680193FFF70FFF084C054620684A
:1026F80016F0E6FE0028FAD0284603B0BDE83040C0
:1027080004B07047182C00201C2C00202420002026
:10271800DFED2B7AB4EEE70AF1EE10FA4ADDDFEDD1
:10272800296A9FED297A01E0B0EE670AB4EEC70A7C
:10273800F1EE10FA70EE667AF6DC9FED247AF4EE8C
:10274800C77AF1EE10FA38D5DFED1E6A9FED207AD0
:1027580001E0F0EE407AF4EEC77AF1EE10FA37EEC7
:10276800A60AF6D4DFED1B7AB4EEE70AF1EE10FA0A
:1027780014DDDFED137A37EEC00A60EE006A9FEDD4
:10278800166A9FED167ADFED167AA6EE867A20EEA7
:10279800266AE6EE877AA6EE270A7047DFED117AF9
:1027A800B4EEE70AF1EE10FA44BFDFED087A37EE2F
:1027B800C00AE2E7F0EE407ABFE7B0EE670AD1E779
:1027C800DB0F4940DB0FC940E4CB1641DB0F49C0A2
:1027D800E4CB16C1DB0FC93F92E741B99730083CFB
:1027E80015A82ABEDB0FC9BF09B909E0194690FB35
:1027F800F1F301FB13030846002BF7D10846704795
:102808000146FBE7F0EEC07AB0EEE07AB4EEE77A84
:10281800F1EE10FAB4BFB0EE676AB0EE476AB5EEF3
:10282800406AF1EE10FA46D0B4EEE77AF1EE10FA0B
:102838008CBFF0EE675AF0EE475AC5EE866A9FEDF8
:102848001F3A9FED1F6A9FED1F4A9FED1F5ADFED4C
:102858001F3ADFED1F4ADFED1F5AA6EEC36AE6EE08
:10286800A34AA6EE864AB7EE006AA6EE845AA6EEFA
:10287800A46AE6EE855AC5EE866AB4EEE77AF1EE0A
:1028880010FA48BFDFED147AF5EEC00A48BF77EEBC
:10289800E66AF1EE10FA48BFDFED107AB5EEC00A2D
:1028A80048BF77EEE66AF1EE10FA48BFF1EE666AC5
:1028B800B0EE660A7047DFED076ADEE739094E3D7C
:1028C800E3B59E3E88FA163E45FE7F3F99FB243FBE
:1028D80069A2163EA7DFA834DB0FC93FDB0F4940CA
:1028E800DFED317A30EE277AFDEEC76A16EE903AC0
:1028F8002033402B02D99FED2D0A7047B4EEE70A2A
:10290800F1EE10FA4DDD9FED2A6ADFED2A6A01E04B
:10291800B0EE677AB4EEE67AF1EE10FA77EE467A20
:10292800F6DC9FED257AF4EEC77AF1EE10FA35D58C
:10293800DFED1F6A9FED217A01E0F0EE407AF4EEB8
:10294800C77AF1EE10FA37EEA60AF6D4DFED167A5A
:10295800B4EEE70AF1EE10FA1BDCDFED197AB4EEFB
:10296800E70AF1EE10FA44BFDFED137A37EEC00A3A
:1029780060EE006A9FED136A9FED137ADFED137A1C
:10298800A6EE867A20EE266AE6EE877AA6EE270A73
:102998007047DFED0F7A37EEC00AE9E7B0EE670A55
:1029A800D4E7F0EE477ABCE7DB0FC93F0000000030
:1029B800DB0FC940E4CB1641DB0F49C0E4CB16C19D
:1029C800DB0FC9BF92E741B99730083C15A82ABE6A
:1029D800DB0F494007EE901AF8EE677A9FED837A8D
:1029E80027EE800A20EE070AFDEEC07A17EE903A2D
:1029F8002033402B00F28C80DFED7D7AB4EEE70ABD
:102A0800F1EE10FA40F3E880B0EE407A9FED796A73
:102A1800DFED796A01E0B0EE677AB4EEE67AF1EEBE
:102A280010FA77EE467AF6DC9FED747AF4EEC77A00
:102A3800F1EE10FA40F1CD809FED6E6ADFED706A1D
:102A480001E0F0EE477AF4EEE67AF1EE10FA37EEAE
:102A5800867AF6D4DFED6B7AB4EEE77AF1EE10FA07
:102A680051DCDFED697AB4EEE77AF1EE10FA44BF93
:102A7800DFED627A37EEC77A27EE076ADFED635A31
:102A8800DFED637ADFED636A9FED635AE6EE257A40
:102A980067EE065AE6EE276AF7EE007AA5EEA67A02
:102AA800F0EE675AE7EE055AE7EE457A87EEA55A43
:102AB800DFED547A30EE277AFDEEC76A16EE903ACB
:102AC8002033402B29D99FED557AF6EE006AB7EEF0
:102AD800006AF7EE004AC4EEA57A002383614361D9
:102AE8000362C36180ED045A67EEA66A27EE866A20
:102AF80027EE877AC0ED006AC0ED026A80ED016AB0
:102B080080ED037A7047DFED3A7A37EEC77AB3E79C
:102B1800B7EE005AF0EE455ACAE7B4EEE70AF1EE0E
:102B280010FA5FDD9FED336ADFED336A01E0B0EE46
:102B3800677AB4EEE67AF1EE10FA77EE467AF6DCCA
:102B48009FED2E7AF4EEC77AF1EE10FA47D59FED95
:102B5800296ADFED2B6A01E0F0EE477AF4EEE67AB7
:102B6800F1EE10FA37EE867AF6D4DFED267AB4EE77
:102B7800E77AF1EE10FA27DCDFED237AB4EEE77A94
:102B8800F1EE10FA44BFDFED1D7A37EEC77A27EE73
:102B9800076ADFED1E4ADFED1E6ADFED1E7AE6EEFC
:102BA800246A67EE064AE6EE267AB7EE006AA4EED5
:102BB800A77AF6EE006A36EE476AF8EE007A27EE54
:102BC800277A66EE266A84E7DFED097A37EEC77A58
:102BD800DDE7B0EE677A3DE7F0EE407A24E7B0EE45
:102BE800677AC2E7F0EE477AAAE700BF27D4D23661
:102BF800DB0F4940DB0FC940E4CB1641DB0F49C06E
:102C0800E4CB16C1DB0FC93FDB0FC9BF92E741B95F
:102C18009730083C15A82ABEF304353F0000008011
:102C280070B406688E4217D90139751E002311F851
:102C3800014F0822634013F0800F4FEA430318BF87
:102C480083F0D503013ADBB2F5D18D42EFD1721C86
:102C58000260337070BC70470023F8E710B44C0969
:102C6800012250F8243001F01F0102FA01F10B4350
:102C780040F824305DF8044B704700BF4B0901F061
:102C88001F0150F82320012303FA01F1114214BF58
:102C980018460020704700BFF0B55B4B5B4A97B001
:102CA8001968914200AF00F0A3805949594A00239E
:102CB8004FF47000C1F888003B607B60136843F4F0
:102CC8008033136003E03B68B3F5A04F09D0136865
:102CD80003F400337B603B6801333B607B68002B67
:102CE800F1D04C4B1B6813F4003318BF01237B60F1
:102CF8007B68012B52D0464C464B474AE260474A14
:102D0800596A11605A6A42F080725A625A6942F4EA
:102D1800FC025A610025032207F10801012341F64C
:102D2800FF764FF09040FD60BE603A73BB7322F0AF
:102D3800F3FC4FF6FF7307F108013948BB6022F036
:102D4800EBFC07F108013748374E22F0E5FC07F1A4
:102D58000801364822F0E0FC07F10801344822F067
:102D6800DBFC07F10801334822F0D6FC07F1080024
:102D780022F02BFDBB683049304AA1FB03133049D0
:102D88009B0CF0204FF0070E5C370B60566084F800
:102D980023009560C2F800E0BD46F0BD294A1D4BEE
:102DA800122111605A685A605A685A605A6842F487
:102DB80080625A605A6822F47C125A605A6842F457
:102DC800E8125A601A6842F080721A601A68920112
:102DD800FCD559680F4A21F003015960596841F040
:102DE80002015960536803F00C03082BFAD182E7FB
:102DF80000221A6062B6144B1B6883F30888134BD1
:102E08001B689847FEE700BFFC9F0020EFBEADDEC1
:102E180000ED00E0001002400005FA0558430020CC
:102E280000040048000800483F190100000C004851
:102E3800001000480014004883DE1B4310E000E047
:102E4800986F00200020024000D8FF1F04D8FF1F01
:102E580070B50F4C0F4DC0EBC00004EB80046869DF
:102E680026693043686182B09209667BA1600025BB
:102E7800012101A863618DF804608DF805208DF8A3
:102E880006508DF8071022F011FC02B070BD00BF8B
:102E9800680B002000100240074BC0EBC00030B4A4
:102EA80003EB8000054C056963692B436361017678
:102EB800427630BC704700BF680B0020001002400B
:102EC8002DE9F04F5E4C54F8204083B0002C71D0AF
:102ED800A66D984691465B4B72682265A160236097
:102EE80004F15E014FF4807304F5AF726161A26171
:102EF800E36023610746307E25F08EF9F068A8B1BB
:102F0800514B00215A68904203F11C0300F0928053
:102F180001310C29F6D100207A1CD2B20C21FFF71E
:102F2800BBFF236DF26862632433E364B068D8B1F1
:102F3800454B00215A68904203F11C0378D00131B7
:102F48000C29F7D100257A1CD2B20B212846FFF7AD
:102F5800A3FF2346F27E3D492846FFF779FF236DFC
:102F6800B268A2632833A36494F85D0016F0D8FC15
:102F7800054694F85C0016F0D3FC18F0080F82465A
:102F880096F819B01AD0CDB118F0110F4FF00B0305
:102F980007F1010714BF4E213E21EF715A46AB716C
:102FA800284616F081FD18F0010F45D0636B5BB31E
:102FB800A36B4BB3204603B0BDE8F08F18F0010FA8
:102FC8000CBF4FF02E084FF04E0819F0020F09D031
:102FD80045B10B227B1CAA71EB7128465A46414623
:102FE80016F062FD19F0010FE0D0BAF1000FDDD044
:102FF80001370C238AF807705A4641468AF806308A
:10300800504616F051FDD1E7337FB27E8DF804208B
:103018009B090021012201A88DF805308DF80610C2
:103028008DF8072022F042FB204603B0BDE8F08F60
:10303800CDB288E7C8B26FE7284616F0CFFDB5E7EE
:10304800242C00206CF80208680B0020E51C0008FE
:1030580000B97047F0B595B0054625F0A5FB6C4E54
:10306800C368026832600446002B00F0C38028461B
:1030780016F056FC674B186018B12922002382719C
:10308800C371227A644D2E2116F00EFD306808F0C7
:10309800BFFB25F0C1F83068604A038823F00103BC
:1030A8001B041B0C038014A91E232B8001270F234C
:1030B8000025138021F84C7D2D230293ADF80C5088
:1030C800ADF80650ADF80E5025F01CFBE379ADF8CD
:1030D800145060229907ADF816500695ADF81C50AB
:1030E800ADF81E50ADF82050ADF82250049200F112
:1030F800838013F0010F0CBF002202224FF480736B
:10310800ADF81470ADF81C20ADF82030002304AAE7
:1031180061793068069307F0E1FF61793068404FC4
:1031280025F0D0FA33685A6C42F400425A641A887F
:1031380092B242F080021A80E2796079196A9207A5
:103148004CBF04220122824021EA02011962196A55
:103158000A431A621A8892B242F001021A80207C4D
:1031680000222921FFF798FE2E49207C00236022A7
:10317800FFF76EFEE068386022F004FA38680368EA
:103188004FF6FE721340036022F0FCF909A822F002
:10319800CDF933686279244938680A913433134485
:1031A800099380221023002509A940F22A3E0E9295
:1031B8000B934FF400724FF400530D95109513952F
:1031C80011950F921293ADF830E022F0BCF96279B4
:1031D80033680C2A98BF1549D86898BF31F812503F
:1031E8003A6813490543DD601368012043F0020380
:1031F8001360087015B0F0BD13F0010F0CBF2A461C
:1032080008220423ADF81E20ADF816307EE700BF73
:10321800E0640020581D0020D6640020D4640020FB
:10322800DC640020BD0400083C500020A8110308FD
:10323800D86400200348D0F83C3113B100F59A70E7
:1032480018477047680B00200348D0F8203113B1A5
:1032580000F58C7018477047680B00200348D0F8B9
:1032680004310BB1FC301847704700BF680B0020D1
:103278000348D0F8E8300BB1E0301847704700BF7A
:10328800680B00200348D0F8CC300BB1C430184785
:10329800704700BF680B00200348D0F8B0300BB16E
:1032A800A8301847704700BF680B00200348D0F8C3
:1032B80094300BB18C301847704700BF680B002062
:1032C8000248836F0BB1703018477047680B0020B5
:1032D8000248C36D0BB1543018477047680B002083
:1032E8000248036C0BB1383018477047680B002050
:1032F8000248436A0BB11C3018477047680B00201E
:103308000248836803B11847704700BF680B002064
:103318001749184B184A194810B4D1F8884044F492
:103328007004C1F888401C6844F001041C605C68A3
:1033380022405A601A6822F0847222F480321A609D
:103348001A6822F480221A605A6822F4FE025A602F
:10335800DA6A22F00F02DA621A6B002410404FF08A
:10336800006218639C608A605DF8044B704700BF78
:1033780000ED00E0001002400CC07FF8CCFC00FF1C
:103388002DE9F04F2DED0E8BDFF8A8B39BB0DBF8DD
:103398000430079058469847002875D0BBF8A850C5
:1033A80000228BF85120002D41F03A84DBF8483098
:1033B800BBF93C60BBF93800DBF82050BBF93A1088
:1033C800DBF82440DFF870A3F71A87EAE772A2EB6C
:1033D800E772B2F5804FDBF82820DCBFCBF84860F5
:1033E8003346401B091B9B1ACBF82C00CBF8301036
:1033F800B3489BF85210CBF8343014F0CBF8DAF815
:103408000030980041F1FE84DBED0C5ADFF82C9374
:10341800DBED0B7AAB4A99ED406AD9ED416A99ED3B
:10342800427AD9F80C311268B8EEE58ADBED0D5A0C
:10343800F8EEE77AF8EEE58A013377EE867A38EE29
:10344800268A78EE878A9342C9ED407A89ED418AC7
:10345800C9ED428AC9F80C3102F0CC829A4B059327
:103468001E78142E03F02A830023D9F814410693FA
:10347800062C01F27781DFE814F0BE15F816FA146D
:103488009116E40809175A158F4BDFF8B0921C788B
:103498000593072C01F0B98199F82131099353B1AB
:1034A8005F1E89F82171012C01F088841BB0BDECE6
:1034B8000E8BBDE8F08F854B5B79002B01F01982EC
:1034C800834B1B78013BDBB2072C89F8213102F0D2
:1034D800768300230A937F4AD9F82C31D2ED006A0B
:1034E8007D4A9FED7E6AD2F800A07D4A0892079A2D
:1034F800D9ED4AAA99ED499ADFF844829FED79AA55
:10350800DFED79BA9FED79DA9FED79BADFED79CA07
:103518009FED79CA794F7A4EC9F82C21D31A07EE54
:10352800903AF8EE677AB7EE007AC6EE279A00244A
:10353800744B0693254677EE6A8A68EEA68AF4EEFF
:10354800C78AF1EE10FA88BFF0EE478A6E4B98ED05
:10355800008A2344D3ED007AF5EE407AF1EE10FAB2
:1035680017D06A4B234493ED007A78EE476AB0EEA1
:10357800E66AF4EEC67AF1EE10FA08D5F5EEC06AFE
:10358800F1EE10FACCBF37EE878A37EE678A83ED03
:10359800008A5F4B1B889A0739D0022D37D09AF8DA
:1035A8002E105C4A07EE901A224492ED007A4A42A5
:1035B800F8EEE76A07EE902A26EE877AF8EEE77AC1
:1035C800B4EEE77AF1EE10FA0AD407EE901AF8EEA4
:1035D800677AF4EEC77AF1EE10FA88BFF0EE477A10
:1035E8004D4A4E4902EB450231F91500B2F90C205B
:1035F800801A07EE100AB8EEC77AD807E7EE4A7ABB
:1036080041F10D81464B93ED008A27EE888A089B8D
:1036180099F86021234493ED01EA78EE4EDA002A06
:1036280000F0D0803F4AD9F8643107991268CB1A64
:10363800934240F3C7809AF84820022A02F0178381
:10364800022D05F00F81384A126891077AD4374A5B
:1036580086ED00DA12689A42C0F2AE80F7EE007A80
:10366800F4EEE7AAF1EE10FA40F1AC800899304B7D
:10367800D1ED017A93ED007AF0EEE77AF4EEC77AAD
:10368800F1EE10FA40F19E80D1ED027AF0EEE77A81
:10369800B4EEE77AF1EE10FA40F39480D1ED037AB4
:1036A800F0EEE77AB4EEE77AF1EE10FA40F38A80AA
:1036B8001D4B1B689A077FD51849174A63E000BF5E
:1036C800A459002068330020A85E0020F05B002089
:1036D800E03C0020786A0020EC6000200024744957
:1036E800045C0020CDCCCC3DAE47813F00000000FB
:1036F8000000C84200003443610BB63BF03A00209A
:10370800E43A0020D83A00206C6A0020D01E00203D
:10371800E8600020DC1E0020EC3C002098600020BF
:10372800546A0020806A0020946000207C6A00208F
:10373800886A002078590020145C0020941D00201D
:10374800C41E0020D74AD849DFF8CCE331F915C0A8
:103758009EED008ADFF8C4E386ED00DA02EB45004F
:1037680028EE0A8AB0F90C00A0EB0C0007EE900ACC
:10377800F8EEE77ADEF8000027EE888A984278EEBD
:103788004EDABFF66BAFB2F90C30B1F900E0C748BA
:10379800AEEB030E00688EEAEE73A3EBEE73834282
:1037A80010DAB1F90230B2F90E209A1A82EAE273FD
:1037B800A3EBE273984205DD0023184689F86031CF
:1037C80008F0F4FABA4B234493ED000A069B29EE5D
:1037D800000A022D20EE2D0AA3EC010A069304F03C
:1037E8008087B44BD6ED006A93ED007AB24BD3EDE7
:1037F800007AB24B93ED006AB14B67EE277A234407
:1038080027EEA87AD3ED007A67EE277AF0EE665AAB
:10381800EDEEA75AB1EE467AB4EEE57AF1EE10FA7B
:1038280008DCB4EEE56AF1EE10FA8CBFB0EE657A0A
:10383800B0EE467A99ED4A6AF7EE007AB4EEE76A96
:10384800F1EE10FAACBF0123002343B1F0EEE66AB3
:10385800F0EEC77AF4EEE67AF1EE10FA01D586EDCD
:10386800007A022D04F02C87964A974B52F82500CF
:103878001B68B0EE4E0A9847944A954B52F82500BB
:103888001B6898479AF8373023B1924B1B88002B56
:1038980001F0BE80B0EE4D8A8F4B38EE400A2344CB
:1038A80093ED008A83ED000A9AF8483030EE480A12
:1038B80020EE298A53B3894B1B78DB0740F1B48685
:1038C800F7EE007AF4EEE7AAF1EE10FA99F8603113
:1038D800C1F20986002B01F04B81D9F86431079AAF
:1038E800D31A7F4A12689A4210DD7E4BD3ED007AD4
:1038F800F0EEEDDAF4EEE7DAF1EE10FA42F1C0811B
:103908000023184689F8603108F050FA764B99F888
:103918007021234493ED000A29EE000A20EE088A5C
:1039280087ED008A32B9069B86ED00DA03ED01DAED
:1039380087ED00DA0135032D08F1040807F10407C3
:1039480006F1040604F104047FF400AE059B1B781D
:10395800072B01F0DD85012B02F0368100230B9344
:1039680099F87831002B41F03682604BDFF8B0A12E
:103978001C68DAF8003094F82C50DE0401F17480E9
:103988005B4B06931A465B4B528B93ED006A5A4B7E
:103998005A4ED3ED005AD6ED036A594B89ED626A47
:1039A80007EE102A574A93ED005AD2ED007AD2ED6D
:1039B800013AD2ED024A89ED606AB8EEC77A35EE6F
:1039C800C64A012336EEC77A89ED5F4AC9ED635AC4
:1039D80089F89031C7EE055A238D5A4206EE102A0F
:1039E800494ADFED4A6A92ED005A494A92ED004A87
:1039F800B7EE007AF4EEC75A35EE045AF1EE10FA33
:103A080088BFF0EE475A35EE275AB8EEC66AF4EE8C
:103A1800E65AF1EE10FA07EE903AB4EEC65AB8BF7D
:103A2800F0EE665AF1EE10FAC9ED665AB8EE677A0A
:103A380001F15184B4EEC75AF1EE10FA88BFB0EE26
:103A4800475A314BDFED336AD3ED017A304B93EDB2
:103A5800014A77EE847A25EE265A77EEA37AB4EEF9
:103A6800E76AF1EE10FA08DCB4EEE77AF1EE10FA44
:103A78008CBFB0EE676AB0EE476A234A638DD2ED19
:103A8800027A9FED247A5A4204EE102A74EEA77A3D
:103A9800B8EEC44A26EE076AF4EEC47AF1EE10FADC
:103AA8004BD43FE0EC3C002098600020846A002062
:103AB800286A002064690020000000209C6A002019
:103AC800346A00206C69002068690020C069002001
:103AD800BC690020E8600020FC1E002085620020F0
:103AE800806A00208C6A0020406A0020EC60002078
:103AF800D4660020603B0020B83C0020C85E00204F
:103B08007C3E0020E43A0020D83A00200000000063
:103B1800F03A00206F12833A546A00207C6A002031
:103B2800145C002007EE103AB8EE474AB4EEE74AB4
:103B3800F1EE10FA88BFB0EE674AEB4BDFEDEB7A97
:103B48005B7824EE274A0BB9B1EE444A002D41F0C8
:103B58001587B7EE003AE64B08931A78002A02F068
:103B6800BC87E44BDFEDE47AD3ED024AD3ED016A7A
:103B780093ED037A66EE244AE5EE264AE4EE074A18
:103B880063EE244AF4EEE74AF1EE10FAB4BFF0EE21
:103B9800673AF0EE643A98BFF0EE647A012ACDED08
:103BA800124A02F0C38793ED067AD3ED052AD3EDC6
:103BB800076A26EE077AA5EE227AA4EE267A23EE85
:103BC800077AB4EEE77AF1EE10FAB4EEE37A8CBF36
:103BD800F0EE676AF0EE476AF1EE10FA88BFF0EE91
:103BE800676AB4BFF0EE637AF0EE477A022A8DED89
:103BF800137A00F0DE8093ED0A7AD3ED092AD3ED2B
:103C08000B3A26EE077AA5EE227AA4EE237A23EE63
:103C1800077AB4EEE67AF1EE10FAB4EEE77A8CBFE2
:103C2800F0EE663AF0EE473AF1EE10FA98BFF0EE91
:103C3800636AA8BFF0EE477A032A8DED147A00F084
:103C4800B88093ED0E7AD3ED0D2AD3ED0F3A26EE18
:103C5800077AA5EE227AA4EE237A23EE077AB4EE49
:103C6800E67AF1EE10FAB4EEE77A8CBFF0EE663A37
:103C7800F0EE473AF1EE10FA98BFF0EE636AA8BF8B
:103C8800F0EE477A042A8DED157A00F09280D3ED94
:103C9800123AD3ED112A93ED137A66EE233AE5EE44
:103CA800223AE4EE073A63EE233AF4EEE63AF1EE0E
:103CB80010FAF4EEE73A8CBFB0EE667AB0EE637AAB
:103CC800F1EE10FA98BFF0EE476AA8BFF0EE637AFB
:103CD800052ACDED163A6CD0D3ED163AD3ED152A58
:103CE80093ED177A66EE233AE5EE223AE4EE073AC8
:103CF80063EE233AF4EEE63AF1EE10FAF4EEE73A20
:103D08008CBFB0EE667AB0EE637AF1EE10FA98BF27
:103D1800F0EE476AA8BFF0EE637A062ACDED173AAF
:103D280047D0D3ED1A3AD3ED192A93ED1B7A66EEF4
:103D3800233AE5EE223AE4EE073A63EE233AF4EE4C
:103D4800E63AF1EE10FAF4EEE73A8CBFB0EE667A96
:103D5800B0EE637AF1EE10FA98BFF0EE476AA8BFAA
:103D6800F0EE637A072ACDED183A22D093ED1E7A49
:103D7800D3ED1D2AD3ED1F3A26EE077AA5EE227A57
:103D8800A3EE847A27EE037AB4EEE67AF1EE10FA1F
:103D9800B4EEE77A8CBFB0EE666AB0EE476AF1EE31
:103DA80010FA8DED197A98BFF0EE466AA8BFF0EECA
:103DB800477A77EEE67AF7EE006AF4EEE67AF1EE05
:103DC80010FAC9ED4A7A44F3118286EEA77A022ADC
:103DD800DDED137A67EE244A67EE877ACDED124A55
:103DE800CDED137A2DD0DDED147A67EE877A032AAC
:103DF800CDED147A25D0DDED157A67EE877A042AA1
:103E0800CDED157A1DD0DDED167A67EE877A052A95
:103E1800CDED167A15D0DDED177A67EE877A062A8A
:103E2800CDED177A0DD0DDED187A67EE877A072A7F
:103E3800CDED187A05D0DDED197A27EE877A8DED6C
:103E4800197A2E4B1B6813F0805C01F00183F6EEA3
:103E5800005AC9ED665A002A02F06286284D294C9C
:103E680099ED636A284B99F99011284E284899EDE5
:103E7800625AD5ED004AB4F90650069C0078648B66
:103E880096F800E00A94BDEEC66A07EE101AD978D3
:103E9800DAF80030D9ED5F6AD9ED607A16EE106A6B
:103EA800BDEEC56A03F0100403F4805803F48003E0
:103EB8000C9300F00107B8EEC77A16EE103A0D48D9
:103EC800002940F0CB879DED125A90ED006A002C36
:103ED80041F0288425EE866A0E49A5EE076AB0EE01
:103EE800675AA6EE265A17E02C3D00206F12833A37
:103EF800565E0020EC3D0020000000003C3B002006
:103F0800E83D0020BC4E0020EC4E00200840002078
:103F1800856200200C3B0020BDEEC56A16EE105AE3
:103F280016EE104AB542A8BF3446AB42C8BF1C467D
:103F380006EE104AB8EEC66A012A81ED006A00F062
:103F4800DC8090ED046A9DED135A25EE866AA5EE95
:103F5800076AB0EE675AA6EE265ABDEEC56A16EE97
:103F6800105A16EE104AB542A8BF3446AB42C8BF35
:103F78001C4606EE104AB8EEC66A022A81ED016AAE
:103F880000F0BB8090ED086A9DED145A25EE866A14
:103F9800A5EE076AB0EE675AA6EE265ABDEEC56AC8
:103FA80016EE105A16EE104AB542A8BF3446AB4278
:103FB800C8BF1C4606EE104AB8EEC66A032A81ED51
:103FC800026A00F09A8090ED0C6A9DED155A25EE74
:103FD800866AA5EE076AB0EE675AA6EE265ABDEEC7
:103FE800C56A16EE105A16EE104AB542A8BF3446F6
:103FF800AB42C8BF1C4606EE104AB8EEC66A042A91
:1040080081ED036A79D090ED106A9DED165A25EE80
:10401800866AA5EE076AB0EE675AA6EE265ABDEE86
:10402800C56A16EE105A16EE104AB542A8BF3446B5
:10403800AB42C8BF1C4606EE104AB8EEC66A052A4F
:1040480081ED046A59D090ED146A9DED175A25EE5A
:10405800866AA5EE076AB0EE675AA6EE265ABDEE46
:10406800C56A16EE105A16EE104AB542A8BF344675
:10407800AB42C8BF1C4606EE104AB8EEC66A062A0E
:1040880081ED056A39D090ED186A9DED185A25EE34
:10409800866AA5EE076AB0EE675AA6EE265ABDEE06
:1040A800C56A16EE105A16EE104AB542A8BF344635
:1040B800AB42C8BF1C4606EE104AB8EEC66A072ACD
:1040C80081ED066A19D090ED1C6A9DED195A65EECE
:1040D800865AE7EE055AE6EEA57AFDEEE77A17EE80
:1040E800900A8642A8BF06468342D8BF334607EEE9
:1040F800903AF8EEE77AC1ED077A002F00F0BA8718
:10410800CD4B1B68002B40F0C287CC4B1B788BB182
:10411800089F387858B1CA4DCA4E0024E0B23368B7
:10412800B5EC010A9847387801348442F6DBC64B6F
:104138001B689847059B1B78072B01F0D981002540
:10414800DAF800305F0501F12581C04B1B78BBB15F
:10415800BF4A069BB2F906205B8B9A4210DCBD4B26
:104168001B78012B01F04285192B01F03F850E2B9E
:1041780006D0082B04D0B84E0023B360C9F83831F4
:1041880099F8C64124B1B54B1B889E0741F00185BB
:1041980099F8CC31002B41F0A280069A947F002C2C
:1041A80000F00386022C01F01A84032C41F01E84CF
:1041B80092F82020C2EB421102EB8102D20092B2A7
:1041C8000699CF7F0237FFB2002B00F02086002A25
:1041D80000F01D86A2490C68B2FBF4F214B2A9F8EB
:1041E800FC41002F03F0B88407EE904AF8EEE77A16
:1041F800F7EE006A86EEA77A974E012FD9ED846A0A
:10420800D6ED007A77EEE67A67EE877AC9ED807A9E
:1042180021D0D6ED017AD9ED856A77EEE67A022FBC
:1042280067EE877AC9ED817A15D0D6ED027AD9ED95
:10423800866A77EEE67A032F67EE877AC9ED827A87
:1042480009D0D6ED037AD9ED876A77EEE67A67EE7C
:10425800877AC9ED837A059A1278092A03F01786B6
:10426800002C40F3A8859FB399ED847AD9ED807A24
:1042780077EE877A012FC9ED847AC6ED007A21D0CE
:1042880099ED857AD9ED817A77EE877A022FC9ED93
:10429800857AC6ED017A15D099ED867AD9ED827ABC
:1042A80077EE877A032FC9ED867AC6ED027A09D0B0
:1042B800D9ED877A99ED837A77EE877AC9ED877A8F
:1042C800C6ED037A013F022FB8BF0227FAB209925E
:1042D800002B099F18BF0227624BDFED676A1A6837
:1042E800059B91781878137807EE903AF8EEE77AFC
:1042F800B0EE007A67EEA67AF4EEC77AF1EE10FA1D
:1043080040F3E587DFED596A37EEC77AB0EE676AA2
:10431800A7EE266AF0EE466A96ED007A9FED546A9B
:1043280027EE066AF0EEC65A89ED526AC9ED555A6B
:1043380099B107EE101AB8EEC75A9FED4F7A66EE9C
:10434800064A25EE075AB7EE007A37EE457A64EE4C
:10435800A54AA4EE857A26EE076A9FED467A537938
:1043680026EE877A27EE067ACBB1DFED436A9FED1A
:10437800436A65EEA65A06EE903AF8EEE66A65EEEE
:10438800A65AF4EEC65AF1EE10FA01F3E082B7EE3F
:10439800006A76EE655AC6EE256A27EE267A0C285C
:1043A8009FED378ADFED376A01F05980B4EEC87A9D
:1043B800F1EE10FA98BFB0EE478AB4EEE68AF1EE55
:1043C80010FAB8BFB0EE668A89ED4C8A002F00F06B
:1043D8000681B0EE007AF4EEC77AF1EE10FA05DD48
:1043E80037EEC77ADFED216AE7EE267A96ED017A95
:1043F800DFED1F6A27EE267AF0EEC75A89ED537A69
:10440800C9ED565A99B106EE901A9FED1B6AF8EE5F
:10441800E66A27EE075A66EE866AB7EE006A36EE57
:10442800666A25EE255AA5EE266A27EE067ADFED9E
:10443800116A937928E000BF5C69002030430020AE
:104448000C3B0020FC3F0020044000201C01002001
:10445800BC4E00202C3D0020C85E0020E8600020F3
:10446800143D0020F06000200000C842D7A3684136
:104478006F12033B000048430AD7233CA4707D3FDA
:1044880000C0F94400C0F9C467EEA67A67EE877ADF
:10449800ABB107EE103AB8EEC77A1FED096A5FEDC7
:1044A800096A27EE257A27EE067AB4EEE67AF1EE67
:1044B80010FA41F33E825FED146A67EEA67A0C2883
:1044C80000F0EA875FED126A1FED127AF4EEE67AE1
:1044D800F1EE10FA88BFF0EE667AF4EEC77AF1EEE4
:1044E80010FAB8BFF0EE477A012FC9ED4D7A76DDA4
:1044F80053785FED1F6A07EE903AF8EEE77AB0EE70
:10450800007A67EEA67A537AF4EEC77AF1EE10FADB
:1045180005DD37EEC77A5FED2B6AE7EE267A96ED72
:10452800027A5FED2D6A27EE267AF0EEC75A89EDFA
:10453800547AC9ED575A9BB106EE903A1FED326A8C
:10454800F8EEE66A27EE075A66EE866AB7EE006A64
:1045580036EE666A25EE255AA5EE266A27EE067A15
:104568005FED3C6AD37967EEA67A67EE877AFBB18E
:1045780007EE103AB8EEC77A1FED416A5FED416A5F
:1045880027EE257A27EE067AB4EEE67AF1EE10FAEF
:1045980001F3CB81B5EEC07AF1EE10FA02F18D8409
:1045A800B7EE006A36EE477AC6EE076A67EEA67A75
:1045B8000C2800F090875FED4E6A1FED4E7AF4EEFE
:1045C800E67AF1EE10FA88BFF0EE667AF4EEC77A72
:1045D800F1EE10FAB8BFF0EE477AC9ED4E7A092825
:1045E80000F02987069B93F82140002C40F0DD86D7
:1045F800002389F8CC31C04B1B7823B9BF4CA37872
:10460800002B41F08C82079823F069F8059B1C78F1
:10461800072C7EF448AF07F06BFAB94B059A401B9C
:104628001478D880FEF73FBF99F86031002B3FF42B
:104638006DA90023184689F8603107F0B7FBFFF72A
:1046480065B9B04B1A78D9F81851AF4F9FEDAF7ACA
:10465800E8003B1883ED007A002A78D0AC49B0EE28
:10466800476AF0EE476A0023F1EC017A013367EEFE
:10467800A77A05EE903AB4EEE77AF1EE10FAF8EE82
:10468800E55AB8BFB0EE677A934276EEA76AA7EE0E
:10469800A56AE9D1F5EEC06A3B18F1EE10FA83ED90
:1046A800007A54DDC6EE265A9A4B9B4A1288F7EEDA
:1046B800007A75EEE75AD3ED007A65EEA77AFDEE3B
:1046C800E77A17EE903A812B42F36E839342A8BFA4
:1046D800134607EE903AF8EEE77A904B411903EB50
:1046E800810393ED057AD3ED003A93ED066A93EDD5
:1046F800014AD3ED046AD3ED034A93ED025AA3EEBF
:10470800A77AA4EE276A66EEC76AA7EE646ABDEECA
:10471800C77AE5EE276A17EE101A812983ED056A34
:10472800C3ED066A42F344838A42A8BF0A4607EEED
:10473800902AF8EEE77AFCEEE77ACDED087ABDF834
:1047480020303A18938015B9132E03F0E884152EFB
:1047580041F0E0836A4BD9F8144138441A468388FB
:1047680022F815306E4B013483FB04231A19E31722
:10477800C3EBA203C3EBC303E41AC9F814416949A4
:10478800D9F81C31079C68480A680078C9F81C41A8
:10479800E31A1A440A60002840F0D68007EE903ADF
:1047A800624DDFF8A081624EB8EEE78A05F5F07435
:1047B80005F51377F5EC017A9BED070ADBF808326B
:1047C800F8EEE77A204627EE800A9847A4F1E00041
:1047D800DBF828319847A4F17000DBF89831984746
:1047E800D5F8EC00DBF8AC309847D6ED007AA8ECA9
:1047F800010AE0EE087A2434A742E6EC017AD9D11E
:10480800059B1C78072C7EF447AE07F071F9059AD2
:104818003B4B1478079A801A1880FEF73DBE99ED35
:10482800557AB1F90000D9ED566AB1F902E0414A6A
:10483800F4EEC76A80EAE0738EEAEE71A3EBE073E8
:10484800F1EE10FAA1EBEE71B8BFF0EE476A8B42B9
:10485800B8BF0B4607EE103A1378B8EEC77A27EEC2
:104868000A7A002B00F05B81334B93ED005AB5EECA
:10487800C05AF1EE10FA40F3E785304BD3ED004A09
:10488800F5EEC04AF1EE10FA40F3DE8534EEC77A51
:1048980066EECB5A87EE246AC5EE856AB7EE007AD3
:1048A800B4EEC76AF1EE10FA88BFB0EE476AB5EE0B
:1048B800C06AF1EE10FA76EE876AB8BFB0EE4D6ABC
:1048C80066EE266AF4EEC76AF1EE10FA88BFF0EEDB
:1048D800476AF5EEC06AF1EE10FAB8BFF0EE4D6A1D
:1048E800174B93ED007A67EE877AA7EEA68AFEF754
:1048F8008EBE0123FEF7E8BD594C002092640020CB
:10490800AC5E00206E3300206436002000000000FA
:10491800941D0020703300206C3300208C3500205B
:1049280093244992AC3D002064330020A459002010
:10493800B03D0020606A00205C6A0020646A0020A4
:10494800586A0020085C002007EE903A9E4A9F4C67
:104958009F49A04FCDF82090F8EEE78A069204F51B
:10496800B875904600268946059BDBED077A1B78CB
:10497800172B6DD094ED007AB8EEC78A082B28EE75
:10498800278A07D1B0EE480A099329F0FDFE099B52
:10499800A8F80000DAF8002091000BD5002E03F0EB
:1049A8004687B0EE480ADBF8083205F170009847F0
:1049B800B0EE408AB0EE480ADBF82831A5F1700065
:1049C8009847DBF8983128469847059B1B78032BB6
:1049D800B0EE408A37D0D4F8F000DBF8AC30B0EE57
:1049E800480A9847D7ED007AA9EC010AE0EE287A40
:1049F8000136032E05F1240508F1020804F1040428
:104A0800E7EC017AB0D1059BDDF820901C78F9E637
:104A1800714B724A234493ED007AD2ED007A704BC1
:104A280067EE277AF7EE006AF4EEE67AF1EE10FA0E
:104A380093ED007A88BFF0EE667A67EE877A27EE04
:104A4800888AFEF729BF29F09FFEA8F80000C2E770
:104A580094ED007A0BEB4602B8EEC78A128FA8F8DD
:104A6800002028EE278A95E75E4B5F4E1B78D6ED2F
:104A7800037A13F0010F5D4B069304BF1B8BA9F853
:104A880084315B4B1B8807EE103AB8EEC77AF4EE18
:104A9800C77AF1EE10FA41F2CE87564A128807EE2D
:104AA800102AB8EEC77AF4EEC77AF1EE10FAC1F21E
:104AB800A980514B514A93ED006AD2ED006A99F9E9
:104AC8009031C9ED626A76EE665A012BC9ED606ACB
:104AD800C9ED5F5A89ED636A01F0AD86079BC9F895
:104AE8009431002237EEC77AFCEEE77A444989ED23
:104AF800667A17EE903AA9F88431012391ED005AAD
:104B080089F890313F4B9A4241F2C5873E4BD3ED2D
:104B1800007AD3ED013AD3ED024AFEF75BBF3B4B77
:104B280093ED006AB4EEEB6AF1EE10FA40F1F28709
:104B3800F7EE005A75EEC65A3CEEC77A65EE8C5A07
:104B4800334BA7EE256A93ED007A26EE076AB5EE99
:104B5800C06AF1EE10FA40F27784CBEE065AB7EE4F
:104B6800007AB0EE476AA6EEE56AF0EE466AA9E674
:104B7800284AD2ED007AB0EEC87AB4EEE77AF1EEC0
:104B880010FA7EF7C3AE244AD2ED007AB0EEED7A81
:104B9800B4EEE77AF1EE10FA7EF7B8AE1F4AD8ED18
:104BA800007A92ED007AF0EEE77AF4EEC77AF1EE49
:104BB80010FA7EF5ABAE01220799C9F8641189F89D
:104BC8006021FEF78EBE00BFAC5E0020A459002015
:104BD800085C0020B03D0020E81E0020506A00203C
:104BE8004C6A002085620020C85E0020D466002040
:104BF800803E0020823E0020B83C00206C3E002011
:104C0800883E00208FD00300E43A0020686A002024
:104C18005C6A0020906A00208C6A0020946A002058
:104C2800804C8148814B8249089326461B68059031
:104C380006944F780478B6F906004FF47A71B1FB00
:104C4800F3F3C3EB431603EB8603DE00B6B2B542BB
:104C580002F0B180DBF87CE0BBF93820DBF860308B
:104C68000EF1010107EE902A13440129CBF87C10BC
:104C7800CBF86030F8EEE77A02F0AA80DBED1B5A39
:104C8800DBED1D6A07EE101A37EEE56AB8EEC75A73
:104C9800012D86EE057A37EE257A77EEC77A8BED09
:104CA8001C7AE7EE866A8BED1B7AF0EE667ACBED1E
:104CB8001E6ACBED1D6A02F09185DBF890E0BBF926
:104CC8003A20DBF864300EF1010107EE902A134414
:104CD8000129CBF89010CBF86430F8EEE77A02F0AF
:104CE8009280DBED205ADBED226A07EE101A37EED0
:104CF800E56AB8EEC75A012D86EE057A37EE257AB1
:104D080077EEC77A8BED217AE7EE866A8BED207A0B
:104D1800F0EE667ACBED236ACBED226A02F0868547
:104D2800DBF8A4E0BBF93C20DBF868300EF10101A8
:104D380007EE902A13440129CBF8A410CBF8683069
:104D4800F8EEE77A02F07A80DBED255ADBED276A88
:104D580007EE101A37EEE56AB8EEC75A012D86EE4F
:104D6800057A37EE257A77EEC77A8BED267AE6EE66
:104D7800276A8BED257AF0EE667ACBED286ACBEDC3
:104D8800276A02F01E85069BDFF8C890D880BBF81A
:104D9800A830059A013B1478ABF8A830089900238D
:104DA8004B608B60CB60FEF774BBA9F8FC41002B0D
:104DB8003FF421AC1F4E0227FFF78EBA1E4B1F4A45
:104DC80019681288174BC96919805A801BB0BDEC45
:104DD8000E8BBDE8F08F1A4B1B7813F0010F194B9F
:104DE800089340F0CD831A78002A00F0C18592001C
:104DF80015491648DFF860A029F086FB144B069386
:104E0800FFF77EB9084B0593DFF84890B7E4B9F887
:104E1800FC41013C24B2002CA9F8FC41C7DD054E39
:104E2800FFF721BAAC5E0020A85E0020045C0020D9
:104E3800F05B0020C85E00207C5400202237002050
:104E480085620020565E0020F83900200C3B0020C7
:104E5800D4660020941D0020145C0020002C01F072
:104E68006782002F42F09286BEF1000F42F00E8555
:104E780090ED006A9DED125AAE4925EE866AFDEE68
:104E8800E44AA5EE076AB0EE675AA6EE265A14EE73
:104E9800903ABDEEC56A16EE105A16EE104AB542A3
:104EA800A8BF3446AB42C8BF1C4606EE104AB8EE4F
:104EB800C66A012A81ED006A00F0DF8090ED046A7D
:104EC8009DED135A25EE866AA5EE076AB0EE675A7D
:104ED800A6EE265ABDEEC56A16EE105A16EE104A10
:104EE800B542A8BF34469D42B8BF1C4606EE104ADC
:104EF800B8EEC66A022A81ED016A00F0BE8090ED24
:104F0800086A9DED145A25EE866AA5EE076AB0EE8A
:104F1800675AA6EE265ABDEEC56A16EE105A16EE68
:104F2800104AB542A8BF34469D42B8BF1C4606EE9B
:104F3800104AB8EEC66A032A81ED026A00F09D8025
:104F480090ED0C6A9DED155A25EE866AA5EE076A66
:104F5800B0EE675AA6EE265ABDEEC56A16EE105A8E
:104F680016EE104AB542A8BF34469D42B8BF1C464B
:104F780006EE104AB8EEC66A042A81ED036A7CD0B0
:104F880090ED106A9DED165A25EE866AA5EE076A21
:104F9800B0EE675AA6EE265ABDEEC56A16EE105A4E
:104FA80016EE104AB542A8BF34469D42B8BF1C460B
:104FB80006EE104AB8EEC66A052A81ED046A5CD08E
:104FC80090ED146A9DED175A25EE866AA5EE076ADC
:104FD800B0EE675AA6EE265ABDEEC56A16EE105A0E
:104FE80016EE104AB542A8BF34469D42B8BF1C46CB
:104FF80006EE104AB8EEC66A062A81ED056A3CD06C
:1050080090ED186A9DED185A25EE866AA5EE076A96
:10501800B0EE675AA6EE265ABDEEC56A16EE105ACD
:1050280016EE104AB542A8BF34469D42B8BF1C468A
:1050380006EE104AB8EEC66A072A81ED066A1CD049
:1050480090ED1C6A9DED195A65EE865AE7EE055AF1
:10505800E6EEA57AFDEEE77A17EE900A8642A8BF3B
:1050680006468342D8BF334607EE903AF8EEE77A11
:10507800C1ED077A002A3FF443A892002E492D4833
:1050880029F042FA2D4B1B68002B3FF43EA82C4B0D
:105098001B78192B07D801212A4A01FA03F31A4071
:1050A800002A41F0ED87DFF8B480274EDAF80030A7
:1050B800990655D5F27AFF2A04D0244B1B789342DF
:1050C80001F2E582B6F90850F27DA8F80050FF2AEF
:1050D80001F0AD841D4B1B78934241F2A8841C4B10
:1050E80033F91240A8F80240082018F019FCB8B3A8
:1050F80099F8C031012B02F07E86164B96F91600FE
:1051080096F90A705A881B88134910FB03F317FB9A
:1051180002F281FB020781FB0301D217DB17C2EB06
:105128002712C3EB21132A441C44A8F80020A8F82E
:10513800024015E00C3B0020F83900205C69002093
:105148006069002032C1300324370020AC2E0020D3
:10515800BC4E0020986000201F85EB51FC3A0020CF
:10516800B8F90070B6F90600B8F90250B6F912108D
:10517800B8F90440B6F91E20B6F90430B8F90EE0C3
:10518800B842A8BF3846A942A8BF2946A242A8BF2C
:105198002246BB42D8BF0346A8F80030B6F9103003
:1051A800B8F90670B8F90800AB42C8BF1946B6F995
:1051B8002A30A8F80210B6F91C10B8F90C50BB42F6
:1051C800A8BF3B46A142C8BF0A46B6F93640A8F870
:1051D8000420B6F92820B8F90A108442A8BF04466A
:1051E800BA42C8BF1346B6F94220A8F80630B6F945
:1051F8003430B6F94E708A42A8BF0A468342D8BFF7
:105208002346A8F80830B6F94030B6F95A00AF423C
:10521800A8BF2F468B42D8BF1346A8F80A30B6F964
:105228004C30B6F958207045A8BF7046AB42C8BF8D
:105238001F46C24BA8F80C709645B8BF1046A8F890
:105248000E009B8913B3BE4DBE4FBF4E05F110042F
:10525800B5F9023000EE103A3846B8EEC00AFBF74E
:105268006BF829F091FAB6F90430B6F9062000B2C5
:10527800984207F1240706F10C0603DB8242134625
:10528800A8BF034625F8023FAC42E1D1AF4B1B78DB
:10529800013B182B01F2D582DFE813F0490AD30A43
:1052A800D30A4609D30AD30AD30A390AD30AD30A36
:1052B800D30AD30AD30A190AFE09D30AD30AD30A8E
:1052C800D30A4609290AD30AD30A190A490AF0EE69
:1052D800676AFFF721B8B0EE465AFEF7B2BB9C49A1
:1052E8009C4AD1F8EC10126844F620608142A8BFAD
:1052F8000146B1F57A7FB8BF4FF47A7189B212F0DE
:10530800100FA9F8CE11DAF8002000F07684D00446
:1053180041F1F387904A17687C8E64088F4E904855
:10532800D9F8D021D6ED037AA0FB010188096421C0
:1053380091FBF0F11429BDEEE77A09EB4206A8BF0C
:10534800142101329142C9F8D02117EE10EADCBFCE
:105358000022C9F8D02109EB4202A6F8D4E1B2F93B
:10536800D42107EE102AB8EEC77A77EEC77AFDEE99
:10537800E77ACDED087ABDF9201081EAE172A2EB57
:10538800E172A24202F3028276494FF07E520A602D
:10539800FEF703BFDBF80830002B3EF4D6AE7249A7
:1053A800A1F14C009847FEF7D0BE1E216948FDF7D1
:1053B80065FC00283FF41CA96C4B1B885B063FF575
:1053C80017A999F82032A34242F03E85654B99ED22
:1053D800890AD3ED018AD9ED4E5A9FED656ADFED52
:1053E800656A20EE657A68EE007AA8EE287AE5EE1E
:1053F800A87AB4EEC67AF1EE10FA88BFB0EE467A13
:10540800B4EEE67AF1EE10FAF4EEC67AB8BFB0EE72
:10541800667AF1EE10FA88BFF0EE467AF4EEE67A94
:10542800F1EE10FAB8BFF0EE667A89ED4C7AC9ED64
:105438004E7AFFF7DDB8FDEEC87A4F4A17EE903A7C
:105448009480D380FFF7CEB8DFED4C6AFFF748BAF7
:10545800DAF800305D023EF5FAACFEF7FCBCB4EEBB
:10546800C87AF1EE10FA98BFB0EE478ABDEEC77A57
:10547800B4EEE68ADFF800E1F1EE10FA17EE103A22
:10548800B8BFB0EE668A89ED4C8AAEF80030002FBE
:105498007EF49FAFFFF7A6B89FED357ADFED356A4A
:1054A8003549F4EEC77AF1EE10FA98BFB0EE677A94
:1054B800FDEEE77AB4EEE67AF1EE10FA17EE903ADE
:1054C800B8BFB0EE667A012F89ED4D7A4B803FF771
:1054D8000FA8FFF787B8BDEEE77A274B17EE102A1B
:1054E8009A80FFF768B8002B3EF410AAFEF7F5B9CA
:1054F80006F0FEFA059B0B991B781F4A401A072BEA
:1055080090807EF41CAE06F0F3FA0546FEF718BE4E
:1055180006F0EEFA184B06931A46059B0A991B7873
:10552800401A012B508000F05183072B7EF416AAF5
:1055380006F0DEFA0B90FEF713BA00BF785700208A
:10554800FA3A0020C867002024370020606900204C
:10555800280100203C3B0020EC600020C85E0020B1
:10556800D34D621000000020C4590020E8600020DC
:1055780000C0F94400C0F9C4AC5E0020000000007F
:105588001B78002B00F0F481D9ED563A99ED556A55
:10559800D9ED607AF04A99ED5F7AD2ED005A99ED2B
:1055A800534AD9ED524AED48ED49F4EEC63AF3EEC6
:1055B800046AF1EE10FA37EEA65A00F1A58390EDD1
:1055C800026A26EE446AF0EE674AE6EE074AF4EE0F
:1055D800C54A34EEE66AF1EE10FA48BFB0EE656AE5
:1055E800012B81ED006A00F0C38190ED066A26EE7A
:1055F800446AF0EE674AE6EE074AF4EEC54A34EE2E
:10560800E66AF1EE10FA48BFB0EE656A022B81ED4A
:10561800016A00F0AD8190ED0A6A26EE446AF0EE68
:10562800674AE6EE074AF4EEC54A34EEE66AF1EE5A
:1056380010FA48BFB0EE656A032B81ED026A00F0EC
:10564800978190ED0E6A26EE446AF0EE674AE6EE20
:10565800074AF4EEC54A34EEE66AF1EE10FA48BF9E
:10566800B0EE656A042B81ED036A00F0818190ED4C
:10567800126A26EE446AF0EE674AE6EE074AF4EE4E
:10568800C54A34EEE66AF1EE10FA48BFB0EE656A34
:10569800052B81ED046A00F06B8190ED166A26EE09
:1056A800446AF0EE674AE6EE074AF4EEC54A74EE3D
:1056B800E66AF1EE10FA48BFF0EE656A062BC1ED16
:1056C800056A00F05581D0ED1A6A66EEC46AF0EEFC
:1056D800674AE6EE874AB3EE046AF4EEC54A74EE0A
:1056E800C66AF1EE10FA48BFF0EE656A072BC1ED05
:1056F800066A00F03D81D0ED1E6A9A4BDFF86CA275
:10570800069326EEC44AE4EE077AF4EEC57A77EEFD
:10571800C67AF1EE10FA48BFF0EE657AC1ED077A65
:10572800FEF7EEBC002F41F03B8225EE866A8C49DD
:10573800A5EE076AB0EE675AA6EE265ABDEEC56A10
:1057480016EE105A16EE104AB542A8BF3446AB42C0
:10575800C8BF1C4606EE104AB8EEC66A012A81ED9B
:10576800006A3FF48AAC90ED046A9DED135A25EE69
:10577800866AA5EE076AB0EE675AA6EE265ABDEE0F
:10578800C56A16EE105A16EE104AB542A8BF34463E
:10579800AB42C8BF1C4606EE104AB8EEC66A022ADB
:1057A80081ED016A3FF469AC90ED086A9DED145AE9
:1057B80025EE866AA5EE076AB0EE675AA6EE265A67
:1057C800BDEEC56A16EE105A16EE104AB542A8BFCD
:1057D8003446AB42C8BF1C4606EE104AB8EEC66A4D
:1057E800032A81ED026A3FF448AC90ED0C6A9DED06
:1057F800155A25EE866AA5EE076AB0EE675AA6EE38
:10580800265ABDEEC56A16EE105A16EE104AB54273
:10581800A8BF3446AB42C8BF1C4606EE104AB8EED5
:10582800C66A042A81ED036A3FF427AC90ED106A3A
:105838009DED165A25EE866AA5EE076AB0EE675A00
:10584800A6EE265ABDEEC56A16EE105A16EE104A96
:10585800B542A8BF3446AB42C8BF1C4606EE104A44
:10586800B8EEC66A052A81ED046A3FF406AC90EDED
:10587800146A9DED175A25EE866AA5EE076AB0EE02
:10588800675AA6EE265ABDEEC56A16EE105A16EEEF
:10589800104AB542A8BF3446AB42C8BF1C4606EE04
:1058A800104AB8EEC66A062A81ED056A3FF4E5ABF0
:1058B80090ED186A9DED185A25EE866AA5EE076ADE
:1058C800B0EE675AA6EE265ABDEEC56A16EE105A15
:1058D80016EE104AB542A8BF3446AB42C8BF1C46B4
:1058E80006EE104AB8EEC66A072A81ED066A3FF44A
:1058F800C4AB90ED1C6A9DED195A65EE865AE7EE29
:10590800055AE6EEA57AFDEEE77A17EE900A86428A
:10591800A8BF06468342C8BF1E4607EE906AF8EE47
:10592800E77AC1ED077AFFF7A5BBDFED0F6AFEF74F
:105938003DBEB5EEC07AF1EE10FA01F1C282B7EEC3
:10594800006A36EE477AC6EE076AFEF7B6BDDFEDA7
:10595800066AFEF722BD00BFE83D0020EC3D0020AE
:105968000C3B0020D46600200000C842145C0020D4
:10597800CB4BDFF890A30693FEF7C2BBC94A537915
:10598800002B3EF4E6A8C84B1B78002B3EF4E1A898
:105998001278DFEDC64A07EE902AC54AB8EE677A54
:1059A800128807EE903A06EE902AF8EEE77AF8EEBB
:1059B800666A67EE277AB7EE007A87EEA63AB4EE03
:1059C800E43AF1EE10FA88BFB0EE643AB4EEC73AA2
:1059D800F1EE10FAB8BFB0EE473AFEF7BCB8B9F826
:1059E800CE2102F57A7292B2FEF7EABBB14A52882A
:1059F800FEF7E6BBB04A059207EE103A1278AF49B7
:105A08000691B8EEC77AF7EE006A0023132AB1F9B7
:105A180004009BED070AB9F81041C9F80C3186EE6D
:105A2800879A01F05F82A64BA64A02EB8405002103
:105A3800C9F80011C9F8041167EE897A93ED001AC4
:105A4800D3ED053A93ED122A93ED173AD3ED091ADF
:105A5800D3ED0E4A93ED016A93ED064A93ED0A7A67
:105A6800D3ED0F5AD3ED132AD3ED186A93ED045AE8
:105A7800D3ED030A69EE288A29EE088AE1EE273A6F
:105A8800A2EE283AE1EE884AA6EE274AE7EE085A3F
:105A980093ED167A93ED0D6A93ED021AD3ED0C1A75
:105AA800C5ED003AE2EEA86A25EE635A27EE437A7E
:105AB80093ED0B2AD3ED152AC5ED204AA0EEE34A53
:105AC80026EE646AD3ED143A83ED054AA1EE275A0F
:105AD800F0EE477AE1EEE45AA2EE086AE2EEC36A13
:105AE800E3EEA87A83ED065AC3ED0E5A83ED0F6AEA
:105AF80085ED403AC3ED176AC3ED187AC9F8081165
:105B0800631C03F01F03A9F81031069B9880059BBE
:105B1800FDF7A6BC6C4B93ED006AFFF718B86B4E07
:105B28003278013A0A2A20D8DFE812F0FA06760716
:105B38002B0710071F001F0034066307D5060B004C
:105B4800BA06634B1B78002B02F0FB821A2017F071
:105B5800E7FE002842F0F5825E4B1B78002B42F0EE
:105B6800F0820923337015F05BFE2379012B00F0D6
:105B78002986022B7EF447AD3378012B7EF443ADA2
:105B8800544B1B78002B7EF43EAD16F07FFDFEF7DC
:105B98003ABD514B9FED517AD3ED087AF4EEC77AAE
:105BA800F1EE10FA00F2FF849FED4D7A4D4ED6EDDE
:105BB800037A77EE877AC6ED037AFEF7E9BA05F03D
:105BC80097FF0A90FDF787BC3C4B069305F090FFC2
:105BD800454AD9F8743112680B90C31AC9F8740190
:105BE80006989A1A8380C280FDF7BABE3F4B9B7B0A
:105BF800002B3EF4C0AAFEF7C3BAD0003FF587AB2E
:105C0800FEF7CBBAB9F884219A4200F2178526200C
:105C180017F02AFE002840F01185354B354AD3EDA0
:105C2800007A354B92ED007A1B78C9ED627A89EDDE
:105C3800637A002B01F0A48577EE676A99F99031B1
:105C4800C9ED5F6A0133C9ED607A02F0F780079BFE
:105C5800C9F8943100229FED227A284989ED667AA5
:105C6800FF2391ED005A89F89031FEF74BBF0120D0
:105C780006F09CF8D9F86431079AD31AFDF7E0BC0E
:105C88001F4BD8ED007A93ED007AF0EEE77AF4EE48
:105C9800C77AF1EE10FA7DF739AEFDF731BE00BFD5
:105CA800D466002084600020C65E0020713DAA3FB3
:105CB800045E0020AC2E0020A85E0020AC5E002010
:105CC800F83500208C3300205C6A002090640020A6
:105CD8002E3D00202F3D0020843D00208FC2753CC2
:105CE80000000000C85E0020143D00207857002006
:105CF800603B0020703E002008400020843E0020C9
:105D0800946A0020145C002090ED016A26EE646A13
:105D1800B0EE674AA6EE074AB4EEC54A34EE666AA4
:105D2800F1EE10FA48BFB0EE656A012B81ED006A0A
:105D38003FF41EAE90ED056A26EE646AB0EE674A3F
:105D4800A6EE074AB4EEC54A34EE666AF1EE10FADA
:105D580048BFB0EE656A022B81ED016A3FF408AED8
:105D680090ED096A26EE646AB0EE674AA6EE074A25
:105D7800B4EEC54A34EE666AF1EE10FA48BFB0EEEA
:105D8800656A032B81ED026A3FF4F2AD90ED0D6A6E
:105D980026EE646AB0EE674AA6EE074AB4EEC54A34
:105DA80034EE666AF1EE10FA48BFB0EE656A042B6D
:105DB80081ED036A3FF4DCAD90ED116A26EE646A6A
:105DC800B0EE674AA6EE074AB4EEC54A34EE666AF4
:105DD800F1EE10FA48BFB0EE656A052B81ED046A52
:105DE8003FF4C6AD90ED156A26EE646AB0EE674AD8
:105DF800A6EE074AB4EEC54A74EE666AF1EE10FAEA
:105E080048BFF0EE656A062BC1ED056A3FF4B0ADF8
:105E1800D0ED196A66EEE46AB0EE674AA6EE874AE4
:105E2800B3EE046AB4EEC54A74EE466AF1EE10FAAF
:105E380048BFF0EE656A072BC1ED066A3FF498ADDE
:105E4800D0ED1D6ACC4BDFF850A3069366EEE44A0A
:105E5800E4EE877AF4EEC57A77EEC67AF1EE10FAB8
:105E6800B8BFF0EE657AC1ED077AFEF749B9C34DC0
:105E7800D9ED017A99ED006A28886B6977EEA77ADF
:105E8800F0EE006AB0EE677AA6EE267A013809EBE2
:105E9800C002D6EE267A083A1033F6EE003A27EE1C
:105EA800237A67EEA37A89ED207AC9ED217ADFF8A3
:105EB800E4924D4609F1800192ED027A92ED036A6F
:105EC800D5ED036AD5ED027A53ED014A13ED025A76
:105ED80037EE674A76EEC65A77EE277AE4EE845AAA
:105EE8000138A2F10802E5EE047A05F1080503F18C
:105EF800080336EE267A01F10801E4EE877AE5EE2A
:105F0800475A67EEA37A25EEA37AC1ED007A81EDB0
:105F1800017AD1D1142E7EF425AC05F0E9FD069A5C
:105F2800974B801A5880D9F81441FEF71BBCD9F852
:105F380018C1B9F81071934BC7F120085FFA88F8B7
:105F480007EB4C1503EB85055FEA980302F0F48034
:105F5800013318018C498D4A05EB000E05F1100339
:105F680013ED024A13ED035A13ED016A13ED047A97
:105F780051ED024A51ED035A51ED016A51ED047A8F
:105F880064EE244A65EE255A66EE266A67EE277A9D
:105F980010339E4542ED024A42ED035A42ED016A32
:105FA80042ED047A01F1100102F11002D8D17849CA
:105FB800A0F11002154401EB020E4A4418F0030345
:105FC80009D0B5EC017AFEEC017A67EE277A013B3D
:105FD800E2EC017AF5D1002F41F00080142E7EF416
:105FE800C1AB05F085FD069A654BD9F81441801AB6
:105FF8005880FEF7B7BB614D2A88D5F804E04FEA10
:10600800520C4FEA8C01D70809EB010309EB820413
:1060180000F0A08001F1100201375C4803EB07177C
:10602800224410330EF1100604F1100151ED032A39
:1060380051ED043A10ED043A10ED032A51ED026ACD
:1060480011ED016A10ED020A10ED018A12ED044A01
:1060580012ED035A53ED044A53ED035A13ED027A35
:1060680053ED017A52ED020A12ED011A73EE238AFA
:1060780072EE221A40ED048A40ED031A70EE268A69
:1060880078EE061A40ED028A40ED011A74EE848A11
:1060980075EE851A43ED048A43ED031A77EE208ADC
:1060A80077EE811A43ED028A43ED011A73EE633AE3
:1060B80075EE655A16ED035A32EE623A74EE644A8A
:1060C80065EE631A16ED044A23EE052A64EE652A86
:1060D800E3EE041A10339F4224EE843AA3EE842A96
:1060E80000F1100006F11006A5EE853A01F1100145
:1060F80002F11002E4EE852A41ED071A01ED082AA3
:1061080002ED073A42ED082A56ED055A16ED065AF1
:1061180070EE666A38EE466A30EEC77A71EE677AD4
:1061280026EE253A65EEE63A25EE674A67EE054A19
:10613800E6EE053AA6EE853AA7EE254AE7EEA54A29
:1061480001ED063A41ED053A02ED064A42ED054AEF
:106158007FF46CAF1FFA8CF6724631460D4822F078
:1061680007FC31466A68204622F002FC059B1B7832
:10617800142B7FF4D8AED0E6D46600207433002008
:10618800AC5E00208C3300201C350020A41D0020AC
:106198000C350020941D0020145C0020D94D2A786D
:1061A800970802F0C581D84807F1010C4FEA4C1C4A
:1061B80000EB0C0E00F12003A0F1700113ED076A4B
:1061C80053ED056A13ED037A53ED017A53ED025A44
:1061D80013ED084A53ED064A13ED045A26EE066AF3
:1061E80066EEA66A27EE077A67EEA77AA4EE046A37
:1061F80020339E45E4EEA46A01F11001A5EE057A6C
:10620800E5EEA57AF1EEC65AB1EEE66AF1EEC76A96
:10621800B1EEE77A41ED085A01ED076A41ED066AE9
:1062280001ED057ACAD1ACF12003034409EB071745
:1062380012F0030118BF08330FD053ED017A13EDA4
:10624800027A67EEA77A0139E7EE077A03F10803C5
:10625800B1EEE77AA7EC017AEFD1142E01F0CE87E0
:106268000134C9F81441FEF7EEB9A84DA848AA6848
:10627800A98927F07BF9059B1E78142E01F0D58794
:10628800D9F814410134C9F81441F1E5D9F81821B5
:10629800A04BA149A14C1846D30019441A448B8835
:1062A800016800EE103A10EE103A643BC82BA8BF04
:1062B800C823782BB8BF782307EE903AB8EEC07A97
:1062C800F8EEE77A04EB820477EE670A77EE876ADE
:1062D80067EE877A20EEA67AB8EE400AC7EE870AFC
:1062E8002046D4F81880E769256A94ED058A22F0DB
:1062F8001FFE059B84ED058A1E78C4F81880142EAD
:10630800E761256201F08787D9F81831844AD9F8FE
:106318001441013382FB0312A2EBE37C0CEB4C0229
:10632800A3EB020C0134C9F818C1C9F8144100E6FE
:10633800BEF1000F41F0DA8090ED006A9DED125A2F
:10634800784925EE866AFDEEE44AA5EE076AB0EEC6
:10635800675AA6EE265A14EE903ABDEEC56A16EEB6
:10636800105A16EE104AB542A8BF3446AB42C8BF11
:106378001C4606EE104AB8EEC66A012A81ED006A8C
:106388003DF4BBAE90ED046A9DED135A25EE866A86
:10639800A5EE076AB0EE675AA6EE265ABDEEC56AA4
:1063A80016EE105A16EE104AB542A8BF34469D4262
:1063B800B8BF1C4606EE104AB8EEC66A022A81ED3E
:1063C800016A3DF49AAE90ED086A9DED145A25EEE7
:1063D800866AA5EE076AB0EE675AA6EE265ABDEEA3
:1063E800C56A16EE105A16EE104AB542A8BF3446D2
:1063F8009D42B8BF1C4606EE104AB8EEC66A032A8C
:1064080081ED026A3DF479AE90ED0C6A9DED155A66
:1064180025EE866AA5EE076AB0EE675AA6EE265AFA
:10642800BDEEC56A16EE105A16EE104AB542A8BF60
:1064380034469D42B8BF1C4606EE104AB8EEC66AFE
:10644800042A81ED036A3DF458AE90ED106A9DED83
:10645800165A25EE866AA5EE076AB0EE675AA6EECA
:10646800265ABDEEC56A16EE105A16EE104AB54207
:10647800A8BF34469D42B8BF1C4606EE104AB8EE87
:10648800C66A052A81ED046A3DF437AE90ED146AB8
:106498009DED175A25EE866AA5EE076AB0EE675A93
:1064A800A6EE265ABDEEC56A16EE105A16EE104A2A
:1064B800B542A8BF34469D42B8BF1C4606EE104AF6
:1064C800B8EEC66A062A81ED056A3DF416AE90ED6F
:1064D800186A9DED185A25EE866AA5EE076AB0EE91
:1064E800675AA6EE265ABDEEC56A16EE105A16EE83
:1064F800104AB542A8BF34469D42B8BF1C46FDF7B6
:10650800DABD00BF6E330020141E00207433002053
:10651800941D0020045C002064360020845B002069
:10652800565555550C3B0020C74BB8F908101A684A
:1065380002B111609B69B8F90A20002B00F0F380C2
:106548001A60032604220225DAF80030990600F1C1
:10655800DA86DB027DF5D9ADBC4BDE7B112E3DF72B
:10656800D4ADBB4C34F9163000EE103A2846B8EEDC
:10657800C00A1EF04FF904EB46040127C6F11206C3
:10658800E819B742C0B207F101073DF4BEAD34F9CE
:10659800023F00EE103AB8EEC00A1EF03BF90E2F8B
:1065A800EED1FDF7B2BDF0EEE76AB7EE005A35EE70
:1065B800665A9FEDA84ADFEDA85A9FEDA86A9FED9D
:1065C800A87A99ED720AF1EEC54AE6EE845AF5EE1C
:1065D800C07AA6EEA56AF1EE10FAA6EE867A48BF52
:1065E800DFEDA07A27EE247A48BF37EEC77A27EE88
:1065F800000A28F0C9F8B0F5617F01F3B58007EE0D
:10660800900AB8EEE70ADFED987A20EE270A07EE3F
:10661800904AB8EEE78AFDEEC07A17EE903A20333A
:10662800402B41F2A7809FED910A28F0ADF800B207
:1066380007EE900AB8EEE77AFFF7B8BA99F89C2106
:10664800002A7FF4EAAA8A4B8A4993ED007AD1EDB1
:10665800007A99F99031C9ED627A77EE676A012B71
:10666800C9ED607AC9ED5F6A89ED637A01F0B88592
:10667800079BC9F89431804B9FED7C7A93ED005AC3
:1066880089ED667A012389F89031FEF73BBA704BA1
:1066980033F91250FEF718BD6B4BB8F900101A68A1
:1066A80002B111609A69B8F9021002B111601A6B4F
:1066B800B8F9041002B111609B6CB8F90620002BE0
:1066C80001F05B871A600526062204253CE76B4D1E
:1066D800002435F9023F00EE103AE0B2B8EEC00AE5
:1066E80001341EF097F8062CF3D1204631E0644DB2
:1066F800002435F9023B00EE103AE0B2B8EEC00AC9
:1067080001341EF087F8042CF3D1204621E04E4BCB
:10671800B8F906101A6802B111609B69B8F9082027
:10672800002B7FF40DAF0326042202250CE7474B0C
:106738009B7B002B41F01982524B1B7813F001030D
:1067480041F01382404A1268002A01F06E871360F4
:106758000120DAF800309A0604D44B4A1278052A48
:1067680040F03484851C461CEDB2F6B2B8F900300E
:1067780000EE103AB8EEC00A1EF04CF8B8F9023034
:1067880000EE103A3046B8EEC00A1EF043F8DAF8C8
:106798000030DEE625F0A4FC3C4B002105208DE806
:1067A8000300A3F108020291532015F067FD0028A9
:1067B8007FF4DBA9364A0823106033702379012B54
:1067C8007DF421AF334F2F4B1B78DC0740F1B180AC
:1067D800D9F828223B689A423FF6CEA93378012B94
:1067E8003DF411AF2C4C2278002A3DF40CAF0B2B52
:1067F80018D801229A4040F6030112EA010816D17E
:1068080012F4C06F0ED0093B012B0BD8452025F0A0
:10681800ABFCFF2025F0A8FC204825F091FC404661
:1068280025F0A2FC1A4B3A685A600B2333700023F8
:106838002370FDF7E8BED9F89421079B9A1AFEF752
:1068480051B9002085E700BF8857002078570020FD
:10685800BC4E0020306E99BC2716983D843459BE32
:10686800A40DC93FDB0F4940D06D393A0000000044
:10687800B83C00206C3E0020883E0020FE3A0020F4
:10688800023B00208562002060690020A8FA020807
:10689800BC3C0020946F00202F3D0020041E0308FC
:1068A800AB4AAC4F52683968C8328A4205D325F0E2
:1068B80037FC00283FF459A9A378032B01F0EE8692
:1068C80023790122934232703FF47DAF022B3FF4CB
:1068D80057A9FDF798BE1A2017F022F800283FF4B0
:1068E80042A99D4B1B88002B7FF43DA99B4B45205B
:1068F8001F6825F039FC0E2025F036FC384614F0C8
:106908001BFC079F384614F017FC954A954B1268F4
:106918001A6038460A23337014F0D6FCFFF723B9FF
:10692800914B1B78DF0701F11E862379012BCDD10E
:10693800884F16F001FF00283FF44AAF3B6803F583
:106948009C530833C9F82832FFF716B925F0C8FB5D
:10695800864A0292A2F10C03252101930091A2F12B
:106968000A035021163A492015F088FC00287FF4C4
:10697800FCA8774B4FF0FF3107221860596032703E
:106988001CE7DFF8CC81734F25F0AAFBD8F8043058
:106998003A6864339342BFF4E8A8402025F084FBAA
:1069A80000287FF4E2A8D8F80030714FDFF8C4A1BE
:1069B8004FF0400B0FE025F0D7FBDAF80020D8F8AD
:1069C8000030013A0133BBF1010BCAF80020C8F8C6
:1069D800003001F0D386FB5C1846002BEBD1002376
:1069E8004FF0FF32C8F800300423C8F80420337091
:1069F800E4E625F075FB14F045FF00283FF4B5A840
:106A080025F08EFB00283FF4B0A8554A554B126874
:106A18001A600A233370D1E64E4F4D4A3B685360E3
:106A280054490023136003220B603270C6E6B6F99E
:106A38001440FEF757BB504B504AD3ED006A504BF9
:106A480092ED006A1B78C9ED626A89ED636A002BD2
:106A580000F0BF8276EE665A99F99031C9ED5F5A17
:106A68000133C9ED606A01F07A80079BC9F8943157
:106A7800002237EE677AFCEEE77A424989ED667ABA
:106A880017EE903AA9F88431FF2391ED005A89F85E
:106A98009031FEF737B83C4BDFED3C7A1C683C4B35
:106AA80099ED667AC3ED007AF0EE674AC3ED017A94
:106AB800C3ED027AF0EE673AFCF78CBF05F018F8E0
:106AC800059B06901E78142E05BF324BD9F8144149
:106AD800D9F814411C80FCF7CBBC2F4BDFED2F7A83
:106AE8001B68C9ED4A7A13F0805C40F05D86DAF8DD
:106AF800003013F4800C00F00A844FF0000CB6EE5E
:106B0800007A67EE877AF4EEE75AF1EE10FA48BF9A
:106B1800F0EE675A40F14886C9ED665AFDF79BB911
:106B2800114B187800F00107FDF7E7BA73EEE77A22
:106B3800B7EE007AF4EEC77AF1EE10FAC9ED4A7AA8
:106B480041F3548384EEA77A8DED127AFDF779B973
:106B5800BC3C0020946F00204C3B0020483B0020A8
:106B6800303B00202C3B002085620020FAF8020808
:106B780094F80208286B0020603B0020703E00203B
:106B880008400020843E0020EC6000200000000047
:106B9800E43A0020AC5E00203C3B0020000000806E
:106BA800B8F1000F01F0A28125EE866AC749A5EE6B
:106BB800076AB0EE675AA6EE265ABDEEC56A16EE0B
:106BC800105A16EE104AB542A8BF3446AB42C8BFA9
:106BD8001C4606EE104AB8EEC66A012A81ED006A24
:106BE8003DF48EAA90ED046A9DED135A25EE866A4F
:106BF800A5EE076AB0EE675AA6EE265ABDEEC56A3C
:106C080016EE105A16EE104AB542A8BF3446AB42EB
:106C1800C8BF1C4606EE104AB8EEC66A022A81EDC5
:106C2800016A3DF46DAA90ED086A9DED145A25EEAF
:106C3800866AA5EE076AB0EE675AA6EE265ABDEE3A
:106C4800C56A16EE105A16EE104AB542A8BF344669
:106C5800AB42C8BF1C4606EE104AB8EEC66A032A05
:106C680081ED026A3DF44CAA90ED0C6A9DED155A2F
:106C780025EE866AA5EE076AB0EE675AA6EE265A92
:106C8800BDEEC56A16EE105A16EE104AB542A8BFF8
:106C98003446AB42C8BF1C4606EE104AB8EEC66A78
:106CA800042A81ED036A3DF42BAA90ED106A9DED4C
:106CB800165A25EE866AA5EE076AB0EE675AA6EE62
:106CC800265ABDEEC56A16EE105A16EE104AB5429F
:106CD800A8BF3446AB42C8BF1C4606EE104AB8EE01
:106CE800C66A052A81ED046A3DF40AAA90ED146A81
:106CF8009DED175A25EE866AA5EE076AB0EE675A2B
:106D0800A6EE265ABDEEC56A16EE105A16EE104AC1
:106D1800B542A8BF3446AB42C8BF1C4606EE104A6F
:106D2800B8EEC66A062A81ED056A3DF4E9A990ED38
:106D3800186A9DED185A25EE866AA5EE076AB0EE28
:106D4800675AA6EE265ABDEEC56A16EE105A16EE1A
:106D5800104AB542A8BF3446AB42C8BF1C4606EE2F
:106D6800104AB8EEC66A072A81ED066A3DF4C8A93A
:106D780090ED1C6A9DED195A65EE865AE7EE055AA4
:106D8800E6EEA57AFDEEE77A17EE902A9642A8BFBE
:106D980016469342D8BF334607EE903AF8EEE77AA4
:106DA800C1ED077AFDF7ACB9DFED497AFDF795BC7F
:106DB8008223FDF7C6BCBBF93830CBF8202007EE9C
:106DC800903A0122F8EEE77ACBF86030CBF87C20D5
:106DD8000023012DCBED1C7ACBED1B7ACBF8743058
:106DE80001F0AB83B5427DF468AFBBF93A30CBF81C
:106DF800643007EE903A00220123F8EEE77ACBF8E8
:106E08002420CBF890300023012DCBED217ACBED57
:106E1800207ACBF8883001F09783B5427DF480AFB3
:106E2800BBF93C30CBF8683007EE903A00220123DA
:106E3800F8EEE77ACBF82820CBF8A4300023012D10
:106E4800CBED267ACBED257ACBF89C307DF49BAF41
:106E58009FED208A032C2AD04FB107EE907AF8EEE6
:106E6800E77AF4EEC87AF1EE10FA01F1D6831A4BFC
:106E7800DFF86C901A68069B99F82011D880DBF827
:106E8800683003EB560393FBF6F60023CBF8286033
:106E980093621363D36229B1104B1B6833F4806388
:106EA8007DF475AF012020F0B5FFFDF770BFB0EE9F
:106EB800480A27F069FC00B2CEE7F7EE006AFDF752
:106EC80075BBF7EE006AFDF7F8BA00BF0C3B00206F
:106ED80000000243000000007C540020E460002011
:106EE800941D0020B14DB24E95ED004A95ED057AFE
:106EF800D5ED014A95ED066AD5ED046A95ED035A7C
:106F0800D5ED025A67EE897A06EB8403A4EE277A58
:106F1800A4EEA76A66EEC76AA5EE476AE5EEA76A19
:106F280020EE070A85ED056AC5ED066A29EE088A8E
:106F380069EE288A83ED007A27F026FCD5ED0E5AF3
:106F4800D5ED176A95ED091AD5ED121A95ED0F5A78
:106F580095ED187A95ED0A2AD5ED132A95ED0D6A67
:106F6800D5ED167A95ED0C3AD5ED0B3A95ED154A17
:106F7800D5ED144AE1EE085A002206EB8401E8EE4A
:106F8800A16A00B2C9F80021A2EE085AC9F8042182
:106F9800C9F80821A8EEA27A26EE656A67EEE67AB5
:106FA800A3EE655AA3EE886AA6EEC47AE8EEA47A40
:106FB80085ED0E5AC1ED205A85ED0F6AC1ED406A84
:106FC80085ED177AC5ED187AFEF79ABD0546FFF7E5
:106FD800C0BA76EEC65AF0EE466A3DE5744B4FEA03
:106FE80088055FEA9708294403EBCC1C4D4437D049
:106FF80008F101084FEA08180CEB080E0CF1100311
:1070080001F1100005F1100213ED024A13ED035AC5
:1070180013ED016A13ED047A50ED024A50ED035A5C
:1070280050ED016A50ED047A64EE244A65EE255A63
:1070380066EE266A67EE277A10339E4542ED024ACD
:1070480042ED035A42ED016A42ED047A00F1100064
:1070580002F11002D8D1A8F11008C44441444544B3
:1070680017F003073EF4BAAFBCEC017AF1EC017AF1
:1070780067EE277A013FE5EC017AF5D1FEF7AEBF5E
:107088004C4B1B88DC0541F161804B4E4B4B96ED18
:10709800017A0F93D6ED006AD6ED027AB3F906703D
:1070A800069BBDEEC77A198BFDEEE66A17EE103A1D
:1070B800FDEEE77A16EE902AADF84A3017EE903AD0
:1070C800ADF84820ADF84C303D4A3E4CB2F902309C
:1070D800B2F900203C489FED3D7AD0ED007A3C485B
:1070E800DFF8FC8000780E904FF47A7503F5E163C1
:1070F80005FB03F302F5E16205FB02F284FB03657D
:107108001D44DB17C3EBE5230F9D77EEC77A84FB9D
:1071180002642E88FDEEE77A761AA3F5FA73144412
:10712800ADF86030D21717EE903AADF850600F9E68
:10713800ADF84E30C2EBE42228462C466D88B38960
:107148000089A4886D1AA2F5FA725B1AADF862205C
:10715800ADF852507289F589ADF85C30401A0E9B33
:10716800ADF858007F1A0020641A521A691AADF84F
:107178005670ADF85440ADF85A20ADF85E10C8F816
:107188000000C8F80400C8F80800C8F80C00002B74
:1071980001F040820F4B104ECDF844900F4D0A96E7
:1071A8001F46CDF840A0814659E000BFF8350020C1
:1071B8008C330020E8600020C85E0020BC4E002010
:1071C80098600020C5B3A2910C3B00200080BB440E
:1071D800E8680020341F002024370020EC680020D5
:1071E800FC3A00201AAB03EB440030F9200C38803D
:1071F8000A9B95F902E00E441EFB00F053F8266046
:10720800012303FA04F4B64B83FB003EC0170C9B22
:107218003442C0EB6E100CBF01244FF0FF3498428B
:107228000EDB0D9B02FB03F2AD4B83FB0263D2170F
:10723800C2EB6313A3EB0C031BB28342A8BF034644
:1072480038F8112003FB042328F811300E9B09F1AC
:107258000109994505F1070507F1020761DAA879DF
:10726800002835D1297895F905200D924E000A9A03
:1072780095F9043095F803E06C78701802EB8000FB
:10728800C2888088121A92B2954802FB03F380FBE9
:1072980003C0DB17C3EB60134FEA520CA3EB0C03DC
:1072A8001BB20C93BEF1000F9CD01AAB03EB440A3F
:1072B800B7F900003AF920AC504511DA8644704518
:1072C80003DCF2455046A8BF704600B238808FE70D
:1072D8001630C0B216F024FB0028C3D13880B5E7B9
:1072E80086DDA0EB0E0ED64503DB7045A8BF7046C1
:1072F80082460FFA8AF038807AE77A4A1768B7F92F
:107308003240FEF70BB828461546FFF72FBAB6EEFF
:10731800007AF4EEC75AF1EE10FA3FF7F0ABFCF73B
:107328009ABD0A9EDDF840A0DDF8449096F90A104F
:10733800B8F800306C486A4A047811FB03F3F17A14
:1073480082FB0302FF294FEAE373C3EB621200F0EA
:1073580000848C4240F2FD830F9B33F9111096F99B
:107368001600B8F802301144A8F800105C4AF17D04
:1073780010FB03F382FB0302FF294FEAE373C3EB1D
:10738800621200F0E3838C4240F2E0830F9B33F9F2
:10739800111096F92200B8F804301144A8F8021028
:1073A8004F4A96F8231010FB03F382FB0302FF29D0
:1073B8004FEAE373C3EB621200F0C5838C4240F2DC
:1073C800C2830F9B33F9111096F92E00B8F80630D6
:1073D8001144A8F80410424A96F82F1010FB03F342
:1073E80082FB0302FF294FEAE373C3EB621200F04A
:1073F800A7838C4240F2A4830F9B33F9111096F9AE
:107408003A00B8F808301144A8F80610344A96F83B
:107418003B1010FB03F382FB0302FF294FEAE373DF
:10742800C3EB621200F089838C4240F286830F9B83
:1074380033F9111096F94600B8F80A301144A8F843
:107448000810274A96F8471010FB03F382FB030243
:10745800FF294FEAE373C3EB621200F06B838C429F
:1074680040F268830F9B33F9111096F95200B8F86F
:107478000C301144A8F80A10194A96F8531010FB5A
:1074880003F382FB0302FF294FEAE373C3EB6212A3
:1074980000F04D838C4240F24A830F9B33F9111060
:1074A80096F95E00B8F80E301144A8F80C100C4A92
:1074B80096F85F1010FB03F382FB0302FF294FEAE3
:1074C800E373C3EB621300F02F83A14280F02C8397
:1074D8000F9A32F911201344A8F80E30FDF7E6BDD3
:1074E8001F85EB51EC600020AC2E002090ED006A67
:1074F8009DED124AE14925EE866AFDEEE43AA4EED6
:10750800076AB0EE674AA6EE264A13EE903AB4EE42
:10751800C45AF1EE10FAB0EE446A88BFB0EE646A5D
:10752800BDEEC66A16EE105A16EE104AB542A8BF4E
:107538003446AB42C8BF1C4606EE104AB8EEC66ACF
:10754800012A81ED006A3CF4D8AD90ED046A9DED06
:10755800134A25EE866AA4EE076AB0EE674AA6EEDD
:10756800264AB4EEC45AF1EE10FAB0EE446A88BF67
:10757800B0EE646ABDEEC66A16EE105A16EE104AF0
:10758800B542A8BF34469D42B8BF1C4606EE104A15
:10759800B8EEC66A022A81ED016A3CF4AEAD90ED00
:1075A800086A9DED144A25EE866AA4EE076AB0EED5
:1075B800674AA6EE264AB4EEC45AF1EE10FAB0EEC7
:1075C800446A88BFB0EE646ABDEEC66A16EE105A09
:1075D80016EE104AB542A8BF34469D42B8BF1C46B5
:1075E80006EE104AB8EEC66A032A81ED026A3CF438
:1075F80084AD90ED0C6A9DED154A25EE866AA4EEE1
:10760800076AB0EE674AA6EE264AB4EEC45AF1EE0F
:1076180010FAB0EE446A88BFB0EE646ABDEEC66A7E
:1076280016EE105A16EE104AB542A8BF34469D42CF
:10763800B8BF1C4606EE104AB8EEC66A042A81EDA9
:10764800036A3CF45AAD90ED106A9DED164A25EE9A
:10765800866AA4EE076AB0EE674AA6EE264AB4EE3A
:10766800C45AF1EE10FAB0EE446A88BFB0EE646A0C
:10767800BDEEC66A16EE105A16EE104AB542A8BFFD
:1076880034469D42B8BF1C4606EE104AB8EEC66A9C
:10769800052A81ED046A3CF430AD90ED146A9DED45
:1076A800174A25EE866AA4EE076AB0EE674AA6EE88
:1076B800264AB4EEC45AF1EE10FAB0EE446A88BF16
:1076C800B0EE646ABDEEC66A16EE105A16EE104A9F
:1076D800B542A8BF34469D42B8BF1C4606EE104AC4
:1076E800B8EEC66A062A81ED056A3CF406AD90ED4F
:1076F800186A9DED184A25EE866AA4EE076AB0EE70
:10770800674AA6EE264AB4EEC45AF1EE10FAB0EE75
:10771800446A88BFB0EE646ABDEEC66A16EE105AB7
:1077280016EE104AB542A8BF34469D42B8BF1C4663
:1077380006EE104AB8EEC66A072A81ED066A3CF4DE
:10774800DCAC90ED1C6A9DED194A65EE865AE7EEB1
:10775800045AE6EEA57AB4EEE75AF1EE10FAC8BF7D
:10776800F0EE647AFCF7B9BC07EE904A9FED440A44
:10777800B8EEE78AFAF7CCFF20EE080AFEF755BF05
:1077880077EEC76AF0EE477AFEF758BABA8E9FEDE1
:107798003D7A07EE902AF8EEE77A3B4A67EE877A59
:1077A800C2ED007AFCF7F9BCB7EE007A77EE677A9B
:1077B800F4EEE75AF1EE10FA88BFF0EE675AFFF7D9
:1077C800ABB901297FF744AB07EE10EAB8EEC77AE8
:1077D800C7EE876AB1EEE68AFFF73CBB012940F3A2
:1077E800AC8607EE10EAB8EEC77AC7EE876AB1EE44
:1077F800E68A032C14D04FB107EE907AF8EEE77AB8
:10780800F4EEC87AF1EE10FA00F10787DBF8603081
:1078180003EB560393FBF6F3CBF82030FFF7E2BAFD
:10782800B0EE480A26F0B0FF00B2E4E7012940F3C1
:107838008B8607EE10EAB8EEC77AC7EE876AB1EE14
:10784800E68A032C14D04FB107EE907AF8EEE77A67
:10785800F4EEC87AF1EE10FA00F1DF86DBF8643056
:1078680003EB560393FBF6F3CBF82430FFF7D5BAB6
:10787800B0EE480A26F088FF00B2E4E70C3B00208F
:1078880084F9223F6F12833A0000002090ED006ACD
:107898009DED124ABA4925EE866AFDEEE43AA4EE59
:1078A800076AB0EE674AA6EE264A13EE904AB4EE8F
:1078B800C45AF1EE10FAB0EE446A88BFB0EE646ABA
:1078C800BDEEC66A16EE105A16EE103AB542A8BFBB
:1078D8003346AC42C8BF234606EE103AB8EEC66A35
:1078E800012A81ED006A3DF4C8AB90ED046A9DED74
:1078F800134A25EE866AA4EE076AB0EE674AA6EE3A
:10790800264AB4EEC45AF1EE10FAB0EE446A88BFC3
:10791800B0EE646ABDEEC66A16EE105A16EE103A5C
:10792800B542A8BF3346A542B8BF234606EE103A73
:10793800B8EEC66A022A81ED016A3DF49EAB90ED6D
:10794800086A9DED144A25EE866AA4EE076AB0EE31
:10795800674AA6EE264AB4EEC45AF1EE10FAB0EE23
:10796800446A88BFB0EE646ABDEEC66A16EE105A65
:1079780016EE103AB542A8BF3346A542B8BF234613
:1079880006EE103AB8EEC66A032A81ED026A3DF4A3
:1079980074AB90ED0C6A9DED154A25EE866AA4EE4F
:1079A800076AB0EE674AA6EE264AB4EEC45AF1EE6C
:1079B80010FAB0EE446A88BFB0EE646ABDEEC66ADB
:1079C80016EE105A16EE103AB542A8BF3346A54235
:1079D800B8BF234606EE103AB8EEC66A042A81ED0F
:1079E800036A3DF44AAB90ED106A9DED164A25EE08
:1079F800866AA4EE076AB0EE674AA6EE264AB4EE97
:107A0800C45AF1EE10FAB0EE446A88BFB0EE646A68
:107A1800BDEEC66A16EE105A16EE103AB542A8BF69
:107A28003346A542B8BF234606EE103AB8EEC66AFA
:107A3800052A81ED046A3DF420AB90ED146A9DEDB2
:107A4800174A25EE866AA4EE076AB0EE674AA6EEE4
:107A5800264AB4EEC45AF1EE10FAB0EE446A88BF72
:107A6800B0EE646ABDEEC66A16EE105A16EE103A0B
:107A7800B542A8BF3346A542B8BF234606EE103A22
:107A8800B8EEC66A062A81ED056A3DF4F6AA90EDBD
:107A9800186A9DED184A25EE866AA4EE076AB0EECC
:107AA800674AA6EE264AB4EEC45AF1EE10FAB0EED2
:107AB800446A88BFB0EE646ABDEEC66A16EE105A14
:107AC80016EE103AB542A8BF3346A542B8BF2346C2
:107AD80006EE103AB8EEC66A072A81ED066A3DF44A
:107AE800CCAA90ED1C6A9DED194A65EE865AE7EE20
:107AF800045AE6EEA57AB4EEE75AF1EE10FAC8BFDA
:107B0800F0EE647AFDEEE77A17EE903A9E42A8BF4F
:107B18001E469C42D8BF344607EE904AF8EEE77AF4
:107B2800C1ED077AFDF7A6BAB6F95C20D3E4B6F939
:107B38005010B5E4B6F9441097E4B6F9381079E472
:107B4800B6F92C105BE4B6F920103DE4B6F9141030
:107B58001FE4B6F9081002E40A4EFCF77CBBD9F81A
:107B68009421079B9A1AFEF784BF074BB8F90A209D
:107B78001B68002B00F059851A600120FEF7E9BD4B
:107B88000C3B0020C85E00208857002090ED006A5A
:107B98009DED124A25EE866AA4EE076AB0EE674AA2
:107BA800A6EE264AB0EE446AB8F1000F00F06C83E6
:107BB800BEF1000F06D0B4EE445AF1EE10FAC8BF79
:107BC800B0EE646AFDEEE44ABDEEC66A14EE904A71
:107BD80016EE103A9C4214EE905A00F31785B34201
:107BE800A8BF334606EE103AB849B8EEC66A012A6D
:107BF80081ED006A3CF484AA90ED046ADDED134A35
:107C080025EE866AA4EE876AF0EE674AE6EE264A13
:107C1800B0EE646ABEF1000F00F0EE84B4EEE45AF0
:107C2800F1EE10FA40F3E8842346B342A8BF334686
:107C380006EE103AB8EEC66A022A81ED016A3CF4F3
:107C48005FAA90ED086ADDED144A25EE866AA4EE77
:107C5800876AF0EE674AE6EE264AB0EE646ABEF13D
:107C6800000F00F0BF84B4EEE45AF1EE10FA40F3CE
:107C7800B9842346B342A8BF334606EE103AB8EE9D
:107C8800C66A032A81ED026A3CF43AAA90ED0C6AAE
:107C9800DDED154A25EE866AA4EE876AF0EE674A9E
:107CA800E6EE264AB0EE646ABEF1000F00F090845A
:107CB800B4EEE45AF1EE10FA40F38A842346B34254
:107CC800A8BF334606EE103AB8EEC66A042A81ED1C
:107CD800036A3CF415AA90ED106ADDED164A25EE0C
:107CE800866AA4EE876AF0EE674AE6EE264AB0EEA8
:107CF800646ABEF1000F00F06184B4EEE45AF1EE5C
:107D080010FA40F35B842346B342A8BF334606EE1D
:107D1800103AB8EEC66A052A81ED046A3CF4F0A967
:107D280090ED146ADDED174A25EE866AA4EE876A9F
:107D3800F0EE674AE6EE264AB0EE646ABEF1000F3E
:107D480000F03284B4EEE45AF1EE10FA40F32C84D9
:107D58002346B342A8BF334606EE103AB8EEC66AC9
:107D6800062A81ED056A3CF4CBA990ED186ADDED91
:107D7800184A25EE866AA4EE876AF0EE674AE6EEB0
:107D8800264AB0EE646ABEF1000F00F00384B4EE38
:107D9800E45AF1EE10FA40F3FD832346B342A8BF3C
:107DA800334606EE103AB8EEC66A072A81ED066A2F
:107DB8003CF4A6A990ED1C6ADDED194A65EE865AD9
:107DC800E4EE875AE5EEA67ABEF1000F00F0DA83FA
:107DD800F4EEC57AF1EE10FA40F1D4832346B342AB
:107DE800A8BF33461D4607EE905AF8EEE77AC1ED74
:107DF800077AFCF785B9364996F916700B8896F913
:107E08000A20B1F90200334917FB03F3524200FB81
:107E180002F081FB0372121181FB0071DB17C0179E
:107E2800C0EB2110991AD31A01440344691A1C445F
:107E3800A8F80010A8F80240FDF792B9D9F89421E3
:107E4800079B9A1AFDF707BF07EE904AB8EEE79A24
:107E5800DFED217A89F8204229EE279AB0EE490A07
:107E6800FAF73EFDFDEEC97A1C4A17EE903A203328
:107E7800402BF0EE408A82ED010A00F26283B0EEF8
:107E8800490AFAF745FC89ED890AFDF7A4BA96ED87
:107E9800000A089326F078FC114A1249D2F8EC201F
:107EA800DFF844E081FB0231D217C2EBA11207EEE2
:107EB800902AF8EEE77AAEF80000FDEEE77A089B24
:107EC80017EE902AAEF80220FCF7CAB90C3B002046
:107ED800986000201F85EB5135FA8E3C0000002089
:107EE80028010020D34D6210AC5E002025EE866A82
:107EF800A5EE076AB0EE675AA6EE265ABDEEC56A29
:107F080016EE101A8B4200F3A681B142A8BF314683
:107F180006EE101AB8EEC66ABCF1000F00F05D84D8
:107F2800CE49012A81ED006A3CF4EAA890ED046A82
:107F38009DED135A25EE866AA5EE076AB0EE675ADC
:107F4800A6EE265ABDEEC56A16EE104AA34200F305
:107F58007C81B442A8BF344606EE104AB8EEC66A21
:107F6800BCF1000F00F01084022A81ED016A3CF494
:107F7800C7A890ED086A9DED145A25EE866AA5EE0D
:107F8800076AB0EE675AA6EE265ABDEEC56A16EE27
:107F9800104AA34200F35D81B442A8BF344606EEFE
:107FA800104AB8EEC66ABCF1000F00F02184032A1B
:107FB80081ED026A3CF4A4A890ED0C6A9DED155A77
:107FC80025EE866AA5EE076AB0EE675AA6EE265A2F
:107FD800BDEEC56A16EE104AA34200F33881B442DA
:107FE800A8BF344606EE104AB8EEC66ABCF1000FC8
:107FF80000F0DF83042A81ED036A3CF481A890ED48
:10800800106A9DED165A25EE866AA5EE076AB0EE4F
:10801800675AA6EE265ABDEEC56A16EE104AA34266
:1080280000F30F81B442A8BF344606EE104AB8EEFA
:10803800C66ABCF1000F00F04A83052A81ED046A84
:108048003CF45EA890ED146A9DED175A25EE866AF9
:10805800A5EE076AB0EE675AA6EE265ABDEEC56AC7
:1080680016EE104AA34200F3EA80B442A8BF344691
:1080780006EE104AB8EEC66ABCF1000F00F0A38302
:10808800062A81ED056A3CF43BA890ED186A9DED3F
:10809800185A25EE866AA5EE076AB0EE675AA6EE6C
:1080A800265ABDEEC56A16EE104AA34200F3CB80ED
:1080B800B442A8BF344606EE104AB8EEC66ABCF110
:1080C800000F00F05183072A81ED066A3CF418A8D6
:1080D80090ED1C6A9DED195A65EE865AE7EE055A31
:1080E800E5EEA67AFDEEE77A17EE902A934204DCD5
:1080F800B24217EE903AA8BF334607EE903AF8EE30
:10810800E77ABCF1000F7FF472AE0C9B002B7FF472
:108118006EAE0A9B9D42B8BFF0EE647A67E69FEDAB
:10812800500A504B25EE800A1C4626F02DFBE080B5
:10813800D9F81441FCF716BB4B494C4A8E46FDF75B
:108148003DBF079813F0C0F8FDF70DBD484B9FEDF4
:10815800496A93ED007A484BDAF80010D3ED003AFB
:10816800434BD3ED017A444B93ED014A404BD3ED99
:10817800026A414BD3ED024A404B37EE237A93ED26
:10818800005AD3ED015A77EE847A37EE057A77EE06
:10819800A57A76EEA46A27EE067A67EE867A66EE08
:1081A800866ABDEEC77AFDEEE77AFDEEE66A17EE5F
:1081B800100A17EE903ACDED0A6ABDF92820ADF8FD
:1081C8004800ADF84A30C8042D4BADF84C200F9349
:1081D80000F1BE81069AB3F90670118BFEF774BFE1
:1081E800D9F89421079B9A1AFEF745BA254B1B68C4
:1081F80013F0805C7EF483ACFEF779BC03F078FC66
:108208000599184B0E7806992A78D9F81441401A1E
:108218009880FEF725B803F06BFC059A114B167889
:10822800069A801A5880FEF76FB803F061FC059A29
:108238000C4B1678069A801A5880FEF721B81C460F
:1082480016E71C46F1E61C4635E71C4684E61C4644
:10825800C8E61C46A3E619465AE600BF0C3B0020B8
:108268000000C842AC5E00200C350020941D0020A0
:10827800D83A00203333333FE43A0020F03A002064
:10828800BC4E00203C3B0020BEF1000F06D0B4EEEF
:10829800445AF1EE10FAC8BFB0EE646ABDEEE44A83
:1082A800BDEEC66A14EE104A16EE103A9C4214EE61
:1082B800107A00F3D181B342A8BF334606EE103AD4
:1082C800B8EEC66ABCF1000F00F0A782EF49012A98
:1082D80081ED006A3BF414AF90ED046A9DED134AFA
:1082E80025EE866AA4EE076AB0EE674AA6EE264A2D
:1082F800B0EE446ABEF1000F05D0B4EEC45AF1EEF8
:1083080010FA00F39581BDEEC66A16EE103AA34244
:10831800B8BF234680F28D8106EE103AB8EEC66AE1
:10832800BCF1000F00F0D082022A81ED016A3BF413
:10833800E7AE90ED086A9DED144A25EE866AA4EE34
:10834800076AB0EE674AA6EE264AB0EE446ABEF166
:10835800000F05D0B4EEC45AF1EE10FA00F36D81A7
:10836800BDEEC66A16EE103AA342B8BF234680F2A5
:10837800658106EE103AB8EEC66ABCF1000F00F04F
:108388009982032A81ED026A3BF4BAAE90ED0C6A39
:108398009DED154A25EE866AA4EE076AB0EE674A97
:1083A800A6EE264AB0EE446ABEF1000F05D0B4EE40
:1083B800C45AF1EE10FA00F34581BDEEC66A16EE16
:1083C800103AA342B8BF234680F23D8106EE103A28
:1083D800B8EEC66ABCF1000F00F08082042A81ED75
:1083E800036A3BF48DAE90ED106A9DED164A25EEBA
:1083F800866AA4EE076AB0EE674AA6EE264AB0EE91
:10840800446ABEF1000F05D0B4EEC45AF1EE10FA7A
:1084180000F31D81BDEEC66A16EE103AA342B8BF3E
:10842800234680F2158106EE103AB8EEC66ABCF112
:10843800000F00F0E881052A81ED046A3BF460AE84
:1084480090ED146A9DED174A25EE866AA4EE076A38
:10845800B0EE674AA6EE264AB0EE446ABEF1000FB7
:1084680005D0B4EEC45AF1EE10FA00F3F880BDEE70
:10847800C66A16EE103AA342B8BF234680F2F080CF
:1084880006EE103AB8EEC66ABCF1000F00F087811C
:10849800062A81ED056A3BF433AE90ED186A9DED2E
:1084A800184A25EE866AA4EE076AB0EE674AA6EE79
:1084B800264AB0EE446ABEF1000F05D0B4EEC45AA5
:1084C800F1EE10FA00F3D080BDEEC66A16EE103A4F
:1084D800A342B8BF234680F2C88006EE103AB8EE31
:1084E800C66ABCF1000F00F00382072A81ED066A14
:1084F8003BF406AE90ED1C6A9DED194A65EE865A6E
:10850800E7EE045AE6EEA57ABEF1000F40F0B1801E
:10851800FDEEE77A17EE903A9C4240F3B18007EE01
:10852800907AF8EEE77ABCF1000F7FF460ACECE5E6
:10853800574F07F18003FDF77BBE9FED568AFFF783
:1085480058B99FED540A9EE49FED528AFFF779B916
:108558000699B3F90670098B8F42BCBF5242ADF839
:108568004C20FEF7B1BD802016F07CFE08B109F062
:108578000FFC13F04DFFFDF7F8BA05260622042577
:10858800FDF7E2BFFDEEE77A17EE903AA342FFF659
:108598002AAC24E4BDEEC66A16EE103AA342BFF632
:1085A800FDAB2346FFF7FDBBBDEEC66A16EE103ADB
:1085B800A342BFF6CEAB2346FFF7CEBBBDEEC66ADD
:1085C80016EE103AA342BFF69FAB2346FFF79FBBB8
:1085D800BDEEC66A16EE103AA342BFF670AB23464C
:1085E800FFF770BBBDEEC66A16EE103AA342BFF69F
:1085F80041AB2346FFF741BBBDEEC66A16EE103A03
:10860800A342BFF612AB2346FFF712BB14EE903A13
:10861800FFF7E8BA204EFEF789BE069BABF8A860C4
:10862800D880DFF86C90FCF7B9BB0120FEF791B851
:108638002346B342A8BF33466EE62346B342A8BFDB
:10864800334696E62346B342A8BF3346BEE62346E2
:10865800B342A8BF3346E6E614EE103A2EE62346A8
:10866800B342A8BF33460BE72346B342A8BF3346FD
:1086780033E7B4EEE75AF1EE10FA7FF749AF234635
:10868800B342A8BF33461F4649E700BF0C3B002052
:10869800941D00200000000024370020DFF8B0827D
:1086A800D8F800001FF064F9994B1B780022022BC0
:1086B800C8F800207EF404A909F082FBFEF700B98F
:1086C80099F87031002B7BF441A9FBF72CB90C9C6D
:1086D800002C7FF4B2AC0A9CA542B8BFB0EE646A25
:1086E800ABE48C4A8C4B10681B6898478B4BD6EDD3
:1086F800006A93ED007A8A4BD3ED007A894B83EDBB
:10870800020A894B67EE277A234427EEA87AD3ED2D
:10871800007A864B67EE277AF0EE665AE7EEAD5A96
:1087280093ED006AB1EE467AF4EEC75AF1EE10FA0C
:1087380008D4F4EEC65AF1EE10FA8CBFB0EE467AC1
:10874800B0EE657A7A4B1B78012B02D0192B7BF49B
:1087580071A8DFED787AF4EEE7DAF1EE10FACCBF23
:1087680001230023FBF771B80C9C002C7FF4ABAC01
:108778000A9CA542B8BFB0EE646AA4E4FB5C002B77
:108788007DF4F3A9FEF72BB90C9C002C7FF4ECAB1D
:108798000A9CA542B8BFB0EE646AFFF7E5BB0C9B24
:1087A800002B7FF475AE0A9B9D42B8BFB0EE646A99
:1087B8006EE60C9C002C7FF41DAC0A9CA542B8BF49
:1087C800B0EE646A16E40C9C002C7FF459AC0A9C49
:1087D800A542B8BFB0EE646A52E40C9900297FF450
:1087E8009FAB0A998D42B8BFB0EE646AFFF798BB99
:1087F8000C9C002C7FF4DBAB0A9CA542B8BFB0EE02
:10880800646AFFF7D4BB0C9B002B7FF414AE0A9B61
:108818009D42B8BFB0EE646A0DE60C9B002B7FF456
:1088280055AD0A9B9D42B8BFB0EE646A4EE5132B66
:1088380005D1B0EE480A25F0A7FF069B1880B0EED8
:10884800480ADBF808323C489847059B1B78132BED
:10885800B0EE408A7CF4AEA825F096FF069B5880BF
:10886800FCF7A8B8DFED357AB4EEE7EAF1EE10FAD6
:108878004BDCDFED337AB4EEE7EAF1EE10FA44D4DC
:10888800304AD2ED007AB1EE677AF4EEC7DAF1EE4B
:1088980010FA37D4F4EEE7DAF1EE10FA88BFF0EE0A
:1088A80067DA294A86ED00DA12689A42BAF6D6AE35
:1088B800FAF7FEBE0C9B002B7FF463AD0A9B9D422A
:1088C800B8BFB0EE646A5CE50C9B002B7FF42CAD5E
:1088D8000A9B9D42B8BFB0EE646A25E50C9B002B4D
:1088E8007FF47CAD0A9B9D42B8BFB0EE646A75E523
:1088F8000C9B002B7FF4F9AD0A9B9D42B8BFB0EEEC
:10890800646AF2E5F0EE47DACBE7DFED10DAC8E7A4
:10891800103D0020106A0020246A002064690020AD
:1089280000000020D83A0020346A00209C6A002009
:108938006069002000009642845B002000C0F84473
:1089480000C0F8C4986A00207C6A0020000000007B
:108958002C6B00202DE9F04FB0F908500D81EDB2D5
:10896800442D8BB00C46164600F00C8207462FD9D2
:10897800812D00F04A8200F28180542D00F0AE80F3
:1089880040F298816E2D00F0CB81802D40F0B280AE
:10899800B54B1D780B3D15F0FF0512D0B34F0022E3
:1089A8000A2621683B88481C20600E702168FF2B2E
:1089B80002F10102A8BFFF23481CAA4220600B70E5
:1089C800EFDB01252B46284663810BB0BDE8F08F0D
:1089D800052D00F0C5811ED8022D77D040F23181D7
:1089E800032D00F09281042D40F084802A46A0498E
:1089F8002046F9F74FFD00212046F9F77BFD226854
:108A08000021531C0125236028462B4611706381E1
:108A18000BB0BDE8F08F242D56D040F2CA80282D27
:108A280000F0B881382D65D10A68924B0125511C98
:108A38002160157022680521501920601170226884
:108A48000A215019206011702268002150192060F5
:108A580011702268197850192060117022685978AD
:108A680050192060117022689978531923602B4699
:108A78001170284663810BB0BDE8F08FA02D11D08E
:108A880040F2B580B82D00F0BE81FE2D32D17A4D6E
:108A980005F1080635F8021B2046F9F72BFDB5420B
:108AA800F8D18EE7754B08461968F9F70BFD744B3A
:108AB80020461968F9F706FD724B1968204601250A
:108AC800F9F700FD2B467EE76F4BF6E704226F4966
:108AD80020460125F9F7DEFC2B46CAE70B68002182
:108AE8005A1C2260197022680125531923602B46ED
:108AF8001170BEE72146284607F0A2FC00287FF443
:108B080060AF742D00F0F480772D0CD13B687A6843
:108B18009A421BBF5A1C3A60014619785C4A2046A3
:108B28001FF00CFB4DE7F52D00F0C8817A683E6810
:108B3800292DA2EB060300F06C8240F24982392D00
:108B480001F03082532D40F07D82721C3A603178FA
:108B5800032900F2F8844A1E4E4D4F48D2B202EB68
:108B6800420205EB42020170557800293FF429AF13
:108B7800013BDBB2AB4240F0E684821C0023136069
:108B8800536013725DB101353B682844013A0133E3
:108B98003B6013F8011C02F8011F9042F7D13F4BCC
:108BA8001B78002B3FF40DAF012519F0BEF82B46BA
:108BB8005FE7202D9ED10B68394D591C6A782160DA
:108BC8001A7023682A78591C21601A702368AA78B9
:108BD800591C21601A7029892046F9F78BFC2368F3
:108BE8006A79591C21601A702268A97909E7822DCF
:108BF80080D10B682B4A2C4D1178294A581C2060CB
:108C0800197011892046F9F775FC284B22681B88D2
:108C1800FF2B02F10101A8BFFF2321601370A9688F
:108C280081F3100189B22046F9F764FC296801F341
:108C38000F0189B22046F9F75DFC1D4B22681978AF
:108C4800DFE6012D7FF456AF0B680022591C216026
:108C58001A7023685A1C22601D7022682521531C33
:108C680023602B46117004E7565E00206424002020
:108C7800386300202D630020AC5E0020ACF7FF1F96
:108C8800B0F7FF1FB4F7FF1FC4640020E41E0308F9
:108C9800DB7602086014030880540020802C002032
:108CA80084600020C65E0020F05D0020045E002085
:108CB800E84E0020522D7FF41DAF0A68AE4E531CBB
:108CC8000321236006F10C071170334606200121A9
:108CD8002268551C2560117022689F4202F101012B
:108CE8002160107000F0CB809979D8790633EFE7CE
:108CF8003B687A689A421BBF5A1C3A600146197849
:108D08009E4A20461FF01AFA5BE60B685A1C0A6056
:108D18001D700B685A1C0A601D700A68002170E6F5
:108D2800974B0A681B88974DFF2BA8BFFF23511C40
:108D380021601370A96881F3100189B22046F9F700
:108D4800D9FB914B20461988F9F7D4FB296801F320
:108D58000F0189B220460125F9F7CCFB2B4688E69E
:108D68000B228A492046F9F795FB082288492046B4
:108D7800F9F790FB0125072286492046F9F78AFB77
:108D88002B4676E6002A3FF41CAE834B1360012580
:108D98002B466EE60B68DFF83082804E591C0222A3
:108DA80021601A70236806275A1C22601F702368E6
:108DB8000A22591C21601A70236801255A19226059
:108DC8001D70B8F800102046F9F794FBB8F80210A7
:108DD8002046F9F78FFB23685A1922601F70236811
:108DE8005022591921601A702368002259192160EC
:108DF8001A7031882046F9F77DFB71882046F9F70B
:108E080079FB2B4635E6664B57E6664B1E780A3EDD
:108E180016F0FF063FF4D5AD634B644F1E4403F1D3
:108E280001080A2314E0502B00F0A28000252946EF
:108E38002268501C206020461370F9F75BFB294616
:108E48002046F9F757FBB0453FF4BBAD18F8013B96
:108E58000A2BE8D1564A9568116805EB85054FF647
:108E6800FF726D009542A8BF15469142A8BF1146F2
:108E780025EAE57521EAE171ADB289B2D8E74D4B33
:108E880021681A78481C20600A70002A3FF499ADBE
:108E9800013AD2B202EB420206EB42025578002DAB
:108EA8003FF48FAD01351D440133226813F8011FCB
:108EB800501CAB4220601170F7D182E53B687A689C
:108EC8009A4241F07F803C4BFF221A704FF0000914
:108ED8003A4D1BF017FB49462022394885F8009087
:108EE80026F00FFC8DF804909DF80430072B01F252
:108EF800CE80DFF8D880324F4A469DF8043003EB25
:108F0800430308EBC3035B7CE3B19DF8043003EB38
:108F1800430308EBC30320215B699BB19DF8043030
:108F280003EB430308EBC303586947F8220010F02A
:108F380013FE2B7857F8230010F056FE2A780132DA
:108F4800D2B22A709DF804300133DBB28DF80430B8
:108F58009DF80430072BD0D92368591C21601A705A
:108F6800002E3FF42EAD174B336001252B4680E5CC
:108F7800BD68396871E700BF60140308D577020837
:108F8800045E0020F05D0020E44E0020EC1E030883
:108F9800F81E0308041F03081D04010854240020B8
:108FA800D0380020565E0020C8FA02085824002055
:108FB8002024002080540020C81F0020C367002000
:108FC800846700208D9C0208DC3C0020243F0020A0
:108FD800212D37D13346721C3A60184D13F8022BF5
:108FE8006A703B6073782B70F31C3B60B378AB708E
:108FF8003846F9F73DFA3B682881591C1A4639600A
:1090080012F8021B69713A605B78AB7101252B4637
:109018002FE5731C3B6033780A2B00F0FB87502B3D
:1090280040F028873846F9F723FA054E308038464D
:10903800F9F71EFA012570802B461AE58460002096
:10904800542400200B3DEF2D00F27D8201A151F840
:1090580025F000BF479C00084F9500084F95000871
:109068004F9500084F9500084F9500084F95000848
:109078004F9500084F9500084F9500084F95000838
:109088004F9500084F9500084F9500084F95000828
:109098004F9500084F9500084F9500084F95000818
:1090A8004F9500084F9500084F9500084F95000808
:1090B8004F950008F19B00084F9500083D9D00085A
:1090C8004F9500081B9D00084F9500084F95000814
:1090D8004F950008F39C00084F9500087D9C0008F8
:1090E8004F950008BF9B00084F950008999B000802
:1090F8004F950008879B00084F950008339B000890
:109108004F950008479F00084F9500084F950008A5
:109118004F9500084F950008CB8900084F95000827
:109128001B9F00084F9500084F950008939F000863
:109138004F950008339E00084F9500084F9500088A
:109148004F9500084F9500084F9500084F95000867
:109158004F9500084F950008DB9E00084F950008C2
:109168008D9E00084F9500084F950008F59D000852
:109178004F9500084F9500084F9500084F95000837
:109188004F9500084F9500084F950008579D000817
:109198004F950008B19A00084F950008C19900083A
:1091A8004F9500081F9900084F950008F798000888
:1091B800D9980008BD9800084F9500084F950008F9
:1091C8004F9500084F9500084F9500084F950008E7
:1091D8004F9500084F9500084F9500084F950008D7
:1091E8004F9500084F9500084F9500084F950008C7
:1091F8004F9500084F9500084F9500084F950008B7
:109208004F9500084F9500084F9500084F950008A6
:109218004F9500084F9500084F9500084F95000896
:109228004F9500084F9500084F9500084F95000886
:109238004F9500084F9500084F9500084F95000876
:109248004F9500084F9500084F9500084F95000866
:109258004F9500084F9500084F9500084F95000856
:109268004F9500084F9500084F9500084F95000846
:109278004F9500084F9500084F9500084F95000836
:109288004F9500084F9500084F9500084F95000826
:109298004F9500084F9500084F9500084F95000816
:1092A8004F9500084F9500084F9500084F95000806
:1092B8004F9500084F9500084F9500084F950008F6
:1092C8004F9500084F9500084F9500084F950008E6
:1092D8004F9500084F9500084F9500084F950008D6
:1092E8004F9500084F9500084F9500084F950008C6
:1092F8004F9500084F9500084F9500084F950008B6
:109308004F950008939800084F9500087D9800082D
:109318001D9800084F9500084F9500084F950008C4
:109328004F9500084F9500084F9500084F95000885
:109338004F9500084F9500084F9500084F95000875
:109348004F9500084F950008C19700084F950008F1
:10935800899700084F950008ED9600086398000863
:10936800479800084F950008819500084F95000818
:10937800599500084F950008199600084F95000860
:10938800EB9500084F9500084F950008C99500080F
:109398009B9500089B960008739600083195000875
:1093A8000F9500084F9500084F9500084F95000845
:1093B8004F9500084F9500084F9500084F950008F5
:1093C8004F9500084F9500084F9500084F950008E5
:1093D8004F9500084F9500084F9500084F950008D5
:1093E8004F950008F59400084F9500084F95000820
:1093F8009D9400084F9500084F9500084F95000868
:10940800379400084F9500084F9500084F950008BD
:109418001D940008A44B1B78DB0700F194800125FC
:1094280001F0F0F901F096FA2B46FFF722BB384617
:10943800F9F71EF83B68ADF804001A46591C396064
:1094480012F8021B3A608DF806105A788DF807203A
:10945800DA1C3A609A788DF808201A1D3A60DA7892
:109468008DF809205A1D3A601B798DF80A3001A839
:109478000023ADF80C30F8F753FF8C4A8C4B126878
:10948800801A4FF0010561F10001C3E904012B4680
:10949800FFF7EFBA731C3B6033780F2B53D8B21C1D
:1094A8003A60C3EBC303834A7178D154F11C396025
:1094B8001344B2785A70321D3A60F2789A70721D6D
:1094C8003A603279DA70B21D3A6072791A71F21D17
:1094D8003A60B2795A7106F108023A60F2799A71E3
:1094E800012521F09BFC2B46FFF7C3BA3846F8F755
:1094F800BFFF714EF0813846F8F7BAFF0125B081F9
:109508002B46FFF7B6BA3846F8F7B2FF6B4E3082F3
:109518003846F8F7ADFF70823846F8F7A9FF0125FD
:10952800B0822B46FFF7A5BA3346721C3A6013F88F
:10953800020B3B60F31C71783B60B27818F026F997
:1095480000287FF43EAA4FF0FF352B46FFF791BA6B
:10955800731C3B603078060600F19C85524B1B78E3
:10956800DD073FF52EAA032828BF0020012501F0BA
:109578002DF92B46FFF77DBA4B4B1B78D8073FF5E3
:1095880020AA012501F090FD01F0E4F92B46FFF730
:1095980070BA3246731C3B60494B12F8021B1970B3
:1095A8003A6072785A70F21C3A60B2789A7038460B
:1095B800F8F75EFF434B0125D8802B46FFF759BAD1
:1095C8003846F8F755FF3F4E30803846F8F750FFD9
:1095D80070803846F8F74CFF0125B0802B46FFF71E
:1095E80048BADFF8F88098F80030002B3FF4E9A972
:1095F800354E00253846F8F73BFF13F007FC98F87E
:109608000030A6EC010A01359D42F3DBFFF7D9B91A
:109618000D2B98D1731C3B603578072D93D8DFF854
:10962800C08038460C26F8F723FF06FB05F608EB42
:109638000605A8803846F8F71BFFE8803846F8F793
:1096480017FF3B6828811A46591C396012F8021B1B
:10965800A9723A605B78EB723846F8F7F1FE01259B
:1096680048F806002B46FFF704BA3346721C3A60E6
:10967800164A13F8021B11703B600F4A73789370F7
:10968800F31C3B60124BB2789A7001252B46FFF70A
:10969800F0B9104B104918684E22012524F034FF08
:1096A8002B46FFF7E6B900BF85620020946F0020C3
:1096B800C81F0020E4370020EC3C0020E43F0020D5
:1096C800E43C0020743E0020F8390020F05B0020C4
:1096D800FC3C0020EC60002048110308565E002086
:1096E80024370020092B7FF72EAFDFF8B4833346E9
:1096F800721CD8F800503A6013F8022B2A703B60AD
:109708007378AB70F31C3B60B378642BA8BF6423F9
:10971800321D6B713A60F378642BA8BF6423721D05
:10972800AB713A603379EB71B31D3B607379642B8D
:10973800A8BF6423F21D2B723A60B379EB7006F16F
:1097480008033B60F3792B713846F8F791FE7A6885
:109758003B686881D11A00290CDD591CD8F8000033
:109768003960521A002A1978417203DD9A1C3A604E
:109778005B784370012514F037F92B46FFF779B968
:10978800B84B1868F31C02462136991E396013F845
:10979800031C1170591E396013F8021C51703B608C
:1097A80013F8011C917003339E4202F10302ECD1BD
:1097B80021F0A8FDFFF705B9C3F34705122D3FF6C1
:1097C800C2AEBDB10AAB0DF1020803EB450946462E
:1097D800A9F126093846F8F74BFE26F8020F4E4540
:1097E800F8D1A14B38F8022F23F8022FB045F9D150
:1097F800112D09D89D4A6B00023B134400212232E7
:1098080023F8021F9A42FBD1994A01231D4613707F
:10981800FFF72FB9731C97493B600A783378002A01
:1098280040F06B8404220A70934A9B00138002F074
:109838005FF9924B012598612B46FFF71AB9904BB7
:109848001B78DA073FF5BDA88E4A1378012543F047
:10985800040313702B46FFF70CB9894B1B78D90703
:109868003FF5AFA8884B4FF4C87201251A802B46E4
:10987800FFF7FFB8854E002338463360F8F7E0FD60
:10988800012530602B46FFF7F4B83346721C3A6066
:1098980013F8025B3B60F31C70783B60B178002DD5
:1098A80000F05D84012D7FF48CA81BF0D3FC2B46BF
:1098B800FFF7DFB8731C3B603378002B00F014848B
:1098C8004FF40040012507F0B7FD2B46FFF7D1B84C
:1098D8006B4B1B7813F001017FF435AE731C3B60B2
:1098E800307801251BF0FAFB2B46FFF7C2B8334648
:1098F800721C3A60664A13F8021BD1703B60654AD5
:1099080073785371F31C3B60634BB278DA700125AE
:109918002B46FFF7AEB83846F8F7AAFD3846F8F7F1
:10992800A7FD3846F8F7A4FD3846F8F7ADFD3B68C3
:109938004C4D1946581C2A68386011F8020B82F8F9
:109948002C003960597882F83610D91C39609B7818
:1099580082F837303846F8F797FD3846F8F794FD1F
:109968003846F8F791FD38462E68F8F781FD70877C
:1099780038462E68F8F77CFD3B687A683087D11A3C
:1099880001290ADD591C2A6839601B7882F82E30B3
:109998003846F8F779FD3B687A68D31A032B09DD56
:1099A80038462E68F8F764FD708638462E68F8F752
:1099B8005FFDB0862868FBE6731C3B60294DDFF825
:1099C800E480337888F8053038462E68F8F750FD7B
:1099D800308438462E68F8F74BFD7A683B68F08388
:1099E800D11A072915DD3846F8F742FDA8F80A000C
:1099F8003846F8F73DFDA8F80C0038462E68F8F709
:109A080037FD708438462E68F8F732FD3B687A686F
:109A1800B084D11A03290BDD3846F8F729FDA8F8D8
:109A28000E003846F8F724FD3B687A68A8F810005D
:109A3800D21A002A05DD591C2A6839601B7882F879
:109A4800263000F0E9FE18F0B3FB144B1B68002B1E
:109A580000F07A832868012521F074FA2B46FFF775
:109A680008B800BFEC600020C22E0020C42E0020E1
:109A7800E82E0020F6320020E44E0020C81F002007
:109A880085620020443B0020AE3E0020D0380020F4
:109A9800EC3C00206C540020FC3C0020143D0020CD
:109AA800F0600020F05B00203346721C3A60DFF85B
:109AB800388313F8022B88F802203B60BD4A73787C
:109AC8001370F31C3B60BC4DB3782B71331D3B60A6
:109AD800F378092BA8BF09233846AB70F8F7C8FC00
:109AE8003B687A682880D11A012905DD3846F8F7DD
:109AF800BFFC3B687A68E8819A4207D05A1C3A60F2
:109B08001B78003318BF012388F8073000F084FE63
:109B18003B687A689A423EF454AF5A1C3A601B7804
:109B2800EB7001252B46FEF7A4BF731C3B6033780E
:109B38000E2B3FF608ADB21C3A60707803283FF64A
:109B480002AD9E49062202FB03F28B18F51C5871E0
:109B58003D60B0788854321D3A60F2785A70721DB0
:109B68003A6032799A70B21D3A607279DA70F21DF1
:109B78003A60B2791A7101252B46FEF77ABF731C39
:109B88003B608F4B32785A7501252B46FEF771BF23
:109B9800721C3A6035781F2D3FF6D5AC052B7FF443
:109BA800D2AC3846F8F74CFC864B43F8250015F044
:109BB80017FFFEF706BF834D05F140063846F8F754
:109BC80057FC3B68A5F88000591C1A46396012F802
:109BD800021B85F882103A605B7885F8833004357B
:109BE800B542EBD1FEF7EDBE731C3B603578132D03
:109BF8003FF6A9ACB31C3B6070781EF0D9FA002878
:109C08003FF4A1AC704B027803F82520F21C3A60AF
:109C180003EB8503B2785A70321D3A60F2789A7075
:109C2800721D3A603279DA70002013F01DFE674B1E
:109C380080F00100012518702B46FEF71ABF644911
:109C4800102B4FF0000228BF10230A604A608A6078
:109C5800CA600A74002B3EF4B4AE3A680139134462
:109C680001323A6012F8010C01F8010F9342F7D162
:109C7800FEF7A7BE731C524D3B6033782B723846F3
:109C8800F8F7F6FBA8833846F8F7F2FB288338463E
:109C9800F8F7EEFB3A686883531C3B601278EA7465
:109CA8007A68D31A032B00F300823B68D11A05297E
:109CB8000EDD5A1C3A601B78EB723846F8F7C0FB89
:109CC8003B68E8605A1C3A601B782B743B687A68DA
:109CD800D21A002A7EF775AE5A1C3A601B7885F8AE
:109CE800213001252B46FEF7C4BE731C3B60394961
:109CF80030780870D21A002A7EF763AEB31C3B6036
:109D08007378003318BF012301254B702B46FEF7EB
:109D1800B0BE3846F8F7ACFB2F4E30603846F8F73F
:109D2800A7FB70603846F8F7A3FB0125B0602B4607
:109D3800FEF79FBE294E002333603846F8F780FBB4
:109D480033680125034333602B46FEF792BE244B4C
:109D58001B68002B3EF435AE16F0C0F8FF283EF421
:109D680030AE3846F8F784FB3F2840F20B821D4E90
:109D7800002535703B687A68B080D21A012A7EF7D0
:109D880020AE1A46591C396012F8021BB1700AA895
:109D98003A6000225D7800F8242D16F071F89DF8DD
:109DA8000430AB423EF40DAE284616F08DF8FEF7AF
:109DB80008BE00BFE03C0020E43F0020DC38002063
:109DC800D4660020144D0020503000201C010020D3
:109DD800C83C00202C3D0020482C0020C4640020F2
:109DE800886200208C620020F05B0020C54B1B7845
:109DF800012B3EF6E6AD731C31463B60DFF840832D
:109E080011F8023B88F80230F31CD21A3960012A93
:109E180070783B6040F3A9813846F8F729FB0125A3
:109E2800A8F800002B46FEF724BE731C3B60B64B17
:109E38003278DFF810831A700023C8F800303846EB
:109E4800F8F7FEFA3A68D8F80030B049B04D034345
:109E5800501CC8F80030386013780B723846F8F791
:109E680007FB28603846F8F703FB68603846F8F7C0
:109E7800FFFAA8603846F8F7FBFA3846F8F7F8FA18
:109E8800FEF79FBD731C3B6096F80080B8F1110F78
:109E98003FF659ABB31C3B609E4D737805F81830FC
:109EA8003846F8F7E5FA40F6CA039842A8BF1846BC
:109EB80040F2EE23984205EB4801B8BF1846012549
:109EC800A0F2EE222B46192092FBF0F24A70FEF720
:109ED800D0BD3346721C904D3A6013F8022B2A719C
:109EE8003B6073786B713846F8F7C2FA3B68288094
:109EF8005A1C3A601B78AB713846F8F7B9FA3B68D8
:109F080068805A1C3A601B78EB7101252B46FEF7D6
:109F1800B0BD3346711C3960804913F8020B887054
:109F28003B607078487093423EF44BADF31C3B6045
:109F38007B4BB2781A7201252B46FEF79ABD072291
:109F4800B3FBF2F2C2EBC2015B1A7FF4FCAAD2B2F5
:109F580002F1FF395FFA89F9002A3EF432ADDFF8E1
:109F6800C4A109F101099846731C3B6096F90010D9
:109F78006C4B002593F902208A4203F1080360D054
:109F88000135042DF6D1FFF7DEBA674B06F108025A
:109F980001363E6016F8011C03F8011FB242F7D1E2
:109FA800FEF70FBD731C3B6033780A2B38D0384658
:109FB800F8F76AFA3846F8F767FA3846F8F764FAAD
:109FC800FEF7FFBC5A1C19463A60554811F8022B97
:109FD800027039605B784370042A06D9FF2A3EF480
:109FE80075AF22680021FEF70CBD504909789942E7
:109FF80003D8022AF5D1FF2BF3D1236801255A197A
:10A0080022601D70002E3EF4DCAC494B33602B46B9
:10A01800FEF72FBD3846F8F72BFA464EFFF706B87D
:10A02800B31C3B60444B72781A70F21C3A60B278E9
:10A038005A70321D3A60F2789A7001252B46FEF765
:10A0480018BD0AEBC50B38468BF80210F8F710FA62
:10A058003B682AF835001A46591C396012F8021B69
:10A068008BF803103A605A788BF80420DA1C3A60AF
:10A078009A788BF806201E1D3E6008F10108DB78EF
:10A088008BF80530C1457FF46FAFFEF79ABC4A469E
:10A09800FEF762BF00F07F00032828BF00200125DB
:10A0A8001BF0F4F82B46FEF7E4BC3846F8F7E0F965
:10A0B800A8843846F8F7DCF93B687A68E884D11A4E
:10A0C80003297FF7F3AD1A46591C396012F8021BB1
:10A0D800A9773A605B7885F820303846F8F7C8F9F0
:10A0E8003B687A686884E1E5144A1368012523F41B
:10A0F800004313602B46FEF7BCBC042A7EF461AC17
:10A10800FFF792BB906400202C3D0020D46600200D
:10A11800482C00205C3100208C3E00200C3D0020A3
:10A12800C81F002000670020D3660020565E00206C
:10A1380035040108DC3C00202D630020E460002089
:10A1480092640020C464002015481649164A174B2B
:10A15800036001250B6013602B46FEF78ABC0125BE
:10A1680021F0B4F82B46FEF784BC114BB1781A885D
:10A17800012512FB00F22B4692FBF1F2A8F8002011
:10A18800FEF777BCC50800F0070301350133EDB2CF
:10A19800084E28461946737018F0E6FFE9E500BF37
:10A1A80068690020BC690020246A0020F5030008C3
:10A1B800523B00208C62002038B50B4C23688BB1D1
:10A1C8005A68821A002A054604DA0CE05A68AA1A64
:10A1D800002A07DB9A68226018461A6890472368A5
:10A1E800002BF3D138BD38BDEC2F00200B4B0022DB
:10A1F80010B4027203F1DC04012102E0072A09DC31
:10A208009979890702D51979815401329C4203F161
:10A218001403F3D15DF8044B704700BF8C16030894
:10A228001F230370704700BF30B401230225142494
:10A2380015212222057244704171C27003700371A6
:10A24800837030BC704700BF2DE9F0410B78057B67
:10A25800DB43DFB200F1130200F11D0302F8015FD6
:10A268009342FBD1DFF890E000F12701002203F8C8
:10A27800012F9942FBD114210524002647FA04F343
:10A2880003F00103002B1E4414BF4FF019084FF0D0
:10A298000A0814F0010FF6B214BFAC464FF0000CD8
:10A2A8000023CA1810FA82F20133434582F814C019
:10A2B800F7D15A1E92B20132013C8B18621C9BB234
:10A2C80001D01946DAE716F0010F14BF19240A2441
:10A2D8000022991810FA81F10132A2420D75F8D1C5
:10A2E80013449BB25A1C0344002192B21975AEF86C
:10A2F80000200261BDE8F081F01F00202DE9F04F39
:10A30800DFF890A0BAF802300B3383B01FFA83F954
:10A3180001F1060B4FF001084FF0000C002711F86F
:10A3280001EB3E464C460122A4F10B039BB201917E
:10A3380005E001339BB2017B29759C4208D0C51802
:10A34800002AF6D1C51801339BB29C422A75F6D172
:10A3580003190136092F019983F814C0F6B20CD0FD
:10A36800092E15D008FA07F313EA0E0F14BF0122BD
:10A3780000220C34A4B20137D6E709F1780959450F
:10A388001FFA89F9CAD1AAF802C003B0BDE8F08F54
:10A398000022EEE7F01F00202DE9F047DFF85C808F
:10A3A800B8F8043004331FFA83FC01F109094FF0AF
:10A3B800010E11F8017B64460026231F0EFA06F2EF
:10A3C8009BB23A40C2B1B0F80CA0C51801339BB299
:10A3D8009C4285F814A0F5D101360434082EA4B2A5
:10A3E800EBD10CF1200C49451FFA8CFCE1D100237C
:10A3F800A8F80430BDE8F0879246E6E7F01F002091
:10A4080010B50168047B0A680223A3401A420AD0E7
:10A41800054A406800241470026822F00102120400
:10A42800120C02604B6010BD1C6600202DE9F0473D
:10A438008C4B1B78DB07074644D58B4B8B4D1C7820
:10A448008B4E012C59D01CD3022C07D189498A4A3A
:10A4580009881288914201D901241C70EB7AE3B172
:10A468002B89D3B1854B1B78BBB107F0CBF90028FA
:10A4780000F09B802B7B83422CBF0121002131708F
:10A488000CE07C497E4A098810886A7B801A8842D9
:10A49800E2DAEB7A0024002BE2D131782A79632AB8
:10A4A80006D8022C774E00F0BA803378002B5DD1A5
:10A4B800754AAB7A8C4238BF0C461470002B4CD1CD
:10A4C800BDE8F0876B4B694D19885B88E878CB1A33
:10A4D80083EAE3728142A2EBE3721DD32B788B42AD
:10A4E8001AD3614B1C78E01E012861D967490978A5
:10A4F80002294FD0012C5E4EA5D15F4A5D491288D2
:10A50800687B0988121A914239DD5D4A12888A42AD
:10A51800A4D200241C70A1E7B1EB400FE1DC524B40
:10A528001C78E11E012940F29480022ADEDC57499A
:10A538004F4E0878DFF84481DFF844C1DFF838E18E
:10A5480000210324022834701C7088F80010ACF82D
:10A558000010AEF8001081D11FE0012C71D0022C40
:10A568000BD10720BDE8F0471DF054BC7068381ABD
:10A57800474B984258DD72709AE7BDE8F08702248D
:10A588001C706BE7022AD2DD4049097802294FF096
:10A59800040464D13949364E09783E48022ACCBFB2
:10A5A80000220122C28081804BE70221317075E7C9
:10A5B800022A9BDC95F800C091FBFCFC0CF1010C15
:10A5C800BCF1080FDFF8B4A0304EA87895F801E088
:10A5D80096F800802A4CDFF8A090254EA8BF4FF0CF
:10A5E800080C8AF800C01FFA8CFA10FB0AF01EFB50
:10A5F8000AFE80B2DFF88CA02080A9F800E00024D1
:10A608004FF0640EB8F1020F34701C70CAF80440A1
:10A618008AF801E07FF439AF0FFA8CF1BDE73078A2
:10A62800A0B9012377603370C2F164021A4B00FBB2
:10A6380002F083FB0023C017A0EBA35064307070B6
:10A6480036E70820BDE8F0471DF0E4BB7368F81A48
:10A658008EE7032C96D10D49097802299AD0044E29
:10A66800FCE600BF856200208C2400208460002066
:10A678009C240020045E002090240020C65E002058
:10A688008E24002094240020E84E0020A85E00209C
:10A698007F969800AC5E00206BCA5F6B2DE9F0478F
:10A6A8000569C3681D4028D00F4606464FF000488C
:10A6B8004FF00009B5FA85F328FA03F2D2431B3BA1
:10A6C80032611540042B16D8DFE803F0312921192F
:10A6D80003007B6A002B32D003F1FF3A1FFA8AFA93
:10A6E800C7F824903C6A34B12368204651469847FD
:10A6F8006468002CF8D1002DDCD1BDE8F0873868FB
:10A70800716B036889B29847002DD3D1F5E7786853
:10A71800B16B036889B29847002DCBD1EDE7B868D3
:10A72800F16B036889B29847002DC3D1E5E7F86853
:10A73800316C036889B29847002DBBD1DDE7F36A15
:10A748001FFA83FACEE700BF1C4C08B5012102208E
:10A758000FF05AFA237803F00502052A2AD003F0ED
:10A768000903092B08D0002101200FF04DFA002120
:10A7780008460FF049FAFEE7114A124B11681A68A9
:10A788000B68114C4FF6FE7003400B60138820686D
:10A7980023F001031B041B0C138018B12A22002389
:10A7A8008271C37102224E210FF07EF920680FF0EA
:10A7B80015FAD8E712F03EFC2378D0E7202C0020C9
:10A7C8007C2C0020742C0020782C0020022828BF24
:10A7D800022010B4084C094B207000EB8002C0EB3B
:10A7E800C20207495DF8044B013003EB4203C0B2D3
:10A7F8000B601DF0F5BB00BF326300204E630020E4
:10A80800EC60002008B50AF07FFBF7F7AFFABDE867
:10A8180008400AF061BB00BF38B5434B5A89998993
:10A82800914224BF00225A81198ADA89914224BFB1
:10A838000022DA81DA788AB3072A2FD03B493C4DC7
:10A8480091F85300012400210A282C709C70D971BA
:10A858003DD00C2865D0DFED377A8ABB364C9FEDAA
:10A86800370AA278002918BFF0EE407A062A04D8E1
:10A87800334901EB820191ED000A217959B3013A7C
:10A88800032A4DD8F7EE007A87EE800A23F07CFF82
:10A898002388984228BF1846208038BDD97921B12D
:10A8A80098780428B8BF04209870204890F853007E
:10A8B8000A280CD00C28CED1DFED227A002ACDD080
:10A8C800072ACBD00A282CD1DFED1F7AC6E70A2049
:10A8D800DFED1E7AC1E79B78154A07EE103A11782A
:10A8E800B8EEC77A27EE277A07EE901AF8EEE77ADD
:10A8F80067EE877AB4EEE70AF1EE10FA10DDC0EEE3
:10A90800077AFDEEE77A17EE903A102BA8BF1023CE
:10A91800012BB8BF0123DBB28B4238BF0B46137043
:10A9280038BDDFED0B7A99E7F05B002078590020FD
:10A93800E03C00206F120339E43F00206F12033817
:10A94800CCFA02080AD7A3390F506E3A5304E938F3
:10A958006F12833A2DE9F047AC4FAD4E0AF0D4FAA6
:10A96800BE421ED2DFF82483DFF8249344462588AC
:10A9780062197DB14A450DD2052D0BD933886188FE
:10A98800C3F30B03994200F0E58014462588621949
:10A99800002DEFD17168304614360FF040FBBE42EF
:10A9A800E4D39C4A1378A3F1170102290FD99A49D5
:10A9B80011F83300002840F0F980D80001444978A4
:10A9C80029B1964911F83330002B00F01781944BC8
:10A9D8005A78022A40F2E480002292495A701A7882
:10A9E8009148022A016000F2D78002EB82018F4B66
:10A9F800C2EBC10203EB4203998C5A8C8C4C9142F6
:10AA0800236001D300225A848A4B9A78042A00F0E2
:10AA1800EC8032B91A88B2F5F07F84BF4FF4F07237
:10AA28001A80854DFFF7F8FE2B68844A1A40002AE1
:10AA380000F0E780D80700F1D380590400F1CB80FB
:10AA48001A0700F1C3809B0400F1B9801EF082FB55
:10AA580010B97B481CF09AFE40200FF017FB8020AD
:10AA68000FF014FB4FF400700FF010FB4FF40030A0
:10AA78000FF00CFB4FF480200FF008FB4FF0007034
:10AA88000FF004FB4FF080600FF000FB4FF0006008
:10AA98000FF0FCFA12F0A8FF00213022694824F0D8
:10AAA80030FE206820F05EFD674B276803F15001F7
:10AAB80002E0043399426DD01A78002AF9D19C78C3
:10AAC800D8788442F5D26149614B0D796149624871
:10AAD8000A70624E624C8460C822642111FB052111
:10AAE800002259609A60DA601A615A619A61DA61E3
:10AAF80083F8202083F8212037600CF0C9FD594BDA
:10AB08009FED595A1B88594A9FED596A50795949FE
:10AB180006EE903AF8EEE66A1388C5EE265A07EE76
:10AB2800103A53881279C1ED005A07EE903AB8EE00
:10AB3800C77A514BF8EEE77A18725A7227EE067AFE
:10AB480067EE867ABDE8F04783ED017AC3ED007AB7
:10AB58000AF0C2B963799B077FF417AF716894F85C
:10AB680004A030460FF05BFA3388BAEB133F04D0E9
:10AB78001436BE42FFF4FAAE13E773887068AA1F52
:10AB8800C3F30B039A4204F10601A8BF1A4623F047
:10AB9800BBFCEDE7012296E700221A70234B2BE756
:10ABA800204902EB420201EB820118E7D8000C1899
:10ABB8006468002C7FF402AF17241470FEE62F4857
:10ABC8000FF064FA40200FF061FA3FE72C480FF0CD
:10ABD8005DFA2B6837E72B480FF058FA2B682FE7F8
:10ABE80029480FF053FA2B6827E79A8AB2F57A7F3B
:10ABF800BFF417AF4FF47A729A8212E718231370D2
:10AC0800E5E643F001032B6014E700BF305003086A
:10AC1800F84B03082C3D0020101A0308AC17030852
:10AC2800326300205A640020F06000204E63002048
:10AC3800EC600020E43F0020C464002009600002AA
:10AC48000067002010210020503000208C3E00209A
:10AC5800EC4E00201C010020F01F002044210020A1
:10AC6800F23C0020581F0020C0C9FB48CC1F002020
:10AC780017B7D1385C1F0020CC3D002009400002E6
:10AC880001600002092000020860000202F00308C7
:10AC98000000040808B50AF037F9F7F767F80AF072
:10ACA8001BF9FFF757FE0120BDE808401DF098B9D1
:10ACB8002DE9F047B24C636820469847002800F019
:10ACC800C180B04B1B780122042B84F83C2000F093
:10ACD800BB80B4F91610B4F91820B4F91A302163FE
:10ACE8006263A363A84B1B88002B69D0A74DD4EDE2
:10ACF8000C7AD5ED004A95ED050A95ED015A95EDCA
:10AD0800067AD5ED035A95ED026AF8EEE76AD5EDB5
:10AD1800047AA4EEA60AA5EE267A67EEC07AA5EE16
:10AD2800C07AE6EE267A85ED057AC5ED067A23F037
:10AD38002BFDD4ED0D6AD5ED094A95ED0E0A95ED7A
:10AD48000A5A95ED0F7AD5ED0D7AD5ED0C5A95ED99
:10AD58000B6A2063F8EEE66AA4EEA60AA5EE267A48
:10AD680067EEC07AA5EEC07AE6EE267A85ED0E7A11
:10AD7800C5ED0F7A23F008FDD4ED0E6AD5ED124A21
:10AD880095ED170A95ED135A95ED187AD5ED167AC3
:10AD9800D5ED155A95ED146A6063F8EEE66AA6EEED
:10ADA800A40AA6EE857A67EEC07AA0EE657AE6EE8A
:10ADB800867A85ED177AC5ED187A23F0E5FCA0634D
:10ADC800734FA17F73480CF0E5FB3B88002B7DD1C6
:10ADD800714EB568714B1B685B0743D4B5F90070B9
:10ADE800216B636BA06B6E4A6E4E92ED026AD2EDD8
:10ADF800006AD2ED015AC91B2163B5F90270DB1B49
:10AE08006363B5F904703568C01B07EE900AB8EEA5
:10AE1800E75A07EE901AB8EEE77A07EE903AF8EE9E
:10AE2800E77A36EE056A36EE877A77EEA57A013547
:10AE3800A06382ED026A82ED007AC2ED017A356084
:10AE4800BDE8F087BDE8F087574BB4F91600B4F9B0
:10AE58001810B4F91A2018802063598061639A8009
:10AE6800A2633FE7514F3B88322B79D0002B5BD14F
:10AE78004F480378002BB1D0DFF83CE1716AB26A21
:10AE88008EFB01730027C9170770C1EB23118EFBD6
:10AE98000203D217C2EB2312F36A29806A80A08AC0
:10AEA80044498EFB03E2DB17C3EB22131B1AAB806A
:10AEB800CF600AF029F8F6F759FF0AF00DF8FFF706
:10AEC80049FD01201DF08CF8B56887E7324E226BEA
:10AED800B568B3F5C87F4FF0000323632B8039882A
:10AEE80018BFF068B7F8008008BF0020B1F5C87F28
:10AEF80018BF3369616B02440B440020B8F5C87F62
:10AF08006063F2603361688035D0D4F838E07169E5
:10AF1800A0637144B8F1010FA88071614ED008F1A7
:10AF2800FF38A7F8008055E7716A226B002020637C
:10AF380028803B880A44322B616B726260636880A8
:10AF480068D0B26AD4F838E0A0631144F26AB162FA
:10AF58007244012BA880F26262D0013B3B8087E7F4
:10AF6800144B2988D8686A88AB8831833062728329
:10AF7800B3830021D9E7A36B7361A063A880CEE7F0
:10AF8800A0600020A85E0020A0360020A436002083
:10AF9800AE3E0020D0600020F01F0020145C00208E
:10AFA800C03D0020BC3D0020AC5E00200C210020EC
:10AFB80009210020EC3C00201F85EB51DFF894C0EC
:10AFC800DFF88CE0C8328CFB02A9C833D217C2EB79
:10AFD800E9128CFB03A9DB17C3EBE913C8316B80BB
:10AFE8002A808CFB013CA28ACB17C3EBEC139B1A7B
:10AFF800AB80CEF80C0009F087FFF6F7B7FE09F032
:10B008006BFFFFF7A7FC40461CF0EAFFB7F800808B
:10B01800B56884E7A26BB162A063F262A8809CE77E
:10B0280009490A4A08700B2013701CF0F3FEB56832
:10B03800338B718B064A2B806980B08B316AA8806C
:10B048003B88D16089E700BF0E210020082100203D
:10B05800EC3C00201F85EB5138B50C4C0C4DAC4234
:10B0680006D26168204614340EF0D9FFAC42F8D3FA
:10B07800084A094B094C1460002209491A705A7091
:10B0880008480860BDE8384014F0AABCF84B03082B
:10B0980030500308EC600020326300204E6300202B
:10B0A800F06000205A64002008B5FFF7D5FF09F0CA
:10B0B8002BFFF6F75BFEBDE8084009F00DBF054B16
:10B0C80010B51A6B044C2178501C09B91A6310BDCD
:10B0D8000246F8E7F01F00201C660020F0B50C2996
:10B0E8002BD8DFE801F06F2A2A2A4C2A2A2A2B2A91
:10B0F8002A2A0700046AB2F80CE097881668674D98
:10B1080024F480540462036A4468C16923F4005338
:10B1180043EA0E3321F4E641A84243EA073341EA01
:10B12800062100F0B58005F50065A84200F0B08062
:10B1380092684460C16102640362F0BD046A968942
:10B148009588D2F800E0554F24F480740462036AAD
:10B158004468C16923F4007343EA062321F07301AC
:10B16800B84243EA052341EA0E017ED04C4DA8427D
:10B178007BD092684460C161C2630362F0BD046A17
:10B1880096899588D2F800E0444F24F010040462B0
:10B19800036A4468816923F0200321F0807143EA3F
:10B1A800061321F4E641B84243EA051341EA0E21A9
:10B1B80048D03B4DA84245D0926844608161826383
:10B1C8000362F0BD046A9389B2F804E01768334E4D
:10B1D80024F001040462056A4468816943EA0E03A5
:10B1E80021F4803125F002059BB221F07301B042B1
:10B1F80043EA050341EA070114D0294DA84211D0BA
:10B2080005F54065A8420DD005F58065A84209D02E
:10B2180005F58065A84205D0926844608161426363
:10B228000362F0BDD689158A578A23F00803334391
:10B238003D43D68824F4407423F00403ADB233436D
:10B248002C43E9E7D589178AD68823F0800343EA97
:10B25800051324F44064558A23F0400344EA870424
:10B2680043EA061344EA8504A6E7D589178AD688EF
:10B2780023F4006343EA052324F44054558A23F455
:10B28800806344EA071443EA062344EA051470E796
:10B29800158A24F4804444EA851449E7002C0140C7
:10B2A800003401402DE9F04FC822002183B07848CE
:10B2B800784CDFF80492784D784E794FDFF8FC81AE
:10B2C80024F01FFA77487849DFF8F4E1DFF8F4C191
:10B2D80000221359834200F0C180B3F1804F00F07F
:10B2E800BF80AB4200F0C880B34200F0C780BB42C9
:10B2F80000F0C680734500F0C580634500F0C48047
:10B30800434500F0C380DFF8C0A153457ED00AF55D
:10B31800806A534508BF092379D01432F02AD8D15E
:10B328005C4C624D624E604F04F1F00802E0143448
:10B33800A04568D0A379002BF9D023794FEA1319D7
:10B3480009F1FF39B9F1050F03F00F03EFD835F80C
:10B35800190040FA03F2D207E9D54FF0010A0AFAB8
:10B3680003F3013B184022F05BFE16F809305149FF
:10B37800184411EBC002DAD051F83000DFF84CE184
:10B38800217A00F138439B0A1EF8033003F01F0EA0
:10B398005B09022B0AFA0EFA69D0032B62D0012B43
:10B3A80003D17B694AEA03037B6193880093B3FA6C
:10B3B80083F3C3F11F039BB2DA0800EB820203F0A8
:10B3C8000703D2F820E09B004FF00F0C0CFA03FCA7
:10B3D8002EEA0C0EC2F820E0D2F820E001FA03F3BE
:10B3E80043EA0E03136269460023022214348DF8DF
:10B3F80004208DF805308DF806308DF807301AF0E6
:10B408008BF9A04596D103B0BDE8F08F082309EB6E
:10B41800C3034FF0010B93F820A00AF01F034FEA73
:10B428005A1ABAF1020F0BFA03F30BD0BAF1030F51
:10B438000ED0DA457FF471AFD1F814A043EA0A03BD
:10B448004B616AE7D1F818A043EA0A038B6164E705
:10B45800D1F81CA043EA0A03CB615EE70023D6E7D4
:10B468000123D4E7FB694AEA0303FB619DE7BB6953
:10B478004AEA0303BB6198E70223C8E70323C6E748
:10B488000423C4E70523C2E70623C0E70723BEE772
:10B49800306100208C1603080004004000080040BA
:10B4A80000100040002C014000100240EC1203087C
:10B4B800F812030848580020CCFA0208004001405E
:10B4C8000014004000340140004401400013030808
:10B4D80001490248FFF7E2B8D0610020004001406E
:10B4E80001490248FFF7DAB8A8610020003401409A
:10B4F80001490248FFF7D2B8A86100200034014092
:10B5080001490248FFF7CAB88061002000040040E2
:10B5180002494FF08040FFF7C1B800BF58610020D2
:10B5280001490248FFF7BAB830610020002C0140F9
:10B5380001490248FFF7B2B830610020002C0140F1
:10B548002DE9F04104684A4DA30AAB4272D009D8EC
:10B55800B3F5801F6AD04A3DAB425AD14FF0700E06
:10B56800022608E0434DAB4268D00335AB4252D1C6
:10B578004FF0C00E042647794FEA970C002961D096
:10B58800B000634685190227D4F80C809F400CEB65
:10B598004503BFB2384D03F1040C47EA080745F8E4
:10B5A800231045F82C20E760EFF31181502282F335
:10B5B8001288821905EBC202136973B3136204334C
:10B5C800821905EBC202576917B11F60536904332A
:10B5D800821905EBC202976917B11F60936904339A
:10B5E800821905EBC202D76917B11F60D36904330A
:10B5F8000027CAB21F6082F31188304405EBC000EF
:10B60800036A6BB9E3684FF6FE721340E360BDE866
:10B61800F081BDE8F081BDE8F08105EB0E03CFE7CE
:10B62800E36843F00103E360BDE8F0814FF0480EA2
:10B638000126A0E74FF0200E00269CE74FF0980E59
:10B64800032698E7BF08022306FA03F0BB40DB4352
:10B65800E768094D9BB23B4087190CEB470CE36048
:10B668000CF1040345F82C1045F823209CE700BF93
:10B678004B0010004D0010003061002030B5036809
:10B688005C4D18885C4CB4FBF2F20139013AAB42CC
:10B6980094B283B089B282B266D05848834263D0EC
:10B6A800B3F1804F60D0A0F5983083425CD000F5AC
:10B6B8008060834258D0524883425BD000F5806056
:10B6C80083427DD022F4407200F58C3092B28342DE
:10B6D8001A80D9621C850ED0484A93420BD002F5D5
:10B6E8004062934207D002F58062934203D002F58C
:10B6F8008062934201D100221A8601225A611A8877
:10B708003C4992B242F001028B421A8062D0B3F1F6
:10B71800804F61D03B4A934260D002F580629342E9
:10B728005ED002F5006293425CD002F580629342DB
:10B738005AD002F59032934258D002F540629342B3
:10B7480056D002F5806293421ED002F58062934281
:10B7580008BF092219D002A84FF0012340F8043D80
:10B7680019F0A4FF03B030BD254822F070028342CF
:10B7780092B2A3D101201A80D9621C8558611A8817
:10B7880092B202431A80C5E708221F4B03EBC2039B
:10B7980001A893F821408DF80440012300228DF878
:10B7A80005308DF807308DF8062019F07FFF1B2C27
:10B7B800D8D1164B019301A819F078FF03B030BD1A
:10B7C80001201A80D9621C8558611A8892B20243F6
:10B7D8001A809CE70022D8E70122D6E70222D4E7A4
:10B7E8000322D2E70422D0E70522CEE70622CCE7DF
:10B7F8000722CAE7002C014000A24A040034014095
:10B808000010004000040040CCFA020819010001B1
:10B81800204B98422DD0B0F1804F2CD0A3F5943313
:10B8280098422AD003F58063984228D003F5006334
:10B83800984226D003F58063984224D003F59033CC
:10B84800984222D003F54063984220D003F58063E4
:10B85800984207D003F58063984208BF092202D0B6
:10B868000020704708220C4B03EBC20393F820001A
:10B8780070470022F7E70122F5E70222F3E70322E7
:10B88800F1E70422EFE70522EDE70622EBE70722BE
:10B89800E9E700BF002C0140CCFA02082DE9F04F7F
:10B8A800013085B0C3B203930B4602918B4C8C4E8A
:10B8B800002B00F09A8032208A4D8B4FDFF82C92B3
:10B8C80021F0A4FA4FF4FA7A4FF0100C4FF47A7082
:10B8D800D9F80430C3F30803002B40F0DE80EFF3FF
:10B8E8001183002B40F0D9802968A26800BF2B681B
:10B8F8009942F9D1D7F800E000FB0EF39B1AB3FB8D
:10B90800FEF300FB01314FF0010E0191D9F804302C
:10B91800C3F30803002B40F08780EFF31183002B5B
:10B9280040F082802B68A16800BF2A689342F9D151
:10B93800D7F800B000FB0BF2521AB2FBFBF200FB87
:10B948000323019A9B1AB3F57A7FDFD3BAF1010A70
:10B95800BED1039B002B40F0BD804FF47A7ADFF80C
:10B968008C9150464FF0100CD9F80430C3F30803FB
:10B97800002B75D1EFF31183002B71D12968A268D0
:10B9880000BF2B689942F9D1D7F800E000FB0EF30D
:10B998009B1AB3FBFEF300FB01314FF0010E01913E
:10B9A800D9F80430C3F3080313BBEFF31183FBB9D1
:10B9B8002B68A16800BF2A689342F9D1D7F800B074
:10B9C80000FB0BF2521AB2FBFBF200FB0323019AB5
:10B9D8009B1AB3F57A7FE3D3BAF1010AC4D1029B6B
:10B9E800013B0293002B7FF466AF05B0BDE8F08FF2
:10B9F800EFF311888CF31288A1682368DB0344BF36
:10BA0800C6F800E0A1682B6832685FFA88F888F306
:10BA18001188D7F800801A4400FB08F35B1AB3FBBF
:10BA2800F8F300FB0233D2E7EFF311888CF31288A6
:10BA3800A1682368DB0344BFC6F800E0A1682B684F
:10BA480032685FFA88F888F31188D7F800801A44BA
:10BA580000FB08F35B1AB3FBF8F300FB023370E753
:10BA6800EFF311828CF31288D4F808E02368D90325
:10BA780003D501233360D4F808E02B683168D2B2CB
:10BA880082F311883A68194400FB02F3A3EB0E0312
:10BA9800B3FBF2F300FB01317FE7EFF311828CF384
:10BAA8001288D4F808E02368D90303D5012333604A
:10BAB800D4F808E02B683168D2B282F311883A686A
:10BAC800194400FB02F3A3EB0E03B3FBF2F300FBF4
:10BAD800013118E7184621F021F83EE710E000E0B0
:10BAE800906F0020946F0020986F002000ED00E018
:10BAF800204B5B68C3F3080330B4BBB9EFF3118381
:10BB0800A3B91D4B1D4C1868A16800BF1A68904264
:10BB1800F9D11B4B1C684FF47A7202FB04F3591AD3
:10BB2800B1FBF4F130BC02FB00107047EFF3118257
:10BB3800102383F3128811498C680B6813F4803F33
:10BB4800104B02D0012018608C680B49D2B20D68E6
:10BB5800186882F311880A4B19684FF47A722844DE
:10BB680002FB01F31B1B30BCB3FBF1F302FB0030FB
:10BB7800704700BF00ED00E0946F002010E000E087
:10BB8800986F0020906F00202DE9F84F8046FFF74E
:10BB9800AFFF254E2549DFF8A0E0254A254D84460C
:10BBA80010274FF47A740120DEF80430C3F3080339
:10BBB800D3B9EFF31183BBB90B68D2F808A000BF63
:10BBC800D1F800904B45F7D1D6F800B004FB0BF93B
:10BBD800A9EB0A09B9FBFBF904FB0393A3EB0C03DC
:10BBE8004345E1D3BDE8F88FEFF3118A87F3128854
:10BBF800D2F808B01368DB0344BF2860D2F808B055
:10BC08000B68D5F800905FFA8AFA8AF31188D6F89B
:10BC180000A0994404FB0AF3A3EB0B03B3FBFAF36C
:10BC280004FB0933DAE700BF986F0020946F002007
:10BC380010E000E0906F002000ED00E02DE9F04FEB
:10BC4800DFF830C1474A4849484E494D80461027D9
:10BC580018F1FF38C0F08480DCF80430C3F308031F
:10BC6800002B5CD1EFF31183002B58D10B6894683B
:10BC780000BF08688342F9D1D6F800904FF47A7073
:10BC880000FB09FEAEEB040EBEFBF9FE00FB03EE63
:10BC9800DCF80430C3F308034FF47A740120FBB9CD
:10BCA800EFF31183E3B90B68D2F808A000BFD1F80D
:10BCB80000904B45F7D1D6F800B004FB0BF9A9EB7F
:10BCC8000A09B9FBFBF904FB0393A3EB0E03B3F5D5
:10BCD8007A7FBDD2DCF80430C3F30803002BDFD031
:10BCE800EFF3118A87F31288D2F808B01368DB03E0
:10BCF80044BF2860D2F808B00B68D5F800905FFA06
:10BD08008AFA8AF31188D6F800A0994404FB0AF34A
:10BD1800A3EB0B03B3FBFAF304FB0933D5E7EFF30B
:10BD2800118487F31288D2F808901368D80303D5D2
:10BD380001232B60D2F808900B682868E4B284F3DA
:10BD48001188D6F800A04FF47A7400EB030E04FBB8
:10BD58000AF3A3EB0903B3FBFAF304FB0E3E97E7E0
:10BD6800BDE8F08F10E000E0946F0020986F00208D
:10BD7800906F002000ED00E030B4EFF31183102243
:10BD880082F312880649074C0A68074801320025E1
:10BD98000A602560DBB2026883F3118830BC704703
:10BDA800946F0020906F002010E000E00F4B1B887C
:10BDB800014643B90E4B0F4A1B7810680BB981F046
:10BDC80001010DF017BF0C4B5A691AB118B91A685E
:10BDD800106058747047094A18681188084A92FB1D
:10BDE800F1F2012102605974704700BF6C6F0020A6
:10BDF8006E6F0020706F0020746F00208C6F002021
:10BE080020A107001D4B70B59C68236D626BDD692E
:10BE1800C2B1A36B2BB12B0702D5236D08221A627E
:10BE280070BD2A06F7D5A26A616A8A4220D0511CE1
:10BE3800A069A162825C2069266D81423285EAD3BD
:10BE4800A362E8E7A906E4D5E26A22B1988C216BDF
:10BE580080B29047DDE7E1699B8C6069DBB24E1CDC
:10BE6800E6614354E169E368994228BFE261D0E79B
:10BE7800226D136823F080031360CCE7242C002084
:10BE88002DE9F04FBF4B1E788BB0002E40F0BC80E0
:10BE9800BD4BBE4C1D78DFF814A3DFF81493DFF810
:10BEA800148305F00105A4F10A0B54F80A3CBBB150
:10BEB800CC2707FB06B718460DF00EFB80B154F8E7
:10BEC8000A0C0DF001FB14F8023C8BB9242831D080
:10BED800F5B154F80A3C18460DF0FEFA0028EED1E8
:10BEE8000136032E04F1CC04DFD10BB0BDE8F08F8E
:10BEF800012B23D0022B2BD0032B37D0042B67D058
:10BF0800052B40D0062B4FD054F80A2C1346D2E705
:10BF180054F80A3C23281A4600F087819C4991F876
:10BF280022108142C7D19B4BCAF80090C3F80C80FD
:10BF38001346C0E7012304F8023CCAE74D2854F829
:10BF48000A2C0CBF0223002304F8023C1346B2E774
:10BF580000233C2804F8023C45D03E28D4D10122D5
:10BF6800032304F8012C04F8023CB2E7C02814D8D3
:10BF78000022042304F8050C04F8040C04F8062C29
:10BF880004F8023CA5E714F8063C14F8052C9A427C
:10BF98002FD814F8043C834203D0002304F8023C51
:10BFA80097E7062304F8023C14F801ECBEF1000FF1
:10BFB80000F08081BEF1010F00F0C481013600233A
:10BFC800032E04F8023C04F1CC047FF46EAF8CE736
:10BFD80014F8043C04F8030C5840052304F8040C36
:10BFE80004F8023C75E7032204F8013C04F8022C2B
:10BFF8006FE714F8042CF9184240013304F8042CB4
:10C0080004F8063C887264E7634B186800283FF41C
:10C018006CAF0DF03BFFDFF8A0A1604DDFF89C91FD
:10C02800DAF800000DF058FA00283FF45EAFDAF8AD
:10C0380000000DF049FA09281BD03F2819D02B68B9
:10C04800002B66D1042800F0A8810C2800F0E680B7
:10C058007F28E5D0A0F12002D2B25E2AE0D80BB941
:10C068002028DDD05A1C09F803002A601EF01CFAAB
:10C07800D6E72C68002C5AD1494B264603F5907B0D
:10C08800002E08BF1E4608335B45F9D1002E00F08C
:10C098007881A3F108083068D8F80020075D135D9F
:10C0A8009F42204402EB040140F06981671E4F441F
:10C0B80022460BB9FD2A5CD907F8013F01322A60F4
:10C0C80010F8013F11F801EF9E45F2D00AB1B045D2
:10C0D80012D034481EF0F0F9B04508D356F8080BD2
:10C0E8001EF0EAF909201EF0DFF94645F6D92E4878
:10C0F8001EF0E2F92A680024944291D2661E4E444A
:10C1080016F8010F1EF0D0F92B6801349C42F7D3C2
:10C1180086E70C2800F082800A2851D00D284FD0DD
:10C128007F2800F0FC80FF2B3FF67AAF92E71C4F88
:10C138004FF0000807F5907B464602E008375F4558
:10C148000DD0224639684846F6F71CF90028F5D183
:10C15800B846002EF2D13E4608375F45F1D1002E91
:10C1680099D1B8F1000F3FF45BAF0E481EF0A4F967
:10C17800B4E7511C202009F80200296009F80130B1
:10C188000A46A4E7594C002085620020B66B0020BF
:10C198000067002000ED00E0B02C0020B42D002046
:10C1A800DCFE0208101F0308181F0308FC9F00206C
:10C1B800EFBEADDE0400FA05183A0020B42C0020CA
:10C1C8001EF0FBF923217D4823F0B2FA002800F085
:10C1D800E280A0EB0900286088B1431E19F803101B
:10C1E800202940F0E88009EB030204E012F8011D61
:10C1F800202948D10346581E002BF7D12B604FF455
:10C2080080720021484623F07CFA6D4B1B78002B86
:10C218003FF46BAE6B481EF04FF901E76A481EF019
:10C228004BF968481EF048F9FAE668496848C97841
:10C23800684ADFF8D0E15363003118BF012101706B
:10C24800654991634021D36382F8401082F84150D8
:10C25800624963480B603832CEF80020584A0123FF
:10C2680013701EF0D9FB57481EF026F94FF40060F2
:10C2780005F0E2F85B4B93F82230232B00F0938013
:10C2880014F8023C3EE62B60574C002204F5907BE4
:10C2980009F8032002E008345C4578D02168484654
:10C2A80007F050FA0028F6D05C4570D263689847CA
:10C2B8000023A3E74D4BADF822E00FCB0DF1280C7E
:10C2C80002AF87E80F004CF824ED14F8051C14F8A9
:10C2D800033C069404EB010E624639464FF0010C0C
:10C2E80006A8CDF81CE0ADF820308DF824C0FCF786
:10C2F80031FBE8B9019F002304F8023C002F3FF40A
:10C30800EFAD54F80A0C1BF095FA013654F80A0CF4
:10C31800B847032E04F1CC047FF4C7ADE5E5013B33
:10C32800002233482B6009F803201EF0C5F877E691
:10C33800029A304B03923946A4F10A00029305F0A1
:10C34800C3FCD7E714F8053C14F8032C06942344DF
:10C3580007936E2A4FF0000308930993ADF8202045
:10C368007FF42CAE06A8F6F78FF806A8F6F780F843
:10C3780006A8F6F77DF806A8F6F77AF81EE622462C
:10C38800A4E61D48A3F108081EF096F8A6E61B4887
:10C398001EF092F88CE728681EE7084806F01CFD96
:10C3A8000BB0BDE8F08F164A14F8023CC2F80C80B6
:10C3B800CAF80090A6E5034666E700BFB42C002043
:10C3C800594C0020181F0308201F0308326300205F
:10C3D800F0240020F01F002039910108183A0020AD
:10C3E8004C1F030800670020DCFE020838FB020827
:10C3F800481F0308A46F0020101F03082C1F030800
:10C4080000ED00E0B02C00202DE9F04F2DED068B5B
:10C41800A34BA44A1C7893B000F59C412031814677
:10C4280007911160002C00F08F869F4A1268904295
:10C4380040F2DB809D4A029216689D499D4A01910F
:10C44800013C1C709C4B009206F480560493002E0D
:10C4580040F0D980994B1B78022B01F0DA80042B2D
:10C4680001F04581012B01F0F980954B9945049B1A
:10C478009B7800F25485002B40F05585914B03932F
:10C4880011F054FA904B1B68DC00054640F1C5805A
:10C49800039B1B7813F0010300F0C880009AB2F9DF
:10C4A8000610019A528C914281F2D381002D40F0FE
:10C4B800C480864C94F88C20002A40F0BE808449C1
:10C4C800844A086890F82D0000211160516091603D
:10C4D800814A002840F0B2801070002B40F0B380F1
:10C4E8007E4B1A78002A40F01581019900984E8BEE
:10C4F800B0F90070898BB0F90200B742CCBF802434
:10C50800002444F040038F42A8BF23469B0843F011
:10C518008004B042C8BF234643F040048842A8BF05
:10C528001C460098A408B0F90470B0F9060044F05D
:10C538008003B742C8BF1C4644F040038F42A8BFDF
:10C5480023469B0843F08007604CB042C8BF3B4677
:10C5580043F0400794F88E608842B8BF3B469E423D
:10C5680001F07E83A4F8902084F892205C4984F836
:10C578008E300E78002E01F0A9825F2B01F01C830B
:10C588006F2B01F03383039B1B78D80700F1C2801F
:10C5980094F89220002A40F0BD80B4F99030322BF4
:10C5A80040F3B88094F88E300120572B84F892001D
:10C5B80000F0A28002990968490741F1F3815A2BDA
:10C5C80041F0F08194F89430002B41F0FD8694F806
:10C5D800963083F0010384F89630002B41F056879B
:10C5E8000C201BF017FC3F4D95E0304B02931E6862
:10C5F800304B2F4A009306F480562F4B0192049338
:10C60800002E3FF427AF00212F48F6F737FB00280C
:10C618007FF420AF17F0B2FF1CE7029B1B6858029B
:10C628003FF536AF039B1B7803F00103274C00222C
:10C6380084F88C20002D3FF442AF274A0121117065
:10C64800002B3FF44DAF029B1B68D9067FF548AF1E
:10C65800254A1278D2063FF543AFDF043FF540AFD5
:10C6680011F050F900287FF43BAF1D4B1B78002BCD
:10C6780001F0B5861D4B9B78002D41F017873BB123
:10C688001B4A1C4B12681B689B1A002BC1F2F486CC
:10C6980010200E4C1BF0BEFB012384F88D301FE7E1
:10C6A800E82F0020C02E0020E42F0020145C00207A
:10C6B800D4660020BC4E0020EC4E0020F63200204C
:10C6C800404B4C00856200203C3B00207420002039
:10C6D800EC600020E43A0020041F0020A74C002052
:10C6E8001C010020E8600020443B00200C3D002095
:10C6F800946F002004620020134B144A19684FF409
:10C708007A73B3FBF1F3C3EB431103EB8103DB0053
:10C71800A2F8A8300E4D029B1B685F0700F1478600
:10C728000C4E05950DF1400A0022CAF8042006F1C6
:10C7380050091092344640F6330B4FF0190840F276
:10C748008337009D0BE000BF045C0020785900206F
:10C75800E86000205030002004344C4522D0A178F5
:10C76800E378994218FB0170F6D294F801E00EF1D3
:10C77800040E18FB037135F91E305B45A8BF5B46F4
:10C78800B3F5617FB8BF4FF461739842E4DA994218
:10C79800E2DB21782729DFD850460434F6F75EFA21
:10C7A8004C45DCD1CB4A059D1378CB4A9AE8030067
:10C7B80082E80300002B40F04985C84B1A78002A0C
:10C7C80000F07285C64B0693C3480121F6F756FA66
:10C7D800002840F09482049BDB78002B40F08F8285
:10C7E800C04B05932B881FB227F001071FFA87F863
:10C7F8004345A5F8008000F08887BB4F4FF0020939
:10C808000E204FF0140A4FF0FF0B87F8009087F8BE
:10C8180001A087F802B01BF0FDFA4946AE48B5F80A
:10C828000080F6F72BFA002841F0958128F00203E2
:10C838009BB243452B800BD0AB4B02201421FF2227
:10C8480018700E2059709A701BF0E4FAB5F8008041
:10C8580018F003011ABF0121084601200DF0D4F990
:10C8680024219D48F6F70AFA30B9039A13785F072E
:10C8780044BF23F004031370059B1B6813F00A0FD1
:10C8880011D006219448F6F7F9F9002800F0B88786
:10C898002B88580641F1278107218F48F6F7EEF9D2
:10C8A800002840F055870C218B48F6F7E7F92A88CD
:10C8B800002800F0438242F480739A422B8009D00A
:10C8C800894B02271421FF220E201F7059709A707D
:10C8D8001BF0A0FA854B1B78082B00F03B820E2B2F
:10C8E80000F03882029BD3F8008018F4806F12D0D1
:10C8F8007F4B1B79002B00F0E48114217648F6F772
:10C90800BDF9002840F0E28114F098FB05F058FAD0
:10C91800029BD3F80080039B93F80090754B19F0A5
:10C92800010900F0448201221A70069B00991B68D5
:10C93800B1F906105A89704801279142077080F2B0
:10C948001C826E4B4FF07E521A60019B6C4FB3F8FD
:10C9580018A0009B97F90420B3F90030387897F8AD
:10C9680001C0002AA3EB0A0714BF01224FF0FF32CF
:10C97800002FB8BF7F42B7F5FA7FA8BF4FF4FA7708
:10C98800B84280F2BC823F1A07EE907AF8EEE77A56
:10C998005C4F9A45C7ED007A03DDF1EE677AC7ED83
:10C9A800007A009BB3F902E0AEEB0A03002BB8BF94
:10C9B8005B42B3F5FA7FA8BF4FF4FA73984280F24E
:10C9C8009B821B1A07EE903AF8EEE77AF245C7ED1C
:10C9D800017A03DDF1EE677AC7ED017A009BB3F9BE
:10C9E8000400A0EB0A03002BB8BF5B42B3F5FA7F43
:10C9F800A8BF4FF4FA736345CCBFA3EB0C03002325
:10CA080002FB03F307EE903AF8EEE77A5045C7EDDC
:10CA1800027ABCBFF1EE677AC7ED027A18F4805249
:10CA280000F04382B1F5FA6F374BA8BF4FF4FA61B3
:10CA3800B1F57A7F1878B8BF4FF47A71A1F57A7199
:10CA4800002841F07880DFF8D8E030488EFB013CC0
:10CA5800CB17C3EB6C1303F1010C6FF0630830F9CB
:10CA68001CC030F9130008FB0313ACEB000103FBF7
:10CA780001F38EFB031EDB17C3EB6E1303441BB2DB
:10CA880007EE903AB8EEE78A87ED038A002A40F06D
:10CA98009D832B885A0640F109811D491D4A91ED55
:10CAA800010AD2ED018A92ED026A91ED034AD2EDB4
:10CAB800033A91ED028A92ED007AD1ED005AD7ED52
:10CAC800011A97ED002A144A144930EE445A78EEB8
:10CAD800C66A29E0084000203C3B0020594C002051
:10CAE800F0600020946000201C3A00202C3D0020BB
:10CAF800B85E002086620020601F0020B81E00205B
:10CB0800E43C0020C85E002094240020943E0020CD
:10CB1800D4040020D40000200C0100207420002040
:10CB28001F85EB510000000075EEC84A65EE266AC5
:10CB380077EE237A37EE639A75EE889A24EEA71A71
:10CB4800B0EE663AA9EE893A13F00303B0EE415A03
:10CB580070EE044A78EE867AA9EE895AF0EE660AF3
:10CB6800A4EEA73AD4EEA70AA4EEE75A33EE013AA8
:10CB7800F0EE607AF0EE674AF6EE000A35EE80AA2B
:10CB8800E9EEC94A20EEC33A35EE665A77EE286ACE
:10CB980077EEC17AAAEE263A25EE205A76EE636A37
:10CBA80034EE48AA74EE814AE9EE897AAAEE265A4A
:10CBB80037EE687A34EE084A64EEA04A63EE036AF8
:10CBC800E4EE074A75EEC05A36EE236A67EEA07A9D
:10CBD800B0EE667A95EE057AE5EE056AE5EE867AB8
:10CBE800B1EE648AF0EE665AF0EE476AB1EE674A33
:10CBF800E8EE246A63EE270A67EEA43AE4EE275AC1
:10CC0800B1EE450AB0EE609AB0EE631AA4EE277A48
:10CC180023EE244AE7EEA76AA5EE249AA0EE031AAB
:10CC2800E8EE245AB0EE448A31EEA16AE0EE240A16
:10CC3800A5EE278A66EEA16A72EE028AE5EE033A4D
:10CC480061EE211A26EE096AA4EEA47AA0EE274A1C
:10CC58000CBFD7ED022A5FED4D2A82ED005AA2EEF5
:10CC6800256AE8EEA06AE2EE081A73EEA33A27EE08
:10CC7800227A34EE044AF0EE005AE3EEA26AA4EEF9
:10CC8800226AA1EEA57AC7ED016AC1ED366A81ED87
:10CC9800356A87ED006A81ED377A82ED013AC2ED97
:10CCA800027AC2ED034A0BB987ED027AB9F1000F97
:10CCB80040F0288111F088F813B0BDEC068BBDE870
:10CCC800F08F039B1B78D9077FF51EAE4FF40F70CA
:10CCD80012F0C8FA00283FF41BAE05F059F84FF4DB
:10CCE8000F7012F029FA00283FF412AE05F050F840
:10CCF8004FF40F7012F020FA0028EED108E69C4B92
:10CD080005931B689B077FF56DADB5F8008018F09B
:10CD1800010F7FF48BAD48F0010398452B803FF459
:10CD280085AD944B022214211A700E20FF225970EF
:10CD38009A701BF06FF8B5F8008077E522F48073DD
:10CD48009BB29A422B807FF4BBAD8B4B1B78082B90
:10CD58007FF4C5AD2A8822F040039BB29A422B800B
:10CD68003FF4C0AD834B02271421FF220E201F7011
:10CD780059709A701BF04EF8B4E5B1F5FA6F80F26D
:10CD88004184187A8B1A03FB00F3C2F5FA6293FB0D
:10CD9800F2F3C3F1640307EE903AF8EEE77A9FEDF9
:10CDA800777A774B67EE877AC3ED007ACDE51B7803
:10CDB8000293002B7FF4B9AD724A1268002A3FF43F
:10CDC800B4AD714A039212F8030CDFF800B21146B1
:10CDD800D71E10F06DFD9BF800A0039A002800F004
:10CDE8005385029BBAF1000F53D107F108017879F6
:10CDF80010F05EFD002841F0E1826449B87A10F035
:10CE080057FD002800F05385BAF1020F41F0D28295
:10CE18005F49F87B10F04CFD002841F0C7825D495E
:10CE2800387D10F045FD002800F05385BAF1040F55
:10CE380041F0B8825849787E10F03AFD002841F058
:10CE4800AD825649B87F10F033FD002800F05385B5
:10CE5800BAF1060F41F09E82514997F8230010F06D
:10CE680027FD002841F092824E4997F8280010F0DB
:10CE78001FFD002800F05385BAF1080F41F08282A7
:10CE8800494997F82D0010F013FD00283FF44DADE7
:10CE980009231A4602EB82021744444A7878B97883
:10CEA8008BF80030107051703FE5019B588B814220
:10CEB800C0F2A683B1F5FA6FD4BFC0EB0101C0F58B
:10CEC800FA614FF47A7303FB01F1DFF804E19EF88D
:10CED80000C0C0F5FA63B1FBF3F1BCF1000F3FF4F9
:10CEE800B2AD9EF80130324801FB03F380FB030129
:10CEF800DB17C3EB6111A6E5DFED2E7A66E5DFED02
:10CF08002D7A45E52C4A2D4B1178186801F001015E
:10CF18000CF070FE13B0BDEC068BBDE8F08F13B9B2
:10CF2800049A01239370264B049A1D7892F82140A5
:10CF380003931B2010F0F4FC012C05F00108814636
:10CF480000F0518605F00205049A1E4E92F8203032
:10CF5800DFF880A01C4F05959346052B00F2E0866C
:10CF6800DFE813F0C100B7003A00E300E500D8009D
:10CF7800946000201C3A00202C3D00200AD7233C56
:10CF8800B81E002088620020C6390020D039002051
:10CF9800D5390020DA390020DF390020E4390020B3
:10CFA800E9390020EE390020F33900208C62002096
:10CFB8001F85EB51000000005C6F0020606F0020AF
:10CFC800856200208C3E0020E460002008000020DC
:10CFD800942400201C010020012C04BF05238BF899
:10CFE8002030B8F1000F12D0019B3088B3F9181027
:10CFF8000022134661F30F0260F31F4261F30F032F
:10D00800009861F31F4303600323426005939B4D1F
:10D01800DBF814102A68914280F0488547F23051B5
:10D028000322CBF81C108BF82020022004F004FA0D
:10D0380017F0A4FA2968DBF81C200A440421CBF86D
:10D0480018208BF82010012C40F09E862A68DBF807
:10D058001810914280F064869AF8000020B910F008
:10D068005FFC002840F05C863A6822F002023A60D1
:10D078002A687388642101FB03234FF4806000222F
:10D08800CBF810308BF820208BF8032004F0A4F99B
:10D098009BF8203061E710F049FC012807D1774D53
:10D0A80072882B68642101FB0233CBF81030B9F188
:10D0B800000F01D0B3797BBB012C00F031866F4D96
:10D0C800DBF810102A689142C0F06B8601238BF8B8
:10D0D8002030012C1ED0F379012B2AD010F0A6FBAA
:10D0E8009BF8203039E7B8F1000FD4D1059D4FF4F3
:10D0F8008060B9F1000F00F0288304F085F9049AE4
:10D1080000231361002D3FF4BBA928461AF082FEC4
:10D11800FFF7B6B9594DABE710F088FB03224FF47F
:10D128007A738BF82020CBF81C30544D7DE7534D93
:10D1380089E710F07BFB032240F6B8338BF82020F8
:10D14800CBF81C304D4D70E74D4F3B78002B01F06C
:10D1580080804C4BDFF84481DFF844B1DFF844A10C
:10D16800019345465E46009099460EE019F8041072
:10D178009847032C28DC88B93B782AF8020F013439
:10D188009C4205F1040580F23781072CE1B2304654
:10D19800DBF80430EADD984700B2EDE738F82420E0
:10D1A8006B88801A4FF47A719B1A01FB00F040F6E5
:10D1B800CA0290FBF3F00844904240F2EE23A8BF65
:10D1C80010469842B8BF184600B2D5E71D212E4830
:10D1D800F5F754FD28B100F07DBD0436A6423FF4B2
:10D1E80058AC31782629F8D1B278F3789A42F4D23B
:10D1F800049BDB78002B7FF44CAC2348F5F73EFD0D
:10D20800DFED227A002801F0548038EE678A204842
:10D218002049FDEEC87ACAF57A73CDED007ABDF9DA
:10D228000020120380FB0240D2171BB2C2EBA012EF
:10D2380003FB02F343F30F33534407EE903AF8EE3F
:10D24800E77A0123C7ED037A0B7022E4124B03E05F
:10D2580004339C423FF4B1AA19782329F8D198786D
:10D26800DA789042F4D20848F5F708FD00283FF430
:10D27800A4AA14201AF0CEFDFFF79FBA946F0020DD
:10D2880014310020D46600203C3B002000007A4482
:10D29800D34D6210301F002050300020283100206C
:10D2A800AC2E002072200020DFF8F892DFF8F8A2F8
:10D2B800AC4F059209F15A084FF0010B494619F88D
:10D2C800010C10F0F5FA00B399F8040099F802304F
:10D2D80099F803E000EB400107EB8101013BD1F82D
:10D2E800A02003EB4303534493420ED097F8CC207D
:10D2F800C1F8A0300BFA00F022EA0000059B81F883
:10D308009CE0C1F8A43087F8CC0009F10609C845AB
:10D31800D4D1954B954A06931946954BDFF88CA2C4
:10D32800126809681B7807910593AAF19C094FF0C8
:10D33800000B9046DAF8043083B31F7877B3DAF835
:10D348000820A8EB0202002A0CDB99F8CC20012166
:10D3580001FA0BF122EA010208F5FA7189F8CC20EA
:10D36800CAF80810059ACAB19AF800205978043208
:10D37800D2B2002940F0738201990098098B30F9E4
:10D38800122001F1C800824240F3D08499F8CC10F1
:10D398009A7841FA0BF3D80740F12E850BF1010B6F
:10D3A800BBF1040F0AF10C0AC4D1FFF70DBA6D4C9A
:10D3B80094F896305BB1039B1B78DE0707D5009B7A
:10D3C800B3F90620019B5B8B9A4200F30485112177
:10D3D8006848F5F753FC002800F0298294F89A3041
:10D3E8002BB994F8943013B93223A4F89830012358
:10D3F80084F89A30FFF794B9DDF800905E4A0292FB
:10D408005E49126842F2010AA1FB091B12EA0A0AE4
:10D418004FEA9B1B00F00882594D5A48544C5A4910
:10D428002E780078267008701EB157490E7886F05D
:10D4380001064C4C0F2184F82410002B00F05B836C
:10D44800019D524BB5F826C0B5F824E0019D0C9318
:10D4580018462D8B00784E4B0E9594F8255005955F
:10D468004C4D0095A3FB00535B0803EB4303C31A21
:10D47800DBB20B90CDF824C002F48052089304F17B
:10D4880028000BF59673CDF8349097F80080DDF8F6
:10D498001490DFF81CC105943E4C0A910F920021AC
:10D4A80006930496CDF80CE0049B002B00F0A082B4
:10D4B800059B039D33F911201FFA82FEAE454FEA02
:10D4C800410303D3099DAE4540F2D7825CF8212081
:10D4D800934580F09782E25EBAF1000F40F0AC828B
:10D4E80001314145E25200F10600DDDB0A9A059C54
:10D4F800294B84F824200F2A49460CBF0122002218
:10D50800DDF8349084F825101A7000F0FB82234B64
:10D518001C491D4ADFF854B004931C46042001231B
:10D528000B70137003F088FFDBF80030A1686268A5
:10D53800E3605B1A934284BF002384F82130029B86
:10D548003C781E68002C00F0E486019A144DB2F86D
:10D5580024E0178B0F4916F48056284640F00E83B6
:10D56800324638E074200020F0600020946F0020DC
:10D57800914E00203C3B0020145C0020D34D6210EB
:10D58800882E0020BC000020BD00002005300020AF
:10D59800ABAAAAAABC4E0020453B0020EC4E0020B6
:10D5A8005C310020DD38002048FB020810210020F3
:10D5B800083000206F12833F437803EB830303EBAB
:10D5C800830303F2EE239BB20132A24221F8023B0D
:10D5D80000F102000ED015F81230002B00F0518235
:10D5E800022BE9D001320B8821F8023BA24200F15C
:10D5F8000200F0D10C9A137801331370FEF727BF9D
:10D60800114662E41B7AC3F1640307EE903AFFF710
:10D61800C4BB019A0099537DD27D013B31F9133087
:10D628001AB1C3F53B6308331BB2A3F57A7307EE4F
:10D63800903A1FED207AC14AF8EEE77A40F2FF31BE
:10D6480067EE877AFCEEE77ACDED037ABDF80C3009
:10D658008B4228BF0B461380FEF707BFB84CD4F89F
:10D668008830A9EB0303002BFEF6FFAEB54AB64B94
:10D67800527C019933F812308A7DDFEDB46A9FED50
:10D68800B46AC97D9BB207EE102A07EE903AB8EE4D
:10D69800C77AF8EEE77A27EE267A67EE867A079A4F
:10D6A800C4F88820C7EE876A40F2FF32FCEEE67ABB
:10D6B800CDED037ABDF80C30934228BF134609B16B
:10D6C800D31A9BB2A348A44D0178A44C35F8116035
:10D6D800226825F81130921B13440131974D2360BD
:10D6E80001F00F021B0902702B80FEF7BEBEFEF789
:10D6F800FFF99B4B9B4A1B68C31A93427EF7B5AE52
:10D708008E4B00221A80FEF7B0BE02219648F5F72C
:10D71800B5FA00283FF48AA82F8018F0020F7FF48A
:10D7280097A848F0020343452B803FF491A88F4BFC
:10D73800022214211A700E20FF2259709A701AF0D2
:10D7480069FBB5F80080FFF783B803F045FED6E41F
:10D75800874AB2F90030002BB8BF5B42B3F5E17FCE
:10D76800BFF6A1A8B2F90230002BB8BF5B42B3F5EF
:10D77800E17FBFF698A87F4B93ED057AD3ED077A42
:10D78800D3ED096A93ED030A77EEA67A30EE070A1D
:10D79800F7EE000AB0EE007AE7EEC70A30EE000AAC
:10D7A800F5F730F8B6EE008A20EE488A9FED720A47
:10D7B80038EE000AFDEEC07A17EE903A2033402B7F
:10D7C80040F217839FED6D0A6D4FDFED6C7A87EDA0
:10D7D800000ABDEEC87AC7ED017A17EE103A203379
:10D7E800402BC7ED027A00F20E85B0EE480AF4F736
:10D7F8008FFF0A2087ED030A1AF00CFBFFF753B8D6
:10D808002A8822F040039BB29A422B803FF444A816
:10D81800564B02271421FF220E201F7059709A7050
:10D828001AF0F8FAFFF738B856490E78FCE594F87C
:10D838009430002B3EF474AF039B1B7813F0010364
:10D848007EF46EAF012284F8943084F89520FEF7B8
:10D8580067BF3B4C012284F88C20FEF7EEBE0129FD
:10D8680000F0888499F8CC20012303FA0BF30BF11C
:10D87800010B1343BBF1040F89F8CC300AF10C0AF1
:10D888007FF458ADFEF7A0BF511D787910F010F85D
:10D8980000283FF4B2AABAF1010F40F08F8507F1D2
:10D8A8000D01B87A10F004F8002840F08385364955
:10D8B800F87B0FF0FDFF00283FF4B1AABAF1030F7F
:10D8C80040F074853149387D0FF0F2FF002840F0B0
:10D8D80069852F49787E0FF0EBFF00283FF4B1AA45
:10D8E800BAF1050F40F05A852A49B87F0FF0E0FFDA
:10D8F800002840F04F85284997F823000FF0D8FFFB
:10D9080000283FF4B1AABAF1070F40F03F85234938
:10D9180097F828000FF0CCFF002840F03385204905
:10D9280097F82D000FF0C4FF00283EF4FEAFBAF1BF
:10D93800090F3EF4FAAFFFF7ABBA00BFE44E002080
:10D94800742000207C6600209C6600200000C842ED
:10D9580000008044F7320020FC320020F83200201A
:10D96800E01F002060E316003C3B00201C3A00202A
:10D9780098600020E4000020DB0FC93F0000000091
:10D98800D4040020914E0020D5390020DA39002037
:10D99800DF390020E4390020E9390020EE39002081
:10D9A800F33900205D2B00F032845B2B00F02982D4
:10D9B8005E2B00F0CD84562B00F0CC84972B00F022
:10D9C800D584A72B00F0BC84B14D2A88920740F07B
:10D9D8004484A3F1B702072A00F22D82DFE812F08F
:10D9E80026022B022B022B0221022B021C021702F9
:10D9F800039B002B3FD05CF8212093454FEA41035D
:10DA0800FFF469ADA34AA34DD25C05EB030E002ACF
:10DA180000F09480022A47D19EF8012002EB82028E
:10DA280002EB820202F2EE2292B2032933DD12B235
:10DA3800BAF1000F3FF454AD089D20F81520B9F154
:10DA4800000F03D10B9D022D7FF64AADB0F8009070
:10DA58004288B0F804E04A4496448F4A0FFA8EFE92
:10DA680082FB0E528D4DA2EBEE7225F803E012B246
:10DA78004FF0010934E51A464B00069D4CF8215039
:10DA88002AE5D3B2022B04D9032B7FF4ABAD73463E
:10DA98009AE53B4698E5012505FA01FE0A9D25EA27
:10DAA8000E0512B20A9517E5E25ABEE77C4A1278CB
:10DAB800002A7FF4B3AAB8F1000F3FF4AFAA012CF3
:10DAC80040F02E819BF82030FFF747BA3146754861
:10DAD800F5F7D4F8002800F09F8084F8936017F0D9
:10DAE80039F8FEF750BD43F0400293422A807FF494
:10DAF8008FAEFEF7D1BE6C4B6C4A0C9201221A70A5
:10DB08006B4B00931B216748F5F7B8F800287FF4A2
:10DB1800FEAC684BDFF8B4B104931946DBF800306B
:10DB2800CA688B609B1AC82B00F2E483029B1E68AC
:10DB380006F480565EE55B78FFF7D5B9CAB2022ACB
:10DB480040F21683032AAFD10E9A0F9D039E002D33
:10DB580008BF324669E728F0010292B242452A809E
:10DB68003FF4DBAD0E2087F8009087F801A087F816
:10DB780002B01AF04FF9B5F80080CEE500220FE0A8
:10DB8800437803EB830303EB830303F2EE239BB297
:10DB98000132A24221F8023B00F102003FF42AAD13
:10DBA80015F812301BB1022BEAD00B88F0E7D3B27C
:10DBB800032BFAD83B46EBE7B2F5FA7FFEF6AAAD9F
:10DBC80094F89230002B7EF4A5AD039B1B780122BC
:10DBD80013EA020584F8922000F0088316F0CEFCC0
:10DBE8002B4DFEF798BD0025FFF7AEB9B2F5FA7FC9
:10DBF800FEF690AD94F89230002B7EF48BAD039A2C
:10DC08001278012184F89210D40700F1028316F0EB
:10DC1800A1FF1F4DFEF77FBD039B274A1B781060AD
:10DC2800DE077EF5B5AC254B1B78002B3EF472ADB4
:10DC3800049BDB78002B7EF46DAD94F893300133B0
:10DC4800DBB2032B84F893307EF664AD1C4B5B7813
:10DC580013B9002D7EF45EAD16F090FCFEF793BC70
:10DC6800184A19491068B4F99020C66981FB060161
:10DC78008911F617701A00F5FF407F3082423EF78F
:10DC880075AC891B0A4412B2A4F89020FEF76EBC4A
:10DC9800E86000205C31002056555555E4200020EE
:10DCA800F41E00203C3B0020453B002005300020AE
:10DCB800BC4E0020EC4E002008620020914E00204F
:10DCC8000C3D00207C540020D34D6210946F00203E
:10DCD80000007A44049BDB78002B7FF482AA5FED76
:10DCE800047AC24938EE678ACAF5FA63FDEEC87A43
:10DCF8001BB2CDED007ABDF90020120381FB0201B1
:10DD0800D217C2EBA11203FB02F343F30F335344C0
:10DD180007EE903AB8EEE78A87ED038AFFF761BA13
:10DD2800059D002D3EF4ACABFFF7EFB9C8398A4228
:10DD380042DA99F8CC109A7841FA0BF3D9073FF5F3
:10DD48002DAB5242012008921AF04AF97B1E089A1C
:10DD5800162B00F2CF80DFE813F0A901BD01900176
:10DD6800E201D101F6017B016601510134011F0175
:10DD7800CD00E2010C01F6017B016601F800E40028
:10DD8800D000BD00A7009300AB460499DBF8002043
:10DD9800CB69059D13448B61002D3EF471ABFFF7F1
:10DDA800B4B90FF043FD032140F6B8328BF82010C8
:10DDB800CBF81C20FFF739B999F8CC30012202FAC8
:10DDC8000BF223EA020308F5FA7289F8CC30CAF894
:10DDD8000820FFF7E3BA00218548F4F74FFF002831
:10DDE8007FF4F5AA322384F89600A4F89830FFF758
:10DDF800EEBAF4F78DFCE7E4002A0CBF01200220FC
:10DE0800A1E70120FCF7E2FC7A4DFEF784BC022072
:10DE180017F03CFAFEF77FBC032017F037FAFEF73D
:10DE28007ABC002017F032FAFEF775BC012017F013
:10DE38002DFAFEF770BC9E2B00F00A839D2B00F094
:10DE48000083AE2B00F0F682AD2B00F0EC82EF2BB6
:10DE580000F0E682FD2B00F0E082FB2B00F0CF8281
:10DE6800FE2B00F0FC82F72B00F00D837B2B7EF459
:10DE780052AC4FF4FA61022017F030F9FEF74BBCB0
:10DE8800D9F8D0005C4B90F836109B78114464297F
:10DE9800A8BF642121EAE17180F83610002B40F018
:10DEA80001831DF02FFADDE4D9F8D000524B90F829
:10DEB80037109B781144FE29A8BFFE2121EAE171A1
:10DEC80080F83710002BECD016200FF073FDD9F82E
:10DED800D000E6E70798484B41781144B1F5967FA2
:10DEE800A8BF4FF4967121EAE17141709B78002B2D
:10DEF80040F0D282D9F8D000D3E7D9F8D0003E4B11
:10DF080081781144C829A8BFC82121EAE17181702C
:10DF18009B78002BC5D014200FF04CFDD9F8D00009
:10DF2800BFE7D9F8D000344B41781144C829A8BFBD
:10DF3800C82121EAE17141709B78002BB1D01320F0
:10DF48000FF038FDD9F8D000ABE7D9F8D0002A4B4C
:10DF580001781144C829A8BFC82121EAE1710170DC
:10DF68009B78002B9DD012200FF024FDD9F8D0000B
:10DF780097E7214B07989B78417911446429A8BFFA
:10DF8800642121EAE1714171002BB3D00E200FF01A
:10DF980011FDD9F8D00084E7D9F8D000164B017AE2
:10DFA8009B781144C829A8BFC82121EAE1710172F0
:10DFB800002B3FF476AF0B200FF0FCFCD9F8D00013
:10DFC8006FE7D9F8D0000C4BC1799B781144C82968
:10DFD800A8BFC82121EAE171C171002B3FF461AFEC
:10DFE8000A200FF0E7FCD9F8D0005AE7D34D6210A9
:10DFF8003C3B0020E860002092640020D9F8D00063
:10E00800C64B81799B781144C829A8BFC82121EA49
:10E01800E1718171002B3FF444AF09200FF0CAFC75
:10E02800D9F8D0003DE7D9F8D000BC4B417993F836
:10E0380002E01144C829A8BFC82121EAE171417151
:10E04800BEF1000F40F04782112F7FF459AF28E747
:10E05800D9F8D000B14B017993F802E01144C829EE
:10E06800A8BFC82121EAE1710171BEF1000F40F09B
:10E078002882102F7FF458AF13E70799A74B0F7921
:10E0880008931744642FA8BF642727EAE7770F711E
:10E098000FF0AAFC089B9B78002B3FF42BAF0320C2
:10E0A80039460FF087FCD9F8D000FAE607989B4B61
:10E0B80001781144FA29A8BFFA2121EAE171017017
:10E0C8009B78002B3FF416AF01200FF073FCD9F8B2
:10E0D800D000E6E60798914B817811446429A8BFDF
:10E0E800642121EAE17181709B78002B3FF402AF33
:10E0F80002200FF05FFCD9F8D000D2E60798874BD2
:10E10800C1799B78114481F30801C171002B3FF458
:10E11800F1AE05200FF04EFCD9F8D000C1E6079803
:10E128007E4B817993F802E011446429A8BF6421E9
:10E1380021EAE1718171BEF1000F40F0D6810D2F07
:10E148007FF418AFD6E6D9F8D000744BC17893F8AD
:10E1580002E01144C829A8BFC82121EAE171C170B1
:10E16800BEF1000F40F07E810F2F7FF4F1AE98E6EC
:10E178000E9A5AE400999B7831F91220B2F5617F22
:10E188004FF4966191FBF3F348DB40F6330191427B
:10E19800A8BF11460C2FA1F5617191FBF3F100F0B6
:10E1A800EF80182F7FF45EABC9B2C8290B46A8BF11
:10E1B800C823D9F8D020D77DD8B2B8423FF452ABA3
:10E1C800DF1B564BD07548BF0737FF109B780137C8
:10E1D800FFB23BB9002F3FF445AB384619F000FFBA
:10E1E800FFF740BB18200FF0E5FBF3E70F2019F00D
:10E1F80011FEB4F8903084F89250FA3BA4F89030AD
:10E20800474DFEF788BAB0EE670AFFF7F2BA00206A
:10E21800F8E5444A424D1360FEF77DBA0C2F40F0F2
:10E228009F8000273946404B09915B78BB423FF4F9
:10E2380019AB3A4B0893384617F028F8089B099908
:10E248009B781BB1C9B20C200FF0B4FB0137FFB2A9
:10E25800C0E7364A0192FFF7D1B80022BB2B1092D3
:10E2680000F08B80B72B00F0B680BE2B00F0AA80A0
:10E27800BD2B7FF4E0AD4FF6FE732D49C8898E891A
:10E28800024433448B81CA8106F03EFEF3F76EFDEB
:10E2980006F022FEFCF75EFB012019F0A1FEB4F89F
:10E2A80090300022FA3BA4F8903084F89220FEF7D0
:10E2B80032BA38EE678A1F4B1F491870FDEEC87ACC
:10E2C800CAF5FA63CDED007ABDF90020120381FB8F
:10E2D8000201D217C2EBA1121BB203FB02F343F3F4
:10E2E8000F33534407EE903AF8EEE77AC7ED037A16
:10E2F800FEF7CFBB114A029B1E68136823F0040384
:10E308001360049A012306F4805682F82130FFF73F
:10E3180071B906F48056FFF76DB900BF926400200A
:10E32800E86000200862002032630020D4660020E4
:10E33800EC3C0020301F0020D34D6210E460002028
:10E348006E4A6F4D137843F004031370FEF7E3B978
:10E35800022057E5FCF79EFC94F88E30FFF72EBBA1
:10E36800182F7FF47FAA00210B4622E7654B644DE6
:10E378004FF4C8721A80FEF7CEB9134602227CE722
:10E38800CFB250E708231A46FEF784BD07231A4682
:10E39800FEF780BD06231A46FEF77CBD05231A4604
:10E3A800FEF778BD04231A46FEF774BD03231A4608
:10E3B800FEF770BD02231A46FEF76CBD01231A460C
:10E3C800FEF768BD022358E784F8942084F8950086
:10E3D8004B4DFEF7EDBF13464FF6FE724DE7002D8D
:10E3E8003EF456A9484C94F88D30002B3EF478A89A
:10E3F80019F0F4FC002384F88D30FEF771B8002181
:10E40800022016F06BFEB4F890300022963BA4F878
:10E41800903084F89220FEF77EB900210120F0E7C1
:10E4280000210846EDE7FF21002017F0BFFB94F814
:10E438008E300CE50121002017F0B8FB94F88E30DF
:10E4480002E50021FF2017F0B1FB94F88E30F8E4C4
:10E458000021012017F0AAFB94F88E30EEE4002189
:10E468000320CEE70F20099308920FF0A3FAD9F8FA
:10E47800D000099B089A77E6234C16F07FF884F8B9
:10E488008D50FEF72DB800210420BAE70B2019F0B3
:10E49800C1FC1B4DFEF73FB915200FF08BFAD9F8D8
:10E4A800D000FEE417200FF085FA23E5002B99D061
:10E4B8001649174A09684FF47A7000FB0313136072
:10E4C80090E71020099308920FF074FAD9F8D00059
:10E4D800099B089ACDE51120099308920FF06AFA72
:10E4E800D9F8D000099B089AAEE50D200993089247
:10E4F8000FF060FA099B089A21E600BF443B002010
:10E50800E8600020AE3E002074200020946F0020B8
:10E51800046200202DE9F04F2DED028B93B00546E3
:10E5280012F08CFDB24B1E7826B113B0BDEC028BF5
:10E53800BDE8F08FAF4F3B685805F6D5DFF8188374
:10E54800D8F80020002A00F01B81AB4CD4F8283101
:10E5580003F5F43348339D42C0F01281A74994F87B
:10E568002C310968C4F828510133DBB2890784F8D3
:10E578002C3101F11E81580701F05C80282BA04B3B
:10E58800029301F0AB815E2090479E4B1B78002BD5
:10E598006BD0994C9C4AD4F83031EB1A934200F274
:10E5A800CD87DFF8B8A29AF80080B8F1000F33D110
:10E5B800DFF86492D9F800000AF08EFFC0B2012893
:10E5C8000ED90228914F41F095823B78002B41F0FB
:10E5D800C483D4F83831EB1AB3F57A6F81F07184BB
:10E5E8008B480768002F40D09AF80030BBB9894B98
:10E5F800D9F800001B689B781E3B012B4FF00201E5
:10E6080041F2B783043015F029FB012200238AF870
:10E61800002084F8443126E07D4807682FB3D4F8F9
:10E62800403140F6B732EB1A93421ED994F83C3188
:10E63800002B01F05682013BDBB284F83C31002B01
:10E6480001F0248117F8011B94F84421076094F81D
:10E65800453171480A440133006884F8442184F83C
:10E6680045310AF03DFFC4F840516C4A029B1278CC
:10E678001B68012A03F101030A9300F0B086684B76
:10E688001B786BB1674F3B6853B1029B5A4CD3F868
:10E6980000B0D4F85831ABEB0303632B00F23F868C
:10E6A800DFF8BC8198F800A0BAF1020F01F0CA8027
:10E6B800564F97F87430032B00F086875A4B1B7817
:10E6C80073B15A4E33685BB14B4CFDF711FAD4F86D
:10E6D800643144F61F62C31A9342834600F2D48021
:10E6E800534B1B78002B4ED1524B1B7843B1424CF5
:10E6F800D4F8B43203F50043E8339D4280F0E58650
:10E708004D4B1B78002B3FF410AF3B4E4B4C4C4D00
:10E7180006F2BD2720680AF0DFFE00283FF405AFA7
:10E7280020680AF0D1FE2B7880465A1E33B1206843
:10E738002A700AF0D1FE0028F2D1F6E60322394603
:10E74800781E20F0C4FF96F8BC3296F8BD2286F8F1
:10E75800BF8283F47F4383F0FF039B1A1FFA88F874
:10E768009BB2B8EB132FD5D196F8BE22DBB29A42F2
:10E77800D0D1781E14F0A0FD2B7818442870C9E772
:10E788001F4B029301E72F4C2278002A40F01E8687
:10E79800DFF8D09099F80040002C65D12A4E3078E7
:10E7A800002841F06582144C284ED4F8AC22317808
:10E7B800274B93FBF1F313449D4295D3254A94F8D4
:10E7C800B032C4F8AC52D75CF90701F1DC83BA0760
:10E7D80001F195837B0701F1F58294F8B032317825
:10E7E800013393FBF1F201FB123384F8B0327BE77B
:10E7F800594C0020145C0020542100209460002013
:10E80800946F0020664F00203F0D03000C0000208D
:10E8180000610020FC600020F8600020674F0020A5
:10E82800744F0020AC4300207C4F0020804F002014
:10E83800C04F0020D14F0020864F00208C4F002071
:10E84800904F0020584F0020C84F0020D04F002084
:10E85800A0860100CC4F0020086100200461002040
:10E86800DA2F0020C94F0020054E376E002F41F0E7
:10E878007080044B89F80070C3F8AC5234E700BFCD
:10E88800D84F00205421002094F86A31002B41F021
:10E898000A80E04B1B6803F00802002A48F603418F
:10E8A8004AF60B404BF60F4249F6074704BF0246AB
:10E8B8000F4613F0040F4FF0190118BF17469A06B8
:10E8C80084F86A1103D547F4804747F0200702F01F
:10E8D8008BFFC7F30909002841F0A883CE4B9B7929
:10E8E800002B41F09C83984664204FF0FF3A4FF08C
:10E8F800000C0A970B97ADF834C0CDF83AC0CDF8A4
:10E908003EC0CDF842C0CDF83090ADF83680ADF8B5
:10E9180038A08DF846000AAF0FCFDFF80CE384F873
:10E9280005C0AEE80F0097E80F00AEE807002EF824
:10E93800023B71464FF0010C1B0CFE271F20C8221A
:10E9480001F81E39A770A27184F807C0E07094F826
:10E958007A01207180F0F10383EA0313DAB2130914
:10E9680083F0E70343EA022383EAC2031BB283EA84
:10E978000312D2B2C3F3072383EA121343EA022332
:10E9880083EAC2031BB283F0C80282EA0212D2B23F
:10E99800C3F3072383EA121343EA022383EAC20379
:10E9A8001BB283EA0C0787EA0717FFB2C3F30722F3
:10E9B80082EA171242EA072200EB0C0382EAC70731
:10E9C8000EEB0C0084F87A31278011F8013B7B406C
:10E9D80083EA0313DBB21A0982EA172242EA032206
:10E9E80082EAC3031BB29FB281422780EDD183F034
:10E9F8007C0383EA0313DBB24FEA131E8EEA172E59
:10EA08008EEA032E8EEAC30E0FFA8EFE1FFA8EF9D7
:10EA1800DFF818C2A4F800905FFA8EFE4FEA1929B1
:10EA280084F8289084F827E00CF5D17804F1220ABC
:10EA3800DCF80000DCF80410DCF80820DCF80C3006
:10EA480047460FC70CF1100CD445B846F0D1DCF896
:10EA580000003860714F9CF8043088F8043007F1E2
:10EA6800270884F8C9E184F8CA9117F8011F3068AB
:10EA78000AF036FDB845F8D194F86B21002A40F029
:10EA88000D876749029B08781B680A2184F86B1177
:10EA9800002801F0DC80DFF898E10128BEF80010BA
:10EAA800059141F208840228BEF8028001F0B4837F
:10EAB800BEF804100491032801F0E8830428BEF886
:10EAC80006A001F0F083BEF808100391052801F0B4
:10EAD800E6830628BEF80AC001F0EA830728BEF8D4
:10EAE8000C1001D0BEF80E2094F87A010A9307465C
:10EAF80087F0300383EA0313DBB24FEA131E494859
:10EB080006978EF07A0E4EEA032E008827718EEA59
:10EB1800C303DFF820E1C0EB00208EFB007E8644B3
:10EB2800C017C0EB6E270797059F4FF0000967F3E2
:10EB38000F09049F68F31F494FF0000867F30F0897
:10EB4800039FCDF82C901BB24FF0000E83EA031000
:10EB580067F30F0E0027C0B261F30F07C3F3072353
:10EB68006CF31F4E62F31F474FF0000C9DF81C20FA
:10EB7800CDF834E083EA10136AF31F48CDF83080EB
:10EB88000E978DF83CC08DF83D2043EA00230DF127
:10EB9800280883EAC007B8E80F003FB287F0C80921
:10EBA80089EA0919DFF880E084F805C05FFA89F975
:10EBB800C7F30727AEE80F0087EA191747EA0923C2
:10EBC80098E8030083EAC9031BB283F023074EF8D1
:10EBD800040B87EA0717FFB2C3F3072282EA17126A
:10EBE800069B704642EA072203F1010882EAC7073A
:10EBF80020F814194FF0230CFE211622C82384F89C
:10EC08007A8127800EF1020E84F807C0A170E270A5
:10EC1800A37111E09460002084600020F722002096
:10EC2800AC2E0020E44E00205C210020562100205C
:10EC3800BC4E00200308208010F8013B7B4083EA8B
:10EC48000313DBB21A0982EA172242EA032282EA94
:10EC5800C3031BB29FB270452780EDD183F0F40344
:10EC680083EA0313DBB21A0982EA172282EA032233
:10EC780082EAC3031BB21FFA83FEE74FA4F800E041
:10EC88005FFA83FC4FEA1E2984F81EC084F81F909F
:10EC98007968BA683868FB6807F5D17EAEE80F0076
:10ECA80038697969BA6904F2C118AEE8070004F254
:10ECB800A31784F8C19184F8C0C117F8011F306800
:10ECC8000AF00EFCB845F8D194F87271002F40F0A4
:10ECD800F385D24B94F87AC1B3F90010B3F9022046
:10ECE800B3F904309FEDCE6A677107EE103A029BC4
:10ECF8001B680A938CF06A0383EA031306EE901AE2
:10ED0800D9B20B0983F0D50343EA012383EAC1038F
:10ED18001BB283EA03115242C9B207EE902AC3F329
:10ED2800072383EA111343EA0123F8EEE77AF8EEA2
:10ED3800E66AB8EEC77A83EAC1031BB267EE867A41
:10ED480066EE866A27EE067A002083F0C80ECDEDBF
:10ED58000C7ACDED0B6A8DED0D7A0E900F90109018
:10ED68008EEA0E180DF128095FFA88F8C3F3072E0A
:10ED7800B9E80F008EEA181E4EEA082E8EEAC80E71
:10ED8800DFF8B0820FFA8EFEA8E80F008EF01E079B
:10ED980099E8070087EA071A5FFA8AFACEF3072785
:10EDA80087EA1A1747EA0A2788E8070087EACA079E
:10EDB8001C214FF0050A4FF01E094FF0FE0EC82225
:10EDC8000CF10103E17084F872A184F8079084F8CB
:10EDD80002E0A8F11001A27108F10C0084F804C047
:10EDE800278084F87A3111F8013B7B4083EA0313CA
:10EDF800DBB21A0982EA172242EA032282EAC30333
:10EE08001BB29FB281422780EDD183F0270383EAAA
:10EE18000313DBB21A0982EA172282EA032282EA82
:10EE2800C3031BB21FFA83FCDFF8EC81A4F800C00F
:10EE38005FFA83FE4FEA1C2C84F825C084F824E08E
:10EE480008F5D17904F1220AD8F80000D8F804109E
:10EE5800D8F80820D8F80C304F460FC708F110082A
:10EE6800D045B946F0D16F4FB8F80030A9F8003056
:10EE780007F1240884F8C6E184F8C7C117F8011F10
:10EE880030680AF02DFBB845F8D194F87331029335
:10EE9800002B40F00D8594F87AA1604B624AB3F9D3
:10EEA8000410B2F90620614F6148DFF888E184F860
:10EEB80004A08AF0220383EA03135FFA83FC4FEA73
:10EEC8001C1383F0590343EA0C2383EACC031BB2D7
:10EED800B2F5FA6F83EA031C5FFA8CFCA8BF4FF403
:10EEE800FA62C3F30723B2F57A7F83EA1C1343EA75
:10EEF8000C23B8BF4FF47A7283EACC03A2F57A7276
:10EF08004FF0640C0CFB02F287FB027C80FB017063
:10EF1800D217C9174FF000091FB2C2EBAC12C1EBF0
:10EF2800A0030DF12808CDF82890CDF82C90CDF845
:10EF38003090CDF8349087F0C80CADF83A20ADF891
:10EF48003830C146B9E80F008CEA0C1C5FFA8CFC1B
:10EF5800C7F3072787EA1C1747EA0C2787EACC0775
:10EF6800AEE80F003FB287F04A0383EA0311C9B243
:10EF7800C7F3072383EA111343EA0123724683EA9E
:10EF8800C103D9F800C09DF8081061710AF10107A2
:10EF980005204A214FF0FE0984F87A7142F810C919
:10EFA80014274FF0C80C84F8730123800EF1040E67
:10EFB800E17184F80290E77084F806C0184612F8E8
:10EFC800011B414081EA0111C9B20B0983EA1023F0
:10EFD80043EA012383EAC10109B288B2724520805D
:10EFE800EDD181F0140181EA0111C9B24FEA111E75
:10EFF8008EEA102E8EEA012E8EEAC10E0FFA8EFED0
:10F008001FFA8EF94FEA192C034B034884F81DC0E8
:10F018005FFA8EFE10E000BF5621002098600020A5
:10F0280088C3E43AF7220020BC4E0020D34D62107A
:10F03800676666665C21002084F81CE0D94F596831
:10F048009A680068DB68A4F8009007F5D179A9E808
:10F058000F0038697969B7F818A0A9E8030004F225
:10F06800A317A9F800A0BA4684F8BFC184F8BEE186
:10F0780004F2BF191AF8011F30680AF031FAD145B5
:10F08800F8D1C94BC94A1B781278013B12F001002C
:10F09800DBB214BFC0214021172B03D8C44A134444
:10F0A8001B7B0293C34B1A8893071ABF002341F0B6
:10F0B8001001012312F4027F18BF022312F0100F6F
:10F0C80018BF062312F0200F18BF1023002840F0A5
:10F0D800EE864FF0030994F87AC10A938CF0460340
:10F0E80083EA0313DAB2130983F0920343EA022393
:10F0F80083EAC2031BB283EA0310C0B2C3F3072238
:10F1080082EA101242EA002282EAC00212B282F0B7
:10F11800C80E8EEA0E1E00235FFA8EFE9DF808A028
:10F128008DF82CA00320C2F307228DF82F9082EAD5
:10F138001E128DF82D308DF82E108DF8300042EA11
:10F148000E2998E8070089EACE0E0FFA8EF8DFF844
:10F158006CE2E37188EA0819AEE803005FFA89F9FE
:10F16800C8F3072888EA191848EA092181EAC90971
:10F1780094F808808EF800200FFA89F988EA0902C5
:10F1880082EA02185FFA88F8C9F3072282EA18129D
:10F1980042EA0822607AA17A94F80B90637182EAB5
:10F1A800C80212B2504080EA0010C0B2C2F307226F
:10F1B80082EA101242EA002282EAC00212B25140E8
:10F1C80081EA0111C9B2C2F3072282EA111242EAA6
:10F1D800012282EAC10212B289EA020989EA0919FE
:10F1E8005FFA89F9C2F3072282EA191242EA092270
:10F1F80094F80C80607BA17B84F804C082EAC90281
:10F2080012B288EA020888EA08185FFA88F8C2F396
:10F21800072282EA181242EA082282EAC80212B2D7
:10F22800504080EA0010C0B2C2F3072282EA1012EE
:10F2380042EA002282EAC00212B2514081EA011178
:10F24800C9B2C2F3072282EA111242EA012282EA13
:10F25800C102E17B94F8109013B281EA030282EABA
:10F268000212D2B2C3F3072383EA121343EA02233A
:10F2780083EAC2031BB289EA030282EA0212D2B20B
:10F28800C3F3072383EA121343EA022383EAC20380
:10F298001BB283F0320282EA0212D2B2C3F307230E
:10F2A80083EA121343EA022383EAC2031BB29AB227
:10F2B8004FF0FE08DBB222800920C8210CF1010CB6
:10F2C80084F802804FEA1228AEF10E02E070A171B4
:10F2D80084F87AC184F812800293637451685EF8E6
:10F2E8000E0C92683EF8023C0EF5CA7CACE80700AA
:10F2F800ACF800309DF808308CF802900EF5D27A00
:10F3080084F8B48184F8B33117F8011F30680AF023
:10F31800E7F8BA45F8D1C4F864B1FFF7E1B9DFF806
:10F32800A0A0DFF8A080DFF8A090412014F0F4F945
:10F33800BAF9023088FB0320DB17C3EBA00080B2C8
:10F3480014F0D0F9BAF9003088FB0320DB17C3EBBF
:10F35800A00080B214F0C6F9BAF9043088FB032083
:10F36800DB17C3EBA00080B214F0BCF999F80010C9
:10F3780038680AF0B5F894F85C3113F0010800F029
:10F38800BF830D4AC4F858B10133DBB2A2FB0312A4
:10F39800D20802EB8202A3EB420384F85C31FFF748
:10F3A8007FB900BF562100202C3D00208562002037
:10F3B80090FB0208E8600020CDCCCCCC5C2100207A
:10F3C8009860002067666666514C0020894B8A4920
:10F3D80018680AF051F800232370FFF7D9B9874F4E
:10F3E800386800283FF44BA94FF0000ADFF83C8248
:10F3F800834CAB4655460AF06FF8F8B1F5B94FF0B3
:10F408000109AA4638680AF05FF883B27E2B00F03B
:10F418002E8298F80120002A49D194F84811B1B1F8
:10F428001B2B84F8482100F0FC810D2B45D038684F
:10F4380088F801900AF050F80028E3D1AA4650460F
:10F448000AAA70495D4614F07FF9FFF718B97D2BB9
:10F4580000F0F38394F84C2122B180F02003DBB252
:10F4680084F84C1194F84721062A10D8B4F84A11A8
:10F4780038681944A4F84A11A118013281F85031AA
:10F4880084F847210AF028F80028BBD1D6E7B4F859
:10F498004A2188F8019013449BB21A0A52FA83F35E
:10F4A800FF2BA4F84A31386802D1574DA3E73868D2
:10F4B8000AF012F80028A5D1C0E73868A4F84A2154
:10F4C8000AF00AF800289DD1B8E794F8B832C4F8D1
:10F4D800B452012B40F2098394F8B9224B49981889
:10F4E80001EB8001013202F001024E6A84F8B92270
:10F4F800BEB1474F0B970DF14808123FA52348F8B6
:10F50800207D802284F8103115232946404684F84E
:10F51800112184F81231B047002840F06B8294F82A
:10F52800B8323C4A013382FB0312A2EBE37202EBCE
:10F5380042029B1A84F8B832FFF7E2B8364A374BD2
:10F5480092F80BE0029A1B881068D4F834213449E9
:10F55800801A4FF47A72DFB202FB0EF21B0A8F7721
:10F568000F7590424FF00007CB774B758F700F7176
:10F5780080F0A8822B4B2C481A689B68C4F830513D
:10F5880080FB02E7D21780FB03E0C2EBA702DB1780
:10F59800C3EBA00310124FEA232C4FF0F40E0A77A6
:10F5A8000127487781F8203030207522782381F8A8
:10F5B80021C081F81AE0CF7681F8220081F8232053
:10F5C80081F82430FEF7EDBFDFF86490D9F8000029
:10F5D80009F076FF00283FF471A8D9F8000001214E
:10F5E80009F06AFF0222002387F8742088F80030A7
:10F5F800FFF764B8C44F0020184F0020F4600020C3
:10F60800542100209A220020A422002090FB020806
:10F618007922002056555555B85E0020045E00201A
:10F62800944F0020F05D0020676666660C0000209D
:10F63800EC3000205E209047D8F800300220984730
:10F64800D64BD74AB3F94C3082FB03124FEAE37921
:10F65800C9EBA2090FFA89F95FFA89F014F052FB95
:10F66800C9F3072014F04EFBD8F800305E20984705
:10F67800D8F8003003209847CA4B1B78D90740F1C7
:10F6880020810EF053F9C84B9FEDC87AD3ED037A69
:10F6980067EE877AFCEEE77ACDED027ABDF808309E
:10F6A800002800F06083D8B21F0A14F02BFB3846FC
:10F6B80014F028FBBE4B1B78042B74D0DFF820A372
:10F6C800B4F82E219AF80010DFF8189392FBF1F3A2
:10F6D80001FB13239BB2B9F80020A4F82E311F01B7
:10F6E800BFB2642303FB02134900B3FBF1F347EAFB
:10F6F8000327C3F303225E20D8F80030BFB21743B4
:10F708009847D8F8003006209847F8B214F0FAFA6B
:10F71800380A14F0F7FAA74AB4F82E31517AB9F832
:10F72800009001330129A4F82E3100F08C85537B19
:10F7380009EB89091FFA89F9002B40F0B383D8F83F
:10F7480000309D4F5E209847D8F800303A209847FF
:10F75800A7FB09377F091FFA87FA5FFA8AF014F0C6
:10F76800D1FA4FEA1A2014F0CDFAD8F800305E200A
:10F778009847D8F800303B209847642303FB179339
:10F788009BB28748053380FB0320DB17C3EBA0003F
:10F79800C0B214F0B7FA002014F0B4FA874FBB795E
:10F7A800002B40F04C8394F82C31D8F80020FEF759
:10F7B800E5BEDFF834929FED828A4FF0240A5E207E
:10F7C80090475046D8F8003098477E4BF9EC016ACC
:10F7D8009B8A07EE103AF8EEE66AB8EEC77A0AF1A5
:10F7E800010AC6EE877A5FFA8AFA67EE887AFDEE32
:10F7F800E77ACDED027ABDF908B05FFA8BF014F024
:10F8080081FACBF3072014F07DFABAF1270F02D062
:10F81800D8F80020D3E794F82C31D8F80020FEF768
:10F82800AABE386809F058FE00287FF400AE386890
:10F8380084F8469188F8019009F04EFE00287FF47C
:10F84800E1ADFBE5FCF754F95F4B1B68A0EB030B3C
:10F8580040F6B8339B4500F2E5815C4B1A793A2AA9
:10F8680000F01C84002388F80030FEF727BF3868B2
:10F8780084F846A184F847A184F8489188F801A043
:10F8880009F02AFE00287FF4BDADD7E594F84411AD
:10F8980094F845314E484A1CFEF7DDBE013A84F81B
:10F8A8006B21FFF711BA013B84F86A31FFF7E4B81E
:10F8B800013B84F873312EE5013F84F87271FFF73C
:10F8C800E4BA3E4A434B1789A3FB0737BF08F8B28F
:10F8D80014F018FA380A14F015FAEBE64FF0000A9B
:10F8E8005E201F6884F82CA19047D8F80030DFF814
:10F8F800FC9017209847504614F004FA364BA3FBA7
:10F9080007239B0BA9FB03125209C2EB0212A3EBBC
:10F918008203D8B214F0F6F9D8F800305E20984780
:10F92800D8F80030182098472C4BA3FB07239B09D5
:10F93800A9FB03125209C2EB0212A3EB8203D8B24D
:10F9480014F0E0F9504614F0DDF9D8F80020FEF77D
:10F958001ABE0024DFF8988027464FF0500A02E0CC
:10F96800DBB283F3118816F804B0601C59463044A2
:10F9780013F0CCFD002840F074810BF101031C4406
:10F98800EFF311838AF31288326E9442E8DB002287
:10F99800DBB2326683F31188FEF76BBF785900201B
:10F9A8006766666685620020C85E0020CDCC4C3E46
:10F9B800E84E0020B85E00201F85EB5184600020CF
:10F9C80000007A44A0600020E02F0020C82F00200B
:10F9D800F8600020CDCCCCCC73B2E745D34D621093
:10F9E800C65E0020045E0020D060002089888888D8
:10F9F8005D3002080A9EBE4240F23A843D4600212C
:10FA080041F2210015F8013B81EA03235A0013F45F
:10FA1800004F80EA020192B289B208BF11464A003B
:10FA280080EA020311F4004F99B293B218BF0B4653
:10FA3800590080EA010213F4004F89B293B208BF5B
:10FA48000B465A0013F4004F80EA020192B289B2C1
:10FA580008BF11464A0080EA020311F4004F99B228
:10FA680093B218BF0B465A0013F4004F80EA020104
:10FA780092B289B208BF11464B0011F4004F80EAD8
:10FA880003029BB292B208BF1A46510080EA0103F2
:10FA980012F4004F9BB289B218BF1946B542B1D1D2
:10FAA8004046F2F727FDB5490A9DB5486D1A152D50
:10FAB800A8BF15252A461EF027FDB24A94F8B83289
:10FAC80015702EE5B04B029A1B781268C4F83421E1
:10FAD800013B012B3FF64EAD102202238A700B71B9
:10FAE80048E514F0F1F8FEF7BEBDA84A02EB830220
:10FAF800566AFDE414F0D8F801233B70FEF770BD98
:10FB0800A34B1B88D90515D4DA0600F18283980621
:10FB180000F1AB83590600F1B0831A0700F1B083F6
:10FB2800D80700F1B08313F0020F0CBF4FF00408A0
:10FB38004FF00C08974B984A1B78D27803F00103D2
:10FB48000AB143F002035320039313F0E5FD934AEF
:10FB5800128802EB820202EB8202900080B213F05C
:10FB6800C1FD002013F0BEFD8D4A8E491288386809
:10FB7800C2EBC212520081FB023111444FEAE27A11
:10FB8800CAEB612A5FFA8AFA514609F0A9FC99F88A
:10FB98000020039B386848EA03088AEA020A002121
:10FBA80089F800A009F09CFC4146386809F098FCE7
:10FBB80099F80030386888EA0303DBB2194689F8F7
:10FBC800003009F08DFC94F85C31002B7FF4D9AB40
:10FBD8004F2013F0A1FD0FF0D1FB0FF0CFFB0FF07A
:10FBE800CDFB0121386809F07BFC6F4A99F8003099
:10FBF80092F80080386808F00108414683F0010354
:10FC080089F8003009F06CFC99F80030386888EA07
:10FC18000308414689F8008009F062FC94F85C31D9
:10FC2800FFF7AFBB614AB2F85E3100210133A2F899
:10FC38005E3188F80010FEF741BD386884F84C91B1
:10FC480009F04AFC00287FF4DDABFFF7F7BB01465B
:10FC58008446039082460490804605900246FEF74B
:10FC680043BF41463A2013F0ADFB0743FFB284E699
:10FC78004F49504B0093A1F13F074F4B4F4A099111
:10FC880001F8404C0AA84E490897F2F70BFD089F67
:10FC98007B1C08933C70089B2922591C08911A70F8
:10FCA800089BEA22591C08911A70089BC822591C03
:10FCB80008910AA81A701DF0B9FC00F101080AA9F8
:10FCC800424608981EF020FC089A02EB080301330C
:10FCD800089302F80840089B5A1C08921C70089B5D
:10FCE8005A1C08921C70089B5A1C08921C70089B8E
:10FCF8005A1C08921C70089B5A1C08921C70089B7E
:10FD08005A1C08921C70089B5A1C08921C70089B6D
:10FD18005A1C08921C70089B5A1C08921C70089B5D
:10FD28005A1C08921C70089B5A1C08921C70089B4D
:10FD38005A1C08921C70089B0122991812A8089155
:10FD48001A7050F8283DDB1B3B7011F041F9174B36
:10FD58003470C3F8AC52FEF7C7BCC4F8385187F802
:10FD68000080FEF73DBC3A68D2067FF59CAC07469A
:10FD78009BE409F0A1FBFEF748BC00BF6422002009
:10FD8800B82D0020CD2D0020E84E002090FB020861
:10FD9800E860002085620020EC4E0020045E002010
:10FDA800E44E002003082080443B0020542100201A
:10FDB8004C5E002038630020701F0308781F03087A
:10FDC800841F0308A54B0B93A3F1400800222121AF
:10FDD800A3F13D0903F8402C88F8021088F80120A7
:10FDE800CDF828900DF08EFD9D4B9E4A1B889E49AC
:10FDF80000280ABF114603270427580500F113827B
:10FE0800DA0700F1378203F00203984A002B1CBF7F
:10FE1800032711463A4696481EF076FB09EB07037E
:10FE280012A8944A013340F8203D9B1A002209F891
:10FE3800072088F8013011F0CBF8FEF7CEBCD8F8CF
:10FE48000030DFF84CA2DFF840925E209847D8F8DF
:10FE5800003028209847DAF8003089FB0329DB179F
:10FE6800C3EBA9095FFA89F013F04CFFC9F3072027
:10FE780013F048FFD8F800305E209847D8F80030D3
:10FE8800042098473B89002B40F0D081DAF80870AD
:10FE980087F31007F8B213F035FFC7F3072013F004
:10FEA80031FF80E49AF8003099FBF3F947E4724A8D
:10FEB800D278002A0CBF4FF004094FF00509FFF76C
:10FEC8000AB90123D9F800003B7009F0FDFA07468A
:10FED800D9F8000009F0F8FA7F067EF481AB8E2885
:10FEE8007EF47EAB9AF80030002B7EF495AB634B22
:10FEF800634A1A602D2384F83C31FEF778BB574AD1
:10FF0800604B0B920DF14808A2F13D0048F8200D16
:10FF18001988DFF87C91A2F1400300204FF00A0E07
:10FF280002F8400C082283F801E040469A70F2F784
:10FF3800BBFAD9F800305449DA1781FB0313C2EB36
:10FF4800A30399B24046F2F7AFFA01F05BFCD9F887
:10FF580008900A9B4FEA1942591C0A911A700A9B89
:10FF68004FEA1922591C0A911A700A9B5A1C0A92C4
:10FF780083F800900A9B5A1C0A921870404611F0A8
:10FF880027F8FEF727BCDFF810919FED408AB9F9F2
:10FF98000230324A0B9207EE903AF8EEE77A0DF10A
:10FFA800480867EE887AA2F14003FDEEE77AA2F1ED
:10FFB8003D0148F8201D02F8400C0822CDED027AD8
:10FFC8005A701E229A70BDF808104046F2F76CFA73
:10FFD800B9F9003007EE903AF8EEE77A404667EE56
:10FFE800887AFDEEE77ACDED027ABDF80810F2F7CF
:08FFF8005BFAB9F9043007EED1
:020000040801F1
:10000000903AF8EEE77A404667EE887AFDEEE77AB6
:10001000CDED027ABDF80810F2F74AFA404610F02A
:10002000DBFFFEF7D8BB1C4B8046B3F900A0642071
:10003000FEF761BC154B194A1B88927903EB8303C9
:1000400003EB83034FEA83081FFA88F8002A40F085
:1000500027814FF0FF330FFA83FA01F0D7FB40B24C
:10006000FEF749BC4C5E0020E8600020541F0308E6
:100070005C1F03086C1F03080F5E00200D5E00204C
:10008000EC4E002000610020944F0020045E002010
:100090006766666658A08B41F05D00208460002092
:1000A0009860002099780393184605F051FF0028C6
:1000B0007FF4DCABCA49CB4FCB4ACC4C0988DFF884
:1000C00048939368F9611168B4F85E21F863C7F842
:1000D0006CB0FB64F962D9F80000FA6509F000F829
:1000E000834600287EF4E9AA5146D9F8000009F0B9
:1000F000E7F9039B94F86021DB780493642A4FF0BE
:10010000040387F8743040F0E28094F86131DFF83E
:10011000FCA2072B08BF84F861B194F86121069214
:1001200007EB021BDBF80410059108461DF082FA6C
:10013000DBF8083003935FFA80FB18461DF07AFA6B
:10014000C3B20BEB0300069A0599059308308AF8B1
:10015000070022F00F008AF80A0002F00F0203EBFA
:10016000CB008AF80D208AF80E005A460AF10F00DB
:100170001EF0CEF9059B03990BF109001A460AF10E
:10018000060318441EF0C4F99AF8073003F1010B76
:10019000D3B1013B5FFA83FC0CF1080CDFF864E299
:1001A000D4440AF10700002310F8011B59408B00CA
:1001B000CA0883EA410302F018024B404EFA02F2E9
:1001C00053408445DBB2EFD1894A04980BF80230E2
:1001D0001EF07AF994F861310022013384F861311C
:1001E00084F860219AF802305BB11AF80610D9F849
:1001F000000009F079F901369AF80230F6B2B342FC
:10020000F3D894F860310322013384F8603187F821
:10021000742088F80020FFF7DDB94FF034088DE432
:1002200011469446039292460492FEF761BC03275E
:100230007049F3E501F0EAFA13F068FD002013F0CD
:1002400065FD94F82C31D8F80020FEF79BB9D8F85A
:1002500000305E209847D8F80030392098475FFA80
:1002600089F013F053FD4FEA192013F04FFDFFF70B
:1002700099BA4FF0240861E4002115E45E4904278F
:10028000CCE54FF0100859E44FF0200856E44FF049
:10029000080853E41146944603929246FEF728BCA0
:1002A000514B1B68D7E611469446FEF721BC114618
:1002B00094460392FEF71CBC1146FEF719BC11468A
:1002C00094460392924604929046FEF711BC97F82A
:1002D0007530DFF838A10596190704BF0133DBB28A
:1002E000072B28BF01234FEA031B07EB0B024349EF
:1002F000107C00228AF80A2011F800C05FFA8BF205
:1003000003920AF10D02039E07EB0B013043BCF18F
:10031000010F1070C96802F101000ED9ACF102069C
:10032000F6B206F1020E9644024602F8011B72452F
:100330004FEA1121F9D101363044BB4421F060026B
:1003400001339BF81110DBB20A43082B027000F155
:1003500001025DD04FEA031B07EB0B00274E007C28
:10036000274916F800C0039E511A06F1100E01EB42
:100370000C0606965FFA8EF60396069E132EC2DDD5
:10038000059EDFF86CE0C9B28A1DD2B242F040008F
:100390008AF8070002F1010BCAB14A1DD2B2083235
:1003A000524403920EF1010C00221CF8010B504044
:1003B000820082EA4002C1084240124801F018015E
:1003C00040FA01F14A4003996145D2B2EDD1049857
:1003D0000BF80E2087F875301EF076F802E700BFA4
:1003E000045E00200C000020F05D0020542100205D
:1003F0008A430020601F0308641F030890FB020863
:10040000914300200007090EEC30002084430020B7
:100410000149059E511AB4E79143002008B50CF03C
:100420007BFD024B024ADA60FEE700BF00ED00E010
:100430000400FA05024A034B127819780FF06EBDDA
:10044000C81F0020C91F00202DE9F04F2DED028BA1
:10045000A0F10A0389B00C46ED2B00F26086DFE8BC
:1004600013F022015E065E065E065E065E065E060E
:100470005E065E065E065E065E065E065E065E065C
:100480005E065E065E065E065E065E065E065E064C
:100490005E062F025E065E065E062C065E065E06A1
:1004A0005E0699015E0656015E063E015E06330158
:1004B0005E0628025E0603025E06EF015E065E0629
:1004C0005E06EA01E4015E06D2015E065E06CC012C
:1004D0005E06A5015E065E065E068A045E065E0690
:1004E0005E065E066C045E0602015E063B0629059A
:1004F0005E065E065E065E065E065E065E06FD043F
:100500005E06CF045E069C045E0665055E064A062E
:100510005E065E065E065E060503F105EA05B905A0
:10052000EE005E065E062803A6025E066F02E90282
:100530005E065E065E065E06DE025E065E06BD02C4
:100540005E065E065E06AF02F303BB037A035E0639
:100550005E065E066C035E065E064C035E065E0685
:100560005E065E065E065E065E065E065E065E066B
:100570005E065E065E065E065E0605035E065E06B7
:100580005E065E065E065E065E065E065E065E064B
:100590005E065E065E065E065E065E065E065E063B
:1005A0005E065E065E065E065E065E065E065E062B
:1005B0005E065E065E065E065E065E065E065E061B
:1005C0005E065E063E035E065E065E065E065E062E
:1005D0005E065E065E065E065E065E065E065E06FB
:1005E0005E065E065E065E065E065E065E065E06EB
:1005F0005E065E065E065E065E065E065E065E06DB
:100600005E065E065E065E065E065E065E065E06CA
:100610005E065E065E065E065E065E065E065E06BA
:100620005E065E065E065E065E065E065E066204A8
:1006300038045E065E065E065E065E060904AF4E80
:10064000337853B1AE4F002537F8021F2046F1F73B
:1006500055FF33780135AB42F6DC012009B0BDEC23
:10066000028BBDE8F08FA54E3378002BF5D0A54F57
:100670000025B846236817F81520591C21601A7008
:1006800098F8011001EB810101EB810101F2EE21EB
:1006900089B22046F1F732FF33780135AB4208F1D9
:1006A0000208E7DCD9E7984D28461CF0C3FF002874
:1006B000D3DD2B460544226813F8011B501C9D42D4
:1006C00020601170F7D1C8E7904D05F1800655F80C
:1006D000041F2046F1F7FAFEAE42F8D1BDE78C4D7B
:1006E00005F14006B5F880102046F1F707FF2368B2
:1006F00095F88220591C21601A70236895F8832090
:100700000435591CAE4221601A70EBD1A5E7814D2A
:100710000B682A7A591C21601A70A98B2046F1F7C0
:10072000EDFE298B2046F1F7E9FE698B2046F1F7B3
:10073000E5FE2368EA7C591C21601A70A98C2046CA
:10074000F1F7DCFEE98C2046F1F7D8FE2368AA7F9A
:10075000591C21601A70236895F82020591C2160CB
:100760001A70698C2046F1F7C9FE2368EA7A591C91
:1007700021601A70E9682046F1F7A8FE23682A7CF8
:10078000591C21601A70236895F82120591C21609A
:100790001A7062E70B68604A581C11782060197063
:1007A00023685278591C21601A7056E70B685A4A20
:1007B0005A4D11785A4A581C206019701168204609
:1007C000F1F784FE2368534A591C127A21601A708B
:1007D00029882046F1F792FEA9882046F1F78EFE7F
:1007E00029892046F1F78AFE20460021F1F786FE8E
:1007F00020460021F1F782FE2FE7084608224549EE
:10080000F1F74CFE29E70B68464A474990785D1C92
:100810002560187023685278581C20601A7023686D
:100820000A79591C21601A7017E70B680122991880
:1008300021601A7011E708460021F1F747FE0CE726
:100840003A4D3B4E05F1200795F90210394B93F9CB
:1008500006208A4203F1080300F064849E42F6D128
:100860000835BD42F0D1F8E6334B03F15A05226852
:100870005979501C2060117022681978501C206032
:10088000117022685978501C206011702268997884
:10089000501C206011702268D978501C20601170A3
:1008A000226819790633501C9D4220601170DED1F8
:1008B000D3E60B68174A591C527D21601A70CCE6AA
:1008C0001E4D05F15006287817F090FC2368027A37
:1008D000591C21601A7023686A78591C21601A70AB
:1008E0002368AA78591C21601A702368EA780435B5
:1008F000591CAE4221601A70E5D1AEE6AC2E002044
:10090000BA4E00205C310020C83C0020104D002071
:10091000144D0020D46600202C3D0020482C0020DF
:10092000C46400200C3D0020CC1F00200067002084
:100930005443002034430020DC3800205030002095
:10094000AF4D0B682A68591C127821601A702B6809
:1009500022689978531C2360002311702A6821684B
:100960001A4401335279481C032B20600A70F5D1D8
:1009700023682A68591C127A21601A7023682A6831
:10098000591CD27821601A7023682A68591C127980
:1009900021601A702B6820465989F1F7AFFD2A684B
:1009A0002368527A591C21601A702A68F8E620469A
:1009B0000021F1F78BFD20460021F1F79FFD4CE669
:1009C000904D08462988F1F799FD69882046F1F78E
:1009D00095FDA9882046F1F791FD3EE68A4D05F187
:1009E0006006A9882046F1F789FDE9882046F1F7DD
:1009F00085FD29892046F1F781FD2368AA7A591CD3
:100A000021601A702368EA7A591C21601A7055F81F
:100A10000C1B2046F1F75AFDB542E2D11DE67B4999
:100A200052232268501C2060137011F8013F002BE4
:100A3000F7D112E6764800232268056803EB4301EC
:100A4000561C6D5C26601570026825680A446E1C91
:100A5000527826602A70026825680A440133927829
:100A6000691C0A2B21602A70E6D1F6E50025814633
:100A7000DFF8C881DFF8C8B10495039505950695A0
:100A800001214FF6FF7A05E001350B2D00F0688358
:100A900018F9011F4F1C4AFA05F3F5D0DE07F3D50C
:100AA000BBF800302B41D807EED505A8F2F7DAF8ED
:100AB000EAE7584D08462988F1F720FD6988204665
:100AC000F1F71CFDB5F90430534AD91782FB032313
:100AD000C1EBA301204689B2F1F710FDBDE50B681B
:100AE0004E4A591C1278216005A81A70F1F7F6FBDE
:100AF00023685A1C22601870AFE50B68484F591CD8
:100B00003A7821601A703B78002B3FF4A6AD00259F
:100B1000EEB2304612F058FB23684278591C21602F
:100B200030461A7012F050FB01892046F1F7E6FCBE
:100B30003B780135AB42EBDC8FE53A4D0846298A1C
:100B4000F1F7DCFC698A2046F1F7D8FCA98A204637
:100B5000F1F7D4FC81E5DFF8ECE00027FEB2714646
:100B600000232268501C206016702268501C2060F0
:100B70001370226811F8010F0133551C062B2560F4
:100B80001070EED10137062F0EF1060EE6D1264980
:100B900000232268501C206017702268501C2060BF
:100BA0001370226811F8010F0133551C0B2B2560BF
:100BB0001070EED123681D4A581C0721206019705F
:100BC00023680021581C20601970236892F8F020D7
:100BD000591C21601A7040E50B68154A15491078B8
:100BE000154A5D1C2560187023688978581C2060A0
:100BF000197023689278591C21601A702DE500BF86
:100C0000F0600020743E002024370020C4FB02085E
:100C1000EC6000209860002067666666F63200206F
:100C2000565E0020E43F0020F74D0020144D0020C8
:100C3000F05B0020EC3C0020FC3C0020F4FB0208B0
:100C4000E8600020D34D00200A68AC4BAC4918780E
:100C5000551C2560107022685878551C256010704E
:100C600022689B78501C206013702046C988F1F7D9
:100C700045FCF2E405A8F1F731FB00283FF4EDACA8
:100C8000BDF814102046F1F739FC23689DF81620B2
:100C9000591C21601A7023689DF81720591C216087
:100CA0001A7023689DF81820591C21601A70236857
:100CB0009DF81920591C21601A7023689DF81A208C
:100CC000591C21601A702046BDF81C10F1F716FC63
:100CD000C3E48C4B03F1700522681978501C206026
:100CE000117022685978501C206011702268997820
:100CF000501C206011702268D978501C206011703F
:100D000022681979501C2060117022685979501C92
:100D100020601170226899790733501C9D42206031
:100D20001170D9D199E4784D0846E989F1F7E6FBCD
:100D3000A9892046F1F7E2FB8FE40B68734D591C3B
:100D40002A7921601A7023686A79591C21601A7007
:100D500029882046F1F7D2FB2368AA79591C216023
:100D60001A7069882046F1F7C9FB2368EA79591C93
:100D700021601A7071E40B6800255A1C0A60204635
:100D800029461D70F1F7A2FB29462046F1F79EFB8C
:100D900029462046F1F79AFB5FE45D4E0B687279B5
:100DA0005C4D591C21601A702B682046198CF1F794
:100DB000A5FB2B682046D98BF1F7A0FB7189204653
:100DC000F1F79CFBB1892046F1F798FB2B68204690
:100DD000598CF1F793FB2B682046998CF1F78EFB29
:100DE000F1892046F1F78AFB318A2046F1F786FB2C
:100DF0002A68236892F82620591C21601A702CE476
:100E0000434EF378002B00F07E820B680822591CB9
:100E100021601A7023680122991821601A702368D2
:100E20003D4D591C2A7921601A702368AA78591CF3
:100E300021601A7029882046F1F760FBE989204675
:100E4000F1F75CFB2368F279591C21601A70236862
:100E5000EA78591C21601A70FFF7FFBB0FF042F8C7
:100E6000FF28054600F06B8208A8002300F80C3D1F
:100E70000FF00AF82268294B511C21601570226876
:100E80001978501C2060117022685978501C20601D
:100E9000117022689978501C2060117022689DF8AA
:100EA0001410501C2060117020469988F1F726FB21
:100EB000FFF7D3BB0B681A4D591C012221601A7031
:100EC0002368AA78591C21601A700AF0EBF923688C
:100ED000144A15495E1C26601870B1F90010B2F969
:100EE0000000F1F785FC23685A1C226018702988DD
:100EF0002046F1F703FBFFF7B0BB00BFE43C002046
:100F0000743E0020E4370020EC3C00208C3E0020A2
:100F1000F05B0020EC600020E43F00208C620020A9
:100F200092640020523B0020543B002020460021C8
:100F3000F1F7E4FA20460021F1F7E0FA204600211B
:100F4000F1F7DCFA2368A64D00265A1C22601E70B9
:100F500023682A68591C92F82C2021601A70236893
:100F60002A68591C92F8362021601A7023682A6872
:100F7000591C92F8372021601A7023685A1C22608D
:100F80001E7023685A1C22601E7023685A1C22603F
:100F90001E702B682046598FF1F7B0FA2B68204657
:100FA000198FF1F7ABFA23682A68591C92F82E20A2
:100FB00021601A7023685A1C22601E702B6820461C
:100FC000598EF1F79BFA2B682046998EF1F796FA25
:100FD000FFF743BB834D844E9FED848ADFF84C823C
:100FE000DFED838A05F120070EE0FCEEE77ACDED18
:100FF000017ABDF8041020460435F1F77FFAAF42BC
:1010000006F118063FF429AB717C0029F3D0794B27
:10101000D5ED007A1B78012BE7D1774B1B68DB04F9
:1010200040F16781F5EE407AF1EE10FA40F08F81E1
:1010300040F2DC51DFE7084610227049F1F72EFA42
:10104000FFF70BBB6E4B9B8AB3F5006F00F2598123
:10105000B3F5806F00F27981B3F5007F34BF0127CB
:101060000227684D05F10C0655F8041B91FBF7F1BA
:10107000204689B2F1F742FAAE42F5D1624D634F94
:1010800005F10C06B5EC010AD7ED077A80EE270AC8
:101090001DF07EFB81B22046F1F730FAB542F1D166
:1010A0005B4D05F10C0655F8041B204689B2F1F79B
:1010B00025FAB542F7D1FFF7D0BA564D0846298830
:1010C000F1F71CFAA9882046F1F718FA2989204679
:1010D000F1F714FAFFF7C1BA0B6800255A1C0A6031
:1010E0001D700B685A1C0A601D700B685A1C0A6040
:1010F00029461D7049E60B68474A4849D078484A56
:101100005D1C2560187023684979581C206019708F
:101110002368D278591C21601A70FFF79EBA00200C
:10112000FFF79CBA23685A1C226019702988204650
:10113000F1F7E4F92368EA78591C21601A702368F2
:101140002A79591C21601A702368AA79591C2160D8
:101150001A7023686A79591C21601A70FFF780BBE6
:10116000DFF8CCA000254FF0A8080135C5F120021A
:1011700008FA02F2A5F120032AFA05F6164328FA26
:1011800003F31E43282D06F001024FF000030BD09D
:101190001343EAD0E8B20CF0C7FB0028E5D029469B
:1011A00005A8F1F75FFDE0E71E4B1B78DA0700F1B9
:1011B000B68000251C4E2F4602E00135282D39D07F
:1011C00029463046F1F75EFD0028F6D0294605A8ED
:1011D000F1F758FD002840F087800137EDE700BFA8
:1011E000EC6000200C3B0020243F00200000404227
:1011F00000E0824408400020145C0020FC3A0020FB
:10120000A0600020D0600020085C002078590020F9
:10121000C83E0020482C0020EC3C00206C540020EC
:10122000FC3C00208562002074660020DB9B91411D
:1012300090E33FF4644B654DB3F850102046F1F74E
:101240005DF900212046F1F759F9614B19684B010E
:1012500003F02002C1F340031343C1F3800243EAC9
:101260004203C1F3C00243EA8203C1F3401243EADE
:10127000C20301F0100119432046F1F73FF903A919
:1012800004222046F1F70AF923682978514A581CAC
:101290002060197011886429A8BF64212046F1F7E5
:1012A0002DF9B9F1960F3FD000212046F1F726F92C
:1012B0002168B7F1190348BFA7F11203A3F3C403D0
:1012C0004A1C226020461A460B7004A9F1F7E6F882
:1012D0002368414A581C112120601970204611686A
:1012E000F1F7F4F8FFF7B9B9394603A8F1F7BAFCFA
:1012F00073E7F4EEC87AF1EE10FA44DA4FF47A713B
:1013000079E60827ADE60B68B178344A581C2060AE
:10131000197023681278591C21601A707FE5059BAB
:1013200043F00103059344E723680322591C21601D
:101330001A7023686A78591C21601A70B8E723680C
:101340005A1C22601870FFF788B9042789E6F4EE6A
:10135000C87AF1EE10FA3FF56BAEF4EEE87AFDEEE6
:10136000E77AF1EE10FA17EE901A1ED86FF4F973BF
:10137000303903FB01F140F2E73391FBF3F101F265
:10138000DB5189B237E6FDEEE77A40F2E73217EE3D
:10139000903A303B02FB03F388FB0312D917C1EBF1
:1013A000622101F2E93189B225E640F2F313A1F599
:1013B000836103FB01F140F2E73391FBF3F101F2AA
:1013C000DD5189B217E600BF2801002032630020FA
:1013D0009460002022370020E4600020E03C0020E0
:1013E00038B5094D2B8823EA0000834228800AD0B3
:1013F000064B1421FF220E2002241C7059709A7093
:1014000016F00CFD288838BDE86000201C3A00204A
:1014100038B5094D2B881843834228800AD0074BE2
:101420001421FF220E2002241C7059709A7016F0AD
:10143000F5FC288838BD00BFE86000201C3A002079
:10144000024A136818431060704700BFE460002030
:1014500030B4034600F12405064C07CC0C3343F8A6
:101460000C0C43F8081C43F8042CAB42F4D130BCFC
:10147000704700BF00FC0208034B33F80C2F0280BA
:101480009B788370704700BF00FC0208084B196806
:1014900061B130B45D68074C642202FB05F2B2FB17
:1014A000F1F2228030BC002018605860704700BF05
:1014B0001424002022370020624B1B78002B3AD0E6
:1014C0002DE9F041604B614D9B79AC68A860013B10
:1014D00082B0041B032B00F28380DFE803F03102AB
:1014E00029290CF027FA002800F08280584B59492E
:1014F0001B78B5F84220D1ED037AEA64DB0700F1EE
:10150000848002FB04F007EE900ADFED536A534B30
:10151000B8EEE77AD5ED127A5A60E7EE267A1A60CD
:10152000BDEEE77AC5ED127A85ED117A83ED027A88
:1015300002B0BDE8F081494A136053609360704780
:10154000474A484BD279DFF8308133F81220B8F996
:1015500002304548B8F9001092B207EE902A40F6E2
:10156000E44707FB02F6C3EB1633B8EE670A4FF405
:101570007A7606FB03F393FBF1F3AB61EEF7E0FE43
:10158000D5F818E0D5ED047ADFED336AB8F902201A
:10159000324BB8F900C0C3F804E00EFB04F007EECC
:1015A000100AB8EEC77ABCEEC06AE7EE267A8DED77
:1015B000016ABDF80410C5ED047ABDEEE77A07FBB9
:1015C00001F7C2EB173706FB07F683ED027A96FBAD
:1015D000FCF685ED037A6E611E6002B0BDE8F08115
:1015E0001E4B00221A605A609A6002B0BDE8F0817A
:1015F0001E4B1B68DE067FF579AF154BB5F8422010
:101600001B78EA64D9070FD47BE7FDEEE77A184E22
:1016100017EE900AA0F57A7101FB01F386FB030631
:10162000D817C0EB26100844B5F94010114B00FB49
:1016300001F083FB0013C017C0EBA3100244EA645F
:101640005FE700BFC65E00208460002014240020F5
:1016500085620020C85E00202FE33E31F05D00204F
:101660007C6600209C66002030240020145C002052
:101670001F85EB51D34D6210DC3C0020F0B5244BAC
:101680005B79012B83B00ED0224900230B804B8065
:10169000214B1B78022B04D1204B48880A881880E4
:1016A0005A8003B0F0BD1E4A1E4B92781E4D33F88F
:1016B0001240A4B207EE904A05F15400B8EE670A52
:1016C000EEF73EFE194A1349107896785378FCEEEF
:1016D000C07A00EB4010CDED017ABDF8042044F64D
:1016E000FB77C3EB033300FB027200FB0474B2FB15
:1016F000F3F2B4FBF3F3B2FBF6F2B3FBF6F392B200
:101700009BB2A5F85020A5F852300A804B80BFE765
:1017100084600020045E0020A85E0020AC5E0020F3
:101720007C6600209C660020142400202D6300208D
:10173000F8B5254D25496879254C264B264E0422BF
:1017400064270A7001284FF0000184F8782084F89B
:101750008170A4F87A10A4F87C1084F88010C4F882
:10176000841031701980598020D0A9791B4A002338
:101770000129136084F888305360936007D00229F0
:1017800004D1174A636453609360F8BDF8BD154AED
:10179000E36053609360D3609FED130A02F1100081
:1017A0004CF25031BDE8F840F1F718B9282204F1A5
:1017B00050001DF0AAFF4CF250319FED0C0A04F1CD
:1017C0005400F1F70BF9D0E784600020E84E0020C8
:1017D00014240020045E0020C65E0020F05D00207E
:1017E0005824002020240020CDCCCC3ECDCCCC3DB4
:1017F000044B587920B1044B1878003018BF0120F1
:10180000704700BF84600020C65E00201F4B187820
:10181000002839D01E4A1389FBB11E4A9FED1E6A6B
:10182000D2ED026A07EE903AF8EEE66AF8EE677AD1
:1018300007EE103A77EEE66AB8EEC77A66EE866A89
:10184000C6EE877AFDEEE77A17EE900A6428A8BF05
:10185000642020EAE070C0B2704710B40F4B547897
:101860001B88117804FB1032091B642300FB01F074
:1018700003FB02F3B3FBF0F06428A8BF64205DF81B
:10188000044B20EAE070C0B2704700BFC65E002083
:1018900084600020F05D00200000C842045E00204B
:1018A0002DE9F04F794D81B0FAF726F9D5F890403F
:1018B0000022C5F88C20002C00F0A580237D052B8C
:1018C000074617D9216A23690B44C31A9342B8BF4C
:1018D00005F190010ADBD5E0137D052B0AD9136AC7
:1018E00012691344FB1A002B80F2CC8051F8042FAC
:1018F000002AF1D14FF0010B0023B9461E46C5F86E
:101900008C3098469A46274623E07A6A39693B7DAF
:10191000A9EB0204B4FBF1F40134A4B213FB04F309
:10192000013301369BB2B6B23C83FB82984506D2A6
:10193000BBF1000F01D1012C5FD99846BA46D5F80A
:101940008C30013305EB8302C5F88C30D2F89070EF
:1019500047B3BB68C3B1FC8A002CD6D1396A48466C
:10196000A9EB01019847D0B195F8DC30002B52D19A
:101970003B7DC7F82490013601334FF00102B6B227
:101980003A83FB820124D1E73B6A3A69A9EB03045D
:10199000B4FBF2F4A4B23C8334BBFB8AC6E73C83BD
:1019A000FB8AC3E72B686A683949013316443C4611
:1019B00085E848004F46C1F800A0BAF1000F27D0D3
:1019C000DAF8203095F8DC20AAF81640FB1ACAF89D
:1019D0001C30CAF82090002A35D1DAF80C3048467D
:1019E00001B0BDE8F04F18473B7D13FB04F3013312
:1019F00001369BB2B6B2FB8298E73A7D062A04BF55
:101A00009846BA469BE72B68214A01332B60146045
:101A100001B0BDE8F08FFAF76FF81E4B1E4A1F4C5D
:101A200011681A68A0EB090002EB000E2268C3F8E7
:101A300000E09042A1EB5111014438BF1046164A14
:101A40002060116094E7FAF757F8DAF80C30044692
:101A50009847FAF751F8DAF82C20DAF82830DAF853
:101A60003010001B9042A3EB53130344014438BFD2
:101A70001046CAF82830CAF83010CAF82C0001B055
:101A8000BDE8F08F4FF0000B36E700BF14240020B4
:101A90007C54002014370020183700201C37002009
:101AA000F0B43423184F194A03FB00F3D2F8E06076
:101AB000FC58FD18002E6B684B600C600DDDD2F8F1
:101AC00090309D421DD09032002303E052F8044F25
:101AD000A54216D00133B342F8D10022342303FBD0
:101AE00000700A720369CB60037D4B72836AC56A1A
:101AF000046BC2690A615B094D618C61CB61F0BC0A
:101B000070470122EAE700BF2801002014240020CA
:101B10002DE9F0414E4ED6F8E040112C7ADC002C35
:101B200040F39380D6F89030984273D0012C5DD06A
:101B3000D6F8943098426DD0022C57D0D6F8983011
:101B4000984267D0032C51D0D6F89C30984261D08F
:101B5000042C4BD0D6F8A03098425BD0052C45D051
:101B6000D6F8A430984255D0062C3FD0D6F8A830ED
:101B700098424FD0072C39D0D6F8AC30984249D093
:101B8000082C33D0D6F8B030984243D0092C2DD051
:101B9000D6F8B43098423DD00A2C27D0D6F8B830C9
:101BA000984237D00B2C21D0D6F8BC30984231D097
:101BB0000C2C1BD0D6F8C03098422BD00D2C15D051
:101BC000D6F8C430984225D00E2C0FD0D6F8C830A5
:101BD00098421FD00F2C09D0D6F8CC30984219D09B
:101BE000112C03D1D6F8D030984213D0D6F89050AB
:101BF0004DB32B7D017D8B420FD3164F00253A4606
